 fontmanager

 Timestamp is 6a163894 (Tue May 26 20:19:32 2026)

 Preferred load address is 10000000

 Start         Length     Name                   Class
 0001:00000000 000280bbH .text$mn                CODE
 0002:00000000 000001e4H .idata$5                DATA
 0002:000001e4 00000008H .00cfg                  DATA
 0002:000001ec 00000004H .CRT$XCA                DATA
 0002:000001f0 00000004H .CRT$XCZ                DATA
 0002:000001f4 00000004H .CRT$XIA                DATA
 0002:000001f8 00000004H .CRT$XIZ                DATA
 0002:000001fc 00000004H .CRT$XPA                DATA
 0002:00000200 00000004H .CRT$XPZ                DATA
 0002:00000204 00000004H .CRT$XTA                DATA
 0002:00000208 00000008H .CRT$XTZ                DATA
 0002:0000020c 00000000H .gfids$y                DATA
 0002:00000210 00012ff0H .rdata                  DATA
 0002:00013200 00000000H .rdata$CastGuardVftablesA DATA
 0002:00013200 00000000H .rdata$CastGuardVftablesC DATA
 0002:00013200 000011b8H .rdata$r                DATA
 0002:000143b8 00000004H .rdata$sxdata           DATA
 0002:000143bc 0000007cH .rdata$voltmd           DATA
 0002:00014438 00000334H .rdata$zzzdbg           DATA
 0002:0001476c 00000004H .rtc$IAA                DATA
 0002:00014770 00000004H .rtc$IZZ                DATA
 0002:00014774 00000004H .rtc$TAA                DATA
 0002:00014778 00000008H .rtc$TZZ                DATA
 0002:00014780 00000120H .xdata$x                DATA
 0002:000148a0 00000930H .edata                  DATA
 0002:000151d0 00000104H .idata$2                DATA
 0002:000152d4 00000014H .idata$3                DATA
 0002:000152e8 000001e4H .idata$4                DATA
 0002:000154cc 00000968H .idata$6                DATA
 0003:00000000 00000244H .data                   DATA
 0003:00000244 00000060H .data$r                 DATA
 0003:000002a4 000007dcH .data$rs                DATA
 0003:00000a80 00000b00H .bss                    DATA
 0004:00000000 00000060H .rsrc$01                DATA
 0004:00000060 00000378H .rsrc$02                DATA

  Address         Publics by Value              Rva+Base       Lib:Object

 0000:00000000       ___AbsoluteZero            00000000     <absolute>
 0000:00000000       ___arm64x_extra_rfe_table  00000000     <absolute>
 0000:00000000       ___arm64x_extra_rfe_table_size 00000000     <absolute>
 0000:00000000       ___arm64x_native_entrypoint 00000000     <absolute>
 0000:00000000       ___arm64x_redirection_metadata 00000000     <absolute>
 0000:00000000       ___arm64x_redirection_metadata_count 00000000     <absolute>
 0000:00000000       ___dynamic_value_reloc_table 00000000     <absolute>
 0000:00000000       ___enclave_config          00000000     <absolute>
 0000:00000000       ___guard_check_icall_a64n_fptr 00000000     <absolute>
 0000:00000000       ___guard_eh_cont_count     00000000     <absolute>
 0000:00000000       ___guard_eh_cont_table     00000000     <absolute>
 0000:00000000       ___guard_fids_count        00000000     <absolute>
 0000:00000000       ___guard_fids_table        00000000     <absolute>
 0000:00000000       ___guard_iat_count         00000000     <absolute>
 0000:00000000       ___guard_iat_table         00000000     <absolute>
 0000:00000000       ___guard_longjmp_count     00000000     <absolute>
 0000:00000000       ___guard_longjmp_table     00000000     <absolute>
 0000:00000000       ___hybrid_auxiliary_iat    00000000     <absolute>
 0000:00000000       ___hybrid_auxiliary_iat_copy 00000000     <absolute>
 0000:00000000       ___hybrid_code_map         00000000     <absolute>
 0000:00000000       ___hybrid_code_map_count   00000000     <absolute>
 0000:00000000       ___x64_code_ranges_to_entry_points 00000000     <absolute>
 0000:00000000       ___x64_code_ranges_to_entry_points_count 00000000     <absolute>
 0000:00000001       ___safe_se_handler_count   00000001     <absolute>
 0000:00000100       ___guard_flags             00000100     <absolute>
 0000:00000000       ___ImageBase               10000000     <linker-defined>
 0001:00000000       ??0?$LEReferenceTo@ULookupSubtable@@@@QAE@ABVLETableReference@@AAW4LEErrorCode@@PBX@Z 10001000 f i AlternateSubstSubtables.obj
 0001:000000e0       ??0?$LEReferenceToArrayOf@G@@QAE@ABVLETableReference@@AAW4LEErrorCode@@PBGK@Z 100010e0 f i AlternateSubstSubtables.obj
 0001:00000200       ?getGlyphCoverage@LookupSubtable@@QBEJABVLETableReference@@KAAW4LEErrorCode@@@Z 10001200 f i AlternateSubstSubtables.obj
 0001:00000300       ?isEmpty@LETableReference@@QBEDXZ 10001300 f i AlternateSubstSubtables.obj
 0001:00000320       ?isValid@LETableReference@@QBEDXZ 10001320 f i AlternateSubstSubtables.obj
 0001:00000340       ?process@AlternateSubstitutionSubtable@@QBEKABV?$LEReferenceTo@UAlternateSubstitutionSubtable@@@@PAVGlyphIterator@@AAW4LEErrorCode@@PBVLEGlyphFilter@@@Z 10001340 f   AlternateSubstSubtables.obj
 0001:00000650       ??0?$LEReferenceTo@UDeviceTable@@@@QAE@ABVLETableReference@@AAW4LEErrorCode@@I@Z 10001650 f i AnchorTables.obj
 0001:00000720       ??0?$LEReferenceTo@UClassDefFormat1Table@@@@QAE@ABVLETableReference@@AAW4LEErrorCode@@@Z 10001720 f i ClassDefinitionTables.obj
 0001:00000720       ??0?$LEReferenceTo@UFormat1AnchorTable@@@@QAE@ABVLETableReference@@AAW4LEErrorCode@@@Z 10001720 f i AnchorTables.obj
 0001:000007c0       ?getAnchor@AnchorTable@@QBEXABVLETableReference@@KPBVLEFontInstance@@AAULEPoint@@AAW4LEErrorCode@@@Z 100017c0 f   AnchorTables.obj
 0001:00000ca0       ?getAnchor@Format1AnchorTable@@QBEXABV?$LEReferenceTo@UFormat1AnchorTable@@@@PBVLEFontInstance@@AAULEPoint@@AAW4LEErrorCode@@@Z 10001ca0 f   AnchorTables.obj
 0001:00000d10       ??0ArabicOpenTypeLayoutEngine@@QAE@PBVLEFontInstance@@JJJABV?$LEReferenceTo@UGlyphSubstitutionTableHeader@@@@AAW4LEErrorCode@@@Z 10001d10 f   ArabicLayoutEngine.obj
 0001:00000d50       ??0UnicodeArabicOpenTypeLayoutEngine@@QAE@PBVLEFontInstance@@JJJAAW4LEErrorCode@@@Z 10001d50 f   ArabicLayoutEngine.obj
 0001:00000de0       ??_EArabicOpenTypeLayoutEngine@@UAEPAXI@Z 10001de0 f i ArabicLayoutEngine.obj
 0001:00000de0       ??_EUnicodeArabicOpenTypeLayoutEngine@@UAEPAXI@Z 10001de0 f i ArabicLayoutEngine.obj
 0001:00000de0       ??_GArabicOpenTypeLayoutEngine@@UAEPAXI@Z 10001de0 f i ArabicLayoutEngine.obj
 0001:00000de0       ??_GUnicodeArabicOpenTypeLayoutEngine@@UAEPAXI@Z 10001de0 f i ArabicLayoutEngine.obj
 0001:00000e10       ?accept@CharSubstitutionFilter@@UBEDKAAW4LEErrorCode@@@Z 10001e10 f   ArabicLayoutEngine.obj
 0001:00000e30       ?adjustGlyphPositions@ArabicOpenTypeLayoutEngine@@MAEXQBGJJDAAVLEGlyphStorage@@AAW4LEErrorCode@@@Z 10001e30 f   ArabicLayoutEngine.obj
 0001:00000f50       ?adjustGlyphPositions@UnicodeArabicOpenTypeLayoutEngine@@MAEXQBGJJDAAVLEGlyphStorage@@AAW4LEErrorCode@@@Z 10001f50 f   ArabicLayoutEngine.obj
 0001:00000fd0       ?characterProcessing@ArabicOpenTypeLayoutEngine@@MAEJQBGJJJDAAPAGAAVLEGlyphStorage@@AAW4LEErrorCode@@@Z 10001fd0 f   ArabicLayoutEngine.obj
 0001:000010f0       ?getDynamicClassID@ArabicOpenTypeLayoutEngine@@UBEPBDXZ 100020f0 f   ArabicLayoutEngine.obj
 0001:00001100       ?getFontTable@LayoutEngine@@MBEPBXK@Z 10002100 f i ArabicLayoutEngine.obj
 0001:00001120       ?glyphPostProcessing@UnicodeArabicOpenTypeLayoutEngine@@MAEJAAVLEGlyphStorage@@0AAW4LEErrorCode@@@Z 10002120 f   ArabicLayoutEngine.obj
 0001:000011c0       ?mapCharsToGlyphs@UnicodeArabicOpenTypeLayoutEngine@@MAEXQBGJJDDAAVLEGlyphStorage@@AAW4LEErrorCode@@@Z 100021c0 f   ArabicLayoutEngine.obj
 0001:00001250       ?getFeatureMap@ArabicShaping@@SAPBUFeatureMap@@AAJ@Z 10002250 f   ArabicShaping.obj
 0001:00001260       ?shape@ArabicShaping@@SAXPBGJJJDAAVLEGlyphStorage@@@Z 10002260 f   ArabicShaping.obj
 0001:000015a0       ?reorderMarks@CanonShaping@@SAXPBGJDPAGAAVLEGlyphStorage@@@Z 100025a0 f   CanonShaping.obj
 0001:00001780       ??0?$LEReferenceTo@UClassDefFormat2Table@@@@QAE@ABVLETableReference@@AAW4LEErrorCode@@@Z 10002780 f i ClassDefinitionTables.obj
 0001:00001820       ??0?$LEReferenceTo@UClassDefinitionTable@@@@QAE@ABVLETableReference@@AAW4LEErrorCode@@@Z 10002820 f i ClassDefinitionTables.obj
 0001:000018c0       ??0?$LEReferenceToArrayOf@UFeatureRecord@@@@QAE@ABVLETableReference@@AAW4LEErrorCode@@PBUFeatureRecord@@K@Z 100028c0 f i Features.obj
 0001:000018c0       ??0?$LEReferenceToArrayOf@UGlyphRangeRecord@@@@QAE@ABVLETableReference@@AAW4LEErrorCode@@PBUGlyphRangeRecord@@K@Z 100028c0 f i ClassDefinitionTables.obj
 0001:000018c0       ??0?$LEReferenceToArrayOf@UTagAndOffsetRecord@@@@QAE@ABVLETableReference@@AAW4LEErrorCode@@PBUTagAndOffsetRecord@@K@Z 100028c0 f i ScriptAndLanguage.obj
 0001:000019f0       ??R?$LEReferenceToArrayOf@G@@QBEABGKAAW4LEErrorCode@@@Z 100029f0 f i ClassDefinitionTables.obj
 0001:00001a20       ?getGlyphClass@ClassDefinitionTable@@QBEJABVLETableReference@@KAAW4LEErrorCode@@@Z 10002a20 f   ClassDefinitionTables.obj
 0001:00001b90       ?hasGlyphClass@ClassDefFormat1Table@@QBEDABVLETableReference@@JAAW4LEErrorCode@@@Z 10002b90 f   ClassDefinitionTables.obj
 0001:00001c90       ?hasGlyphClass@ClassDefFormat2Table@@QBEDABVLETableReference@@JAAW4LEErrorCode@@@Z 10002c90 f   ClassDefinitionTables.obj
 0001:00001da0       ?hasGlyphClass@ClassDefinitionTable@@QBEDABVLETableReference@@JAAW4LEErrorCode@@@Z 10002da0 f   ClassDefinitionTables.obj
 0001:00001e40       ??0?$LEReferenceToArrayOf@G@@QAE@ABVLETableReference@@AAW4LEErrorCode@@IK@Z 10002e40 f i ContextualGlyphInsertionProc2.obj
 0001:00001f30       ??0ContextualGlyphInsertionProcessor2@@QAE@ABV?$LEReferenceTo@UMorphSubtableHeader2@@@@AAW4LEErrorCode@@@Z 10002f30 f   ContextualGlyphInsertionProc2.obj
 0001:00002260       ??_EContextualGlyphInsertionProcessor2@@UAEPAXI@Z 10003260 f i ContextualGlyphInsertionProc2.obj
 0001:00002260       ??_GContextualGlyphInsertionProcessor2@@UAEPAXI@Z 10003260 f i ContextualGlyphInsertionProc2.obj
 0001:000022b0       ?beginStateTable@ContextualGlyphInsertionProcessor2@@UAEXXZ 100032b0 f   ContextualGlyphInsertionProc2.obj
 0001:000022c0       ?endStateTable@ContextualGlyphInsertionProcessor2@@UAEXXZ 100032c0 f   ContextualGlyphInsertionProc2.obj
 0001:000022c0       ?endStateTable@ContextualGlyphSubstitutionProcessor2@@UAEXXZ 100032c0 f   ContextualGlyphSubstProc2.obj
 0001:000022c0       ?endStateTable@ContextualGlyphSubstitutionProcessor@@UAEXXZ 100032c0 f   ContextualGlyphSubstProc.obj
 0001:000022c0       ?endStateTable@IndicRearrangementProcessor2@@UAEXXZ 100032c0 f   IndicRearrangementProcessor2.obj
 0001:000022c0       ?endStateTable@IndicRearrangementProcessor@@UAEXXZ 100032c0 f   IndicRearrangementProcessor.obj
 0001:000022c0       ?endStateTable@LigatureSubstitutionProcessor2@@UAEXXZ 100032c0 f   LigatureSubstProc2.obj
 0001:000022c0       ?endStateTable@LigatureSubstitutionProcessor@@UAEXXZ 100032c0 f   LigatureSubstProc.obj
 0001:000022c0       @_guard_check_icall_nop@4  100032c0 f   MSVCRT:guard_support.obj
 0001:000022d0       ?getDynamicClassID@ContextualGlyphInsertionProcessor2@@UBEPBDXZ 100032d0 f   ContextualGlyphInsertionProc2.obj
 0001:000022e0       ?processStateEntry@ContextualGlyphInsertionProcessor2@@UAEGAAVLEGlyphStorage@@AAJGAAW4LEErrorCode@@@Z 100032e0 f   ContextualGlyphInsertionProc2.obj
 0001:000024f0       ?swapLong@LESwaps@@SAKK@Z  100034f0 f i ContextualGlyphInsertionProc2.obj
 0001:00002510       ??0ContextualGlyphSubstitutionProcessor@@QAE@ABV?$LEReferenceTo@UMorphSubtableHeader@@@@AAW4LEErrorCode@@@Z 10003510 f   ContextualGlyphSubstProc.obj
 0001:00002870       ??_EContextualGlyphSubstitutionProcessor@@UAEPAXI@Z 10003870 f i ContextualGlyphSubstProc.obj
 0001:00002870       ??_GContextualGlyphSubstitutionProcessor@@UAEPAXI@Z 10003870 f i ContextualGlyphSubstProc.obj
 0001:000028c0       ?beginStateTable@ContextualGlyphSubstitutionProcessor@@UAEXXZ 100038c0 f   ContextualGlyphSubstProc.obj
 0001:000028d0       ?getDynamicClassID@ContextualGlyphSubstitutionProcessor@@UBEPBDXZ 100038d0 f   ContextualGlyphSubstProc.obj
 0001:000028e0       ?processStateEntry@ContextualGlyphSubstitutionProcessor@@UAEFAAVLEGlyphStorage@@AAJEAAW4LEErrorCode@@@Z 100038e0 f   ContextualGlyphSubstProc.obj
 0001:00002ac0       ??0ContextualGlyphSubstitutionProcessor2@@QAE@ABV?$LEReferenceTo@UMorphSubtableHeader2@@@@AAW4LEErrorCode@@@Z 10003ac0 f   ContextualGlyphSubstProc2.obj
 0001:00002df0       ??_EContextualGlyphSubstitutionProcessor2@@UAEPAXI@Z 10003df0 f i ContextualGlyphSubstProc2.obj
 0001:00002df0       ??_GContextualGlyphSubstitutionProcessor2@@UAEPAXI@Z 10003df0 f i ContextualGlyphSubstProc2.obj
 0001:00002e40       ?beginStateTable@ContextualGlyphSubstitutionProcessor2@@UAEXXZ 10003e40 f   ContextualGlyphSubstProc2.obj
 0001:00002e50       ?getDynamicClassID@ContextualGlyphSubstitutionProcessor2@@UBEPBDXZ 10003e50 f   ContextualGlyphSubstProc2.obj
 0001:00002e60       ?processStateEntry@ContextualGlyphSubstitutionProcessor2@@UAEGAAVLEGlyphStorage@@AAJGAAW4LEErrorCode@@@Z 10003e60 f   ContextualGlyphSubstProc2.obj
 0001:00003480       ??0?$LEReferenceTo@UClassDefinitionTable@@@@QAE@ABVLETableReference@@AAW4LEErrorCode@@I@Z 10004480 f i ContextualSubstSubtables.obj
 0001:00003480       ??0?$LEReferenceTo@UScriptListTable@@@@QAE@ABVLETableReference@@AAW4LEErrorCode@@I@Z 10004480 f i GlyphLookupTables.obj
 0001:00003550       ?matchGlyphCoverages@ContextualSubstitutionBase@@SADABV?$LEReferenceToArrayOf@G@@GPAVGlyphIterator@@ABVLETableReference@@AAW4LEErrorCode@@D@Z 10004550 f   ContextualSubstSubtables.obj
 0001:000036a0       ?matchGlyphIDs@ContextualSubstitutionBase@@SADABV?$LEReferenceToArrayOf@G@@GPAVGlyphIterator@@D@Z 100046a0 f   ContextualSubstSubtables.obj
 0001:00003730       ?process@ChainingContextualSubstitutionFormat1Subtable@@QBEKABVLETableReference@@PBVLookupProcessor@@PAVGlyphIterator@@PBVLEFontInstance@@AAW4LEErrorCode@@@Z 10004730 f   ContextualSubstSubtables.obj
 0001:00004460       ?process@ChainingContextualSubstitutionFormat2Subtable@@QBEKABVLETableReference@@PBVLookupProcessor@@PAVGlyphIterator@@PBVLEFontInstance@@AAW4LEErrorCode@@@Z 10005460 f   ContextualSubstSubtables.obj
 0001:00005430       ?process@ChainingContextualSubstitutionFormat3Subtable@@QBEKABVLETableReference@@PBVLookupProcessor@@PAVGlyphIterator@@PBVLEFontInstance@@AAW4LEErrorCode@@@Z 10006430 f   ContextualSubstSubtables.obj
 0001:00005970       ?process@ChainingContextualSubstitutionSubtable@@QBEKABV?$LEReferenceTo@UChainingContextualSubstitutionSubtable@@@@PBVLookupProcessor@@PAVGlyphIterator@@PBVLEFontInstance@@AAW4LEErrorCode@@@Z 10006970 f   ContextualSubstSubtables.obj
 0001:00005c60       ?process@ContextualSubstitutionFormat1Subtable@@QBEKABVLETableReference@@PBVLookupProcessor@@PAVGlyphIterator@@PBVLEFontInstance@@AAW4LEErrorCode@@@Z 10006c60 f   ContextualSubstSubtables.obj
 0001:000062f0       ?process@ContextualSubstitutionFormat2Subtable@@QBEKABVLETableReference@@PBVLookupProcessor@@PAVGlyphIterator@@PBVLEFontInstance@@AAW4LEErrorCode@@@Z 100072f0 f   ContextualSubstSubtables.obj
 0001:00006b60       ?process@ContextualSubstitutionSubtable@@QBEKABVLETableReference@@PBVLookupProcessor@@PAVGlyphIterator@@PBVLEFontInstance@@AAW4LEErrorCode@@@Z 10007b60 f   ContextualSubstSubtables.obj
 0001:00007150       ?getGlyphCoverage@CoverageTable@@QBEJABVLETableReference@@KAAW4LEErrorCode@@@Z 10008150 f   CoverageTables.obj
 0001:000075d0       ?process@CursiveAttachmentSubtable@@QBEKABV?$LEReferenceTo@UCursiveAttachmentSubtable@@@@PAVGlyphIterator@@PBVLEFontInstance@@AAW4LEErrorCode@@@Z 100085d0 f   CursiveAttachmentSubtables.obj
 0001:00007960       ?getAdjustment@DeviceTable@@QBEFABV?$LEReferenceTo@UDeviceTable@@@@GAAW4LEErrorCode@@@Z 10008960 f   DeviceTables.obj
 0001:00007a70       _Java_sun_java2d_loops_DrawGlyphListAA_DrawGlyphListAA@20 10008a70 f   DrawGlyphList.obj
 0001:00007a70       _Java_sun_java2d_loops_DrawGlyphList_DrawGlyphList@20 10008a70 f   DrawGlyphList.obj
 0001:00007ae0       _Java_sun_java2d_loops_DrawGlyphListLCD_DrawGlyphListLCD@20 10008ae0 f   DrawGlyphList.obj
 0001:00007b90       _RefineBounds              10008b90 f   DrawGlyphList.obj
 0001:00008040       _initLCDGammaTables        10009040 f   DrawGlyphList.obj
 0001:00008080       _initLUT                   10009080 f   DrawGlyphList.obj
 0001:000081b0       _setupBlitVector           100091b0 f   DrawGlyphList.obj
 0001:00008570       _setupLCDBlitVector        10009570 f   DrawGlyphList.obj
 0001:00008b20       ?process@ExtensionSubtable@@QBEKABV?$LEReferenceTo@UExtensionSubtable@@@@PBVLookupProcessor@@GPAVGlyphIterator@@PBVLEFontInstance@@AAW4LEErrorCode@@@Z 10009b20 f   ExtensionSubtables.obj
 0001:00008c10       ??0?$LEReferenceTo@UFeatureTable@@@@QAE@XZ 10009c10 f i Features.obj
 0001:00008c10       ??0?$LEReferenceTo@UPairValueRecord@@@@QAE@XZ 10009c10 f i PairPositioningSubtables.obj
 0001:00008c40       ?getFeatureTable@FeatureListTable@@QBE?AV?$LEReferenceTo@UFeatureTable@@@@ABVLETableReference@@GPAKAAW4LEErrorCode@@@Z 10009c40 f   Features.obj
 0001:00008dc0       ??0FontInstanceAdapter@@QAE@PAUJNIEnv_@@PAV_jobject@@1PAMJJJPAUTTLayoutTableCache@@@Z 10009dc0 f   FontInstanceAdapter.obj
 0001:00009080       ??_EFontInstanceAdapter@@UAEPAXI@Z 1000a080 f i FontInstanceAdapter.obj
 0001:00009080       ??_GFontInstanceAdapter@@UAEPAXI@Z 1000a080 f i FontInstanceAdapter.obj
 0001:000090b0       ??_ELEFontInstance@@UAEPAXI@Z 1000a0b0 f i FontInstanceAdapter.obj
 0001:000090b0       ??_GLEFontInstance@@UAEPAXI@Z 1000a0b0 f i FontInstanceAdapter.obj
 0001:000090d0       ?CallBooleanMethod@JNIEnv_@@QAAEPAV_jobject@@PAU_jmethodID@@ZZ 1000a0d0 f i FontInstanceAdapter.obj
 0001:000090f0       ?CallIntMethod@JNIEnv_@@QAAJPAV_jobject@@PAU_jmethodID@@ZZ 1000a0f0 f i FontInstanceAdapter.obj
 0001:00009110       ?CallObjectMethod@JNIEnv_@@QAAPAV_jobject@@PAV2@PAU_jmethodID@@ZZ 1000a110 f i FontInstanceAdapter.obj
 0001:00009130       ?NewObject@JNIEnv_@@QAAPAV_jobject@@PAV_jclass@@PAU_jmethodID@@ZZ 1000a130 f i FontInstanceAdapter.obj
 0001:00009150       ?canDisplay@FontInstanceAdapter@@UBEDK@Z 1000a150 f i FontInstanceAdapter.obj
 0001:00009170       ?getAscent@FontInstanceAdapter@@UBEJXZ 1000a170 f i FontInstanceAdapter.obj
 0001:00009170       ?getDescent@FontInstanceAdapter@@UBEJXZ 1000a170 f i FontInstanceAdapter.obj
 0001:00009170       ?getLeading@FontInstanceAdapter@@UBEJXZ 1000a170 f i FontInstanceAdapter.obj
 0001:00009170       ___scrt_stub_for_is_c_termination_complete 1000a170 f i MSVCRT:ucrt_stubs.obj
 0001:00009170       __is_c_termination_complete 1000a170 f i MSVCRT:ucrt_stubs.obj
 0001:00009180       ?getFontTable@FontInstanceAdapter@@UBEPBXK@Z 1000a180 f   FontInstanceAdapter.obj
 0001:000091a0       ?getFontTable@FontInstanceAdapter@@UBEPBXKAAI@Z 1000a1a0 f   FontInstanceAdapter.obj
 0001:00009270       ?getFontTable@LEFontInstance@@UBEPBXKAAI@Z 1000a270 f i FontInstanceAdapter.obj
 0001:00009290       ?getGlyphAdvance@FontInstanceAdapter@@UBEXKAAULEPoint@@@Z 1000a290 f   FontInstanceAdapter.obj
 0001:000092a0       ?getGlyphPoint@FontInstanceAdapter@@UBEDKJAAULEPoint@@@Z 1000a2a0 f   FontInstanceAdapter.obj
 0001:00009320       ?getKernPairs@FontInstanceAdapter@@UBEPAXXZ 1000a320 f i FontInstanceAdapter.obj
 0001:00009330       ?getKerningAdjustment@FontInstanceAdapter@@UBEXAAULEPoint@@@Z 1000a330 f   FontInstanceAdapter.obj
 0001:00009460       ?getScaleFactorX@FontInstanceAdapter@@UBEMXZ 1000a460 f i FontInstanceAdapter.obj
 0001:00009470       ?getScaleFactorY@FontInstanceAdapter@@UBEMXZ 1000a470 f i FontInstanceAdapter.obj
 0001:00009480       ?getSubFont@FontInstanceAdapter@@UBEPBVLEFontInstance@@QBGPAJJJAAW4LEErrorCode@@@Z 1000a480 f i FontInstanceAdapter.obj
 0001:00009490       ?getUnitsPerEM@FontInstanceAdapter@@UBEJXZ 1000a490 f i FontInstanceAdapter.obj
 0001:000094a0       ?getWideGlyphAdvance@FontInstanceAdapter@@UBEXKAAULEPoint@@@Z 1000a4a0 f   FontInstanceAdapter.obj
 0001:00009530       ?getXPixelsPerEm@FontInstanceAdapter@@UBEMXZ 1000a530 f i FontInstanceAdapter.obj
 0001:00009540       ?getYPixelsPerEm@FontInstanceAdapter@@UBEMXZ 1000a540 f i FontInstanceAdapter.obj
 0001:00009550       ?mapCharToGlyph@FontInstanceAdapter@@UBEKK@Z 1000a550 f   FontInstanceAdapter.obj
 0001:00009580       ?mapCharToGlyph@FontInstanceAdapter@@UBEKKPBVLECharMapper@@@Z 1000a580 f   FontInstanceAdapter.obj
 0001:000095e0       ?mapCharToWideGlyph@FontInstanceAdapter@@UBEKKPBVLECharMapper@@@Z 1000a5e0 f   FontInstanceAdapter.obj
 0001:00009640       ?mapCharsToWideGlyphs@FontInstanceAdapter@@UBEXQBGJJDPBVLECharMapper@@QAK@Z 1000a640 f   FontInstanceAdapter.obj
 0001:00009700       ?pixelsToUnits@FontInstanceAdapter@@UBEXAAULEPoint@@0@Z 1000a700 f i FontInstanceAdapter.obj
 0001:00009700       ?pixelsToUnits@LEFontInstance@@UBEXAAULEPoint@@0@Z 1000a700 f i LEFontInstance.obj
 0001:00009740       ?setKernPairs@FontInstanceAdapter@@UBEXPAX@Z 1000a740 f i FontInstanceAdapter.obj
 0001:00009750       ?transformFunits@FontInstanceAdapter@@UBEXMMAAULEPoint@@@Z 1000a750 f   FontInstanceAdapter.obj
 0001:000097f0       ?unitsToPoints@FontInstanceAdapter@@UBEXAAULEPoint@@0@Z 1000a7f0 f i FontInstanceAdapter.obj
 0001:000097f0       ?unitsToPoints@LEFontInstance@@UBEXAAULEPoint@@0@Z 1000a7f0 f i LEFontInstance.obj
 0001:00009830       ?xPixelsToUnits@FontInstanceAdapter@@UBEMM@Z 1000a830 f i FontInstanceAdapter.obj
 0001:00009840       ?xUnitsToPoints@FontInstanceAdapter@@UBEMM@Z 1000a840 f i FontInstanceAdapter.obj
 0001:00009850       ?yPixelsToUnits@FontInstanceAdapter@@UBEMM@Z 1000a850 f i FontInstanceAdapter.obj
 0001:00009860       ?yUnitsToPoints@FontInstanceAdapter@@UBEMM@Z 1000a860 f i FontInstanceAdapter.obj
 0001:00009870       ??0GDEFMarkFilter@@QAE@ABV?$LEReferenceTo@UGlyphDefinitionTableHeader@@@@AAW4LEErrorCode@@@Z 1000a870 f   GDEFMarkFilter.obj
 0001:000098b0       ??1GDEFMarkFilter@@UAE@XZ  1000a8b0 f   GDEFMarkFilter.obj
 0001:000098d0       ??_EGDEFMarkFilter@@UAEPAXI@Z 1000a8d0 f i GDEFMarkFilter.obj
 0001:000098d0       ??_GGDEFMarkFilter@@UAEPAXI@Z 1000a8d0 f i GDEFMarkFilter.obj
 0001:00009900       ??_ELEGlyphFilter@@UAEPAXI@Z 1000a900 f i GDEFMarkFilter.obj
 0001:00009900       ??_GLEGlyphFilter@@UAEPAXI@Z 1000a900 f i GDEFMarkFilter.obj
 0001:00009920       ?accept@GDEFMarkFilter@@UBEDKAAW4LEErrorCode@@@Z 1000a920 f   GDEFMarkFilter.obj
 0001:00009940       ??0GXLayoutEngine@@QAE@PBVLEFontInstance@@JJABV?$LEReferenceTo@UMorphTableHeader@@@@AAW4LEErrorCode@@@Z 1000a940 f   GXLayoutEngine.obj
 0001:00009980       ??_EGXLayoutEngine@@UAEPAXI@Z 1000a980 f i GXLayoutEngine.obj
 0001:00009980       ??_GGXLayoutEngine@@UAEPAXI@Z 1000a980 f i GXLayoutEngine.obj
 0001:000099c0       ?adjustGlyphPositions@GXLayoutEngine2@@MAEXQBGJJDAAVLEGlyphStorage@@AAW4LEErrorCode@@@Z 1000a9c0 f   GXLayoutEngine2.obj
 0001:000099c0       ?adjustGlyphPositions@GXLayoutEngine@@MAEXQBGJJDAAVLEGlyphStorage@@AAW4LEErrorCode@@@Z 1000a9c0 f   GXLayoutEngine.obj
 0001:000099f0       ?computeGlyphs@GXLayoutEngine@@MAEJQBGJJJDAAVLEGlyphStorage@@AAW4LEErrorCode@@@Z 1000a9f0 f   GXLayoutEngine.obj
 0001:00009a70       ?getDynamicClassID@GXLayoutEngine@@UBEPBDXZ 1000aa70 f   GXLayoutEngine.obj
 0001:00009a80       ??0GXLayoutEngine2@@QAE@PBVLEFontInstance@@JJABV?$LEReferenceTo@UMorphTableHeader2@@@@JAAW4LEErrorCode@@@Z 1000aa80 f   GXLayoutEngine2.obj
 0001:00009ac0       ??_EGXLayoutEngine2@@UAEPAXI@Z 1000aac0 f i GXLayoutEngine2.obj
 0001:00009ac0       ??_GGXLayoutEngine2@@UAEPAXI@Z 1000aac0 f i GXLayoutEngine2.obj
 0001:00009b00       ?computeGlyphs@GXLayoutEngine2@@MAEJQBGJJJDAAVLEGlyphStorage@@AAW4LEErrorCode@@@Z 1000ab00 f   GXLayoutEngine2.obj
 0001:00009b90       ?getDynamicClassID@GXLayoutEngine2@@UBEPBDXZ 1000ab90 f   GXLayoutEngine2.obj
 0001:00009ba0       ?getGlyphClassDefinitionTable@GlyphDefinitionTableHeader@@QBE?BV?$LEReferenceTo@UClassDefinitionTable@@@@ABV?$LEReferenceTo@UGlyphDefinitionTableHeader@@@@AAW4LEErrorCode@@@Z 1000aba0 f   GlyphDefinitionTables.obj
 0001:00009c00       ?getMarkAttachClassDefinitionTable@GlyphDefinitionTableHeader@@QBE?BV?$LEReferenceTo@UClassDefinitionTable@@@@ABV?$LEReferenceTo@UGlyphDefinitionTableHeader@@@@AAW4LEErrorCode@@@Z 1000ac00 f   GlyphDefinitionTables.obj
 0001:00009c60       ??0GlyphIterator@@QAE@AAV0@@Z 1000ac60 f   GlyphIterator.obj
 0001:00009d20       ??0GlyphIterator@@QAE@AAV0@G@Z 1000ad20 f   GlyphIterator.obj
 0001:00009de0       ??0GlyphIterator@@QAE@AAV0@K@Z 1000ade0 f   GlyphIterator.obj
 0001:00009ea0       ??0GlyphIterator@@QAE@AAVLEGlyphStorage@@PAVGlyphPositionAdjustments@@DGKABV?$LEReferenceTo@UGlyphDefinitionTableHeader@@@@AAW4LEErrorCode@@@Z 1000aea0 f   GlyphIterator.obj
 0001:00009fc0       ??1GlyphIterator@@UAE@XZ   1000afc0 f   GlyphIterator.obj
 0001:00009fe0       ??_EGlyphIterator@@UAEPAXI@Z 1000afe0 f i GlyphIterator.obj
 0001:00009fe0       ??_GGlyphIterator@@UAEPAXI@Z 1000afe0 f i GlyphIterator.obj
 0001:0000a010       ?adjustCurrGlyphPositionAdjustment@GlyphIterator@@QAEXMMMM@Z 1000b010 f   GlyphIterator.obj
 0001:0000a0b0       ?applyInsertions@GlyphIterator@@QAEJXZ 1000b0b0 f   GlyphIterator.obj
 0001:0000a0d0       ?findFeatureTag@GlyphIterator@@QAEDXZ 1000b0d0 f   GlyphIterator.obj
 0001:0000a150       ?findMark2Glyph@GlyphIterator@@QAEDXZ 1000b150 f   GlyphIterator.obj
 0001:0000a290       ?getCurrGlyphID@GlyphIterator@@QBEKXZ 1000b290 f   GlyphIterator.obj
 0001:0000a2c0       ?getCurrStreamPosition@GlyphIterator@@QBEJXZ 1000b2c0 f   GlyphIterator.obj
 0001:0000a2d0       ?getMarkComponent@GlyphIterator@@QBEJJ@Z 1000b2d0 f   GlyphIterator.obj
 0001:0000a320       ?ignoresMarks@GlyphIterator@@QBEDXZ 1000b320 f   GlyphIterator.obj
 0001:0000a330       ?insertGlyphs@GlyphIterator@@QAEPAKJAAW4LEErrorCode@@@Z 1000b330 f   GlyphIterator.obj
 0001:0000a350       ?isRightToLeft@GlyphIterator@@QBEDXZ 1000b350 f   GlyphIterator.obj
 0001:0000a360       ?next@GlyphIterator@@QAEDK@Z 1000b360 f   GlyphIterator.obj
 0001:0000a3b0       ?nextInternal@GlyphIterator@@AAEDK@Z 1000b3b0 f   GlyphIterator.obj
 0001:0000a500       ?prev@GlyphIterator@@QAEDK@Z 1000b500 f   GlyphIterator.obj
 0001:0000a550       ?prevInternal@GlyphIterator@@AAEDK@Z 1000b550 f   GlyphIterator.obj
 0001:0000a6a0       ?reset@GlyphIterator@@QAEXGK@Z 1000b6a0 f   GlyphIterator.obj
 0001:0000a6d0       ?setCurrGlyphBaseOffset@GlyphIterator@@QAEXJ@Z 1000b6d0 f   GlyphIterator.obj
 0001:0000a710       ?setCurrGlyphID@GlyphIterator@@QAEXG@Z 1000b710 f   GlyphIterator.obj
 0001:0000a750       ?setCurrGlyphPositionAdjustment@GlyphIterator@@QAEXMMMM@Z 1000b750 f   GlyphIterator.obj
 0001:0000a7e0       ?setCurrStreamPosition@GlyphIterator@@QAEXJ@Z 1000b7e0 f   GlyphIterator.obj
 0001:0000a850       ?setCursiveEntryPoint@GlyphIterator@@QAEXAAULEPoint@@@Z 1000b850 f   GlyphIterator.obj
 0001:0000a890       ?setCursiveExitPoint@GlyphIterator@@QAEXAAULEPoint@@@Z 1000b890 f   GlyphIterator.obj
 0001:0000a8d0       ?setCursiveGlyph@GlyphIterator@@QAEXXZ 1000b8d0 f   GlyphIterator.obj
 0001:0000a910       ?coversScript@GlyphLookupTableHeader@@QBEDABVLETableReference@@KAAW4LEErrorCode@@@Z 1000b910 f   GlyphLookupTables.obj
 0001:0000a980       ?coversScriptAndLanguage@GlyphLookupTableHeader@@QBEDABVLETableReference@@KKAAW4LEErrorCode@@D@Z 1000b980 f   GlyphLookupTables.obj
 0001:0000a9f0       ??0GlyphPositionAdjustments@@QAE@J@Z 1000b9f0 f   GlyphPositionAdjustments.obj
 0001:0000aa90       ??1GlyphPositionAdjustments@@QAE@XZ 1000ba90 f   GlyphPositionAdjustments.obj
 0001:0000aae0       ?applyCursiveAdjustments@GlyphPositionAdjustments@@QAEXAAVLEGlyphStorage@@DPBVLEFontInstance@@@Z 1000bae0 f   GlyphPositionAdjustments.obj
 0001:0000ae20       ?setCursiveGlyph@GlyphPositionAdjustments@@QAEXJD@Z 1000be20 f   GlyphPositionAdjustments.obj
 0001:0000aed0       ?setEntryPoint@GlyphPositionAdjustments@@QAEXJAAULEPoint@@D@Z 1000bed0 f   GlyphPositionAdjustments.obj
 0001:0000af90       ?setExitPoint@GlyphPositionAdjustments@@QAEXJAAULEPoint@@D@Z 1000bf90 f   GlyphPositionAdjustments.obj
 0001:0000b050       ?process@GlyphPositioningTableHeader@@QBEXABV?$LEReferenceTo@UGlyphPositioningTableHeader@@@@AAVLEGlyphStorage@@PAVGlyphPositionAdjustments@@DKKABV?$LEReferenceTo@UGlyphDefinitionTableHeader@@@@AAW4LEErrorCode@@PBVLEFontInstance@@PBUFeatureMap@@JD@Z 1000c050 f   GlyphPositioningTables.obj
 0001:0000b0d0       ??0GlyphPositioningLookupProcessor@@QAE@ABV?$LEReferenceTo@UGlyphPositioningTableHeader@@@@KKPBUFeatureMap@@JDAAW4LEErrorCode@@@Z 1000c0d0 f   GlyphPosnLookupProc.obj
 0001:0000b130       ??1GlyphPositioningLookupProcessor@@UAE@XZ 1000c130 f   GlyphPosnLookupProc.obj
 0001:0000b140       ??_EGlyphPositioningLookupProcessor@@UAEPAXI@Z 1000c140 f i GlyphPosnLookupProc.obj
 0001:0000b140       ??_GGlyphPositioningLookupProcessor@@UAEPAXI@Z 1000c140 f i GlyphPosnLookupProc.obj
 0001:0000b170       ?applySubtable@GlyphPositioningLookupProcessor@@UBEKABV?$LEReferenceTo@ULookupSubtable@@@@GPAVGlyphIterator@@PBVLEFontInstance@@AAW4LEErrorCode@@@Z 1000c170 f   GlyphPosnLookupProc.obj
 0001:0000b730       ??0GlyphSubstitutionLookupProcessor@@QAE@ABV?$LEReferenceTo@UGlyphSubstitutionTableHeader@@@@KKPBVLEGlyphFilter@@PBUFeatureMap@@JDAAW4LEErrorCode@@@Z 1000c730 f   GlyphSubstLookupProc.obj
 0001:0000b7a0       ??1GlyphSubstitutionLookupProcessor@@UAE@XZ 1000c7a0 f   GlyphSubstLookupProc.obj
 0001:0000b7b0       ??_EGlyphSubstitutionLookupProcessor@@UAEPAXI@Z 1000c7b0 f i GlyphSubstLookupProc.obj
 0001:0000b7b0       ??_GGlyphSubstitutionLookupProcessor@@UAEPAXI@Z 1000c7b0 f i GlyphSubstLookupProc.obj
 0001:0000b7e0       ?applySubtable@GlyphSubstitutionLookupProcessor@@UBEKABV?$LEReferenceTo@ULookupSubtable@@@@GPAVGlyphIterator@@PBVLEFontInstance@@AAW4LEErrorCode@@@Z 1000c7e0 f   GlyphSubstLookupProc.obj
 0001:0000bc70       ?process@GlyphSubstitutionTableHeader@@QBEJABV?$LEReferenceTo@UGlyphSubstitutionTableHeader@@@@AAVLEGlyphStorage@@DKKABV?$LEReferenceTo@UGlyphDefinitionTableHeader@@@@PBVLEGlyphFilter@@PBUFeatureMap@@JDAAW4LEErrorCode@@@Z 1000cc70 f   GlyphSubstitutionTables.obj
 0001:0000bcf0       ??0HanOpenTypeLayoutEngine@@QAE@PBVLEFontInstance@@JJJABV?$LEReferenceTo@UGlyphSubstitutionTableHeader@@@@AAW4LEErrorCode@@@Z 1000ccf0 f   HanLayoutEngine.obj
 0001:0000bd30       ??_EHanOpenTypeLayoutEngine@@UAEPAXI@Z 1000cd30 f i HanLayoutEngine.obj
 0001:0000bd30       ??_GHanOpenTypeLayoutEngine@@UAEPAXI@Z 1000cd30 f i HanLayoutEngine.obj
 0001:0000bd60       ?characterProcessing@HanOpenTypeLayoutEngine@@MAEJQBGJJJDAAPAGAAVLEGlyphStorage@@AAW4LEErrorCode@@@Z 1000cd60 f   HanLayoutEngine.obj
 0001:0000bdf0       ?getDynamicClassID@HanOpenTypeLayoutEngine@@UBEPBDXZ 1000cdf0 f   HanLayoutEngine.obj
 0001:0000be00       ??0HangulOpenTypeLayoutEngine@@QAE@PBVLEFontInstance@@JJJAAW4LEErrorCode@@@Z 1000ce00 f   HangulLayoutEngine.obj
 0001:0000be40       ??0HangulOpenTypeLayoutEngine@@QAE@PBVLEFontInstance@@JJJABV?$LEReferenceTo@UGlyphSubstitutionTableHeader@@@@AAW4LEErrorCode@@@Z 1000ce40 f   HangulLayoutEngine.obj
 0001:0000be80       ??_EHangulOpenTypeLayoutEngine@@UAEPAXI@Z 1000ce80 f i HangulLayoutEngine.obj
 0001:0000be80       ??_GHangulOpenTypeLayoutEngine@@UAEPAXI@Z 1000ce80 f i HangulLayoutEngine.obj
 0001:0000beb0       ?characterProcessing@HangulOpenTypeLayoutEngine@@MAEJQBGJJJDAAPAGAAVLEGlyphStorage@@AAW4LEErrorCode@@@Z 1000ceb0 f   HangulLayoutEngine.obj
 0001:0000c400       ?getDynamicClassID@HangulOpenTypeLayoutEngine@@UBEPBDXZ 1000d400 f   HangulLayoutEngine.obj
 0001:0000c410       ?getCharClass@IndicClassTable@@QBEKG@Z 1000d410 f   IndicClassTables.obj
 0001:0000c470       ?getFilterZeroWidth@IndicReordering@@SADJ@Z 1000d470 f   IndicClassTables.obj
 0001:0000c4a0       ?getScriptClassTable@IndicClassTable@@SAPBU1@J@Z 1000d4a0 f   IndicClassTables.obj
 0001:0000c4c0       ?getWorstCaseExpansion@IndicReordering@@SAJJ@Z 1000d4c0 f   IndicClassTables.obj
 0001:0000c4e0       ??0IndicOpenTypeLayoutEngine@@QAE@PBVLEFontInstance@@JJJAAW4LEErrorCode@@@Z 1000d4e0 f   IndicLayoutEngine.obj
 0001:0000c530       ??0IndicOpenTypeLayoutEngine@@QAE@PBVLEFontInstance@@JJJDABV?$LEReferenceTo@UGlyphSubstitutionTableHeader@@@@AAW4LEErrorCode@@@Z 1000d530 f   IndicLayoutEngine.obj
 0001:0000c5a0       ??_EIndicOpenTypeLayoutEngine@@UAEPAXI@Z 1000d5a0 f i IndicLayoutEngine.obj
 0001:0000c5a0       ??_GIndicOpenTypeLayoutEngine@@UAEPAXI@Z 1000d5a0 f i IndicLayoutEngine.obj
 0001:0000c5d0       ?characterProcessing@IndicOpenTypeLayoutEngine@@MAEJQBGJJJDAAPAGAAVLEGlyphStorage@@AAW4LEErrorCode@@@Z 1000d5d0 f   IndicLayoutEngine.obj
 0001:0000c720       ?getDynamicClassID@IndicOpenTypeLayoutEngine@@UBEPBDXZ 1000d720 f   IndicLayoutEngine.obj
 0001:0000c730       ?glyphProcessing@IndicOpenTypeLayoutEngine@@MAEJQBGJJJDAAVLEGlyphStorage@@AAW4LEErrorCode@@@Z 1000d730 f   IndicLayoutEngine.obj
 0001:0000c800       ??0IndicRearrangementProcessor@@QAE@ABV?$LEReferenceTo@UMorphSubtableHeader@@@@AAW4LEErrorCode@@@Z 1000d800 f   IndicRearrangementProcessor.obj
 0001:0000cb00       ??_EIndicRearrangementProcessor@@UAEPAXI@Z 1000db00 f i IndicRearrangementProcessor.obj
 0001:0000cb00       ??_GIndicRearrangementProcessor@@UAEPAXI@Z 1000db00 f i IndicRearrangementProcessor.obj
 0001:0000cb50       ?beginStateTable@IndicRearrangementProcessor@@UAEXXZ 1000db50 f   IndicRearrangementProcessor.obj
 0001:0000cb60       ?doRearrangementAction@IndicRearrangementProcessor@@QBEXAAVLEGlyphStorage@@W4IndicRearrangementVerb@@AAW4LEErrorCode@@@Z 1000db60 f   IndicRearrangementProcessor.obj
 0001:0000d650       ?getDynamicClassID@IndicRearrangementProcessor@@UBEPBDXZ 1000e650 f   IndicRearrangementProcessor.obj
 0001:0000d660       ?processStateEntry@IndicRearrangementProcessor@@UAEFAAVLEGlyphStorage@@AAJEAAW4LEErrorCode@@@Z 1000e660 f   IndicRearrangementProcessor.obj
 0001:0000d720       ??0?$LEReferenceToArrayOf@UIndicRearrangementStateEntry2@@@@QAE@ABVLETableReference@@AAW4LEErrorCode@@IK@Z 1000e720 f i IndicRearrangementProcessor2.obj
 0001:0000d810       ??0IndicRearrangementProcessor2@@QAE@ABV?$LEReferenceTo@UMorphSubtableHeader2@@@@AAW4LEErrorCode@@@Z 1000e810 f   IndicRearrangementProcessor2.obj
 0001:0000d900       ??_EIndicRearrangementProcessor2@@UAEPAXI@Z 1000e900 f i IndicRearrangementProcessor2.obj
 0001:0000d900       ??_GIndicRearrangementProcessor2@@UAEPAXI@Z 1000e900 f i IndicRearrangementProcessor2.obj
 0001:0000d940       ?beginStateTable@IndicRearrangementProcessor2@@UAEXXZ 1000e940 f   IndicRearrangementProcessor2.obj
 0001:0000d960       ?doRearrangementAction@IndicRearrangementProcessor2@@QBEXAAVLEGlyphStorage@@W4IndicRearrangementVerb@@AAW4LEErrorCode@@@Z 1000e960 f   IndicRearrangementProcessor2.obj
 0001:0000e550       ?getDynamicClassID@IndicRearrangementProcessor2@@UBEPBDXZ 1000f550 f   IndicRearrangementProcessor2.obj
 0001:0000e560       ?processStateEntry@IndicRearrangementProcessor2@@UAEGAAVLEGlyphStorage@@AAJGAAW4LEErrorCode@@@Z 1000f560 f   IndicRearrangementProcessor2.obj
 0001:0000e620       ??0IndicReorderingOutput@@QAE@PAGAAVLEGlyphStorage@@PAVMPreFixups@@@Z 1000f620 f i IndicReordering.obj
 0001:0000e6a0       ?adjustMPres@IndicReordering@@SAXPAVMPreFixups@@AAVLEGlyphStorage@@AAW4LEErrorCode@@@Z 1000f6a0 f   IndicReordering.obj
 0001:0000e6d0       ?applyPresentationForms@IndicReordering@@SAXAAVLEGlyphStorage@@J@Z 1000f6d0 f   IndicReordering.obj
 0001:0000e710       ?decomposeReorderMatras@IndicReorderingOutput@@QAEXPBUIndicClassTable@@JJJ@Z 1000f710 f i IndicReordering.obj
 0001:0000ea60       ?finalReordering@IndicReordering@@SAXAAVLEGlyphStorage@@J@Z 1000fa60 f   IndicReordering.obj
 0001:0000eb60       ?findSyllable@IndicReordering@@CAJPBUIndicClassTable@@PBGJJ@Z 1000fb60 f   IndicReordering.obj
 0001:0000ebd0       ?getFeatureMap@IndicReordering@@SAPBUFeatureMap@@AAJ@Z 1000fbd0 f   IndicReordering.obj
 0001:0000ebe0       ?getv2FeatureMap@IndicReordering@@SAPBUFeatureMap@@AAJ@Z 1000fbe0 f   IndicReordering.obj
 0001:0000ebf0       ?reorder@IndicReordering@@SAJPBGJJPAGAAVLEGlyphStorage@@PAPAVMPreFixups@@AAW4LEErrorCode@@@Z 1000fbf0 f   IndicReordering.obj
 0001:000103d0       ?saveMatra@IndicReorderingOutput@@AAEXGJK@Z 100113d0 f i IndicReordering.obj
 0001:00010480       ?v2process@IndicReordering@@SAJPBGJJPAGAAVLEGlyphStorage@@AAW4LEErrorCode@@@Z 10011480 f   IndicReordering.obj
 0001:000109f0       ?writeMpre@IndicReorderingOutput@@QAEXXZ 100119f0 f i IndicReordering.obj
 0001:00010a50       ??0KernTable@@QAE@ABVLETableReference@@AAW4LEErrorCode@@@Z 10011a50 f   KernTable.obj
 0001:00010e20       ?process@KernTable@@QAEXAAVLEGlyphStorage@@AAW4LEErrorCode@@@Z 10011e20 f   KernTable.obj
 0001:00010f80       ??0KhmerOpenTypeLayoutEngine@@QAE@PBVLEFontInstance@@JJJABV?$LEReferenceTo@UGlyphSubstitutionTableHeader@@@@AAW4LEErrorCode@@@Z 10011f80 f   KhmerLayoutEngine.obj
 0001:00010fc0       ??_EKhmerOpenTypeLayoutEngine@@UAEPAXI@Z 10011fc0 f i KhmerLayoutEngine.obj
 0001:00010fc0       ??_GKhmerOpenTypeLayoutEngine@@UAEPAXI@Z 10011fc0 f i KhmerLayoutEngine.obj
 0001:00010ff0       ?characterProcessing@KhmerOpenTypeLayoutEngine@@MAEJQBGJJJDAAPAGAAVLEGlyphStorage@@AAW4LEErrorCode@@@Z 10011ff0 f   KhmerLayoutEngine.obj
 0001:00011110       ?getDynamicClassID@KhmerOpenTypeLayoutEngine@@UBEPBDXZ 10012110 f   KhmerLayoutEngine.obj
 0001:00011120       ?getFeatureMap@KhmerReordering@@SAPBUFeatureMap@@AAJ@Z 10012120 f   KhmerReordering.obj
 0001:00011130       ?reorder@KhmerReordering@@SAJPBGJJPAGAAVLEGlyphStorage@@@Z 10012130 f   KhmerReordering.obj
 0001:00011900       ??1LECharMapper@@UAE@XZ    10012900 f   LEFontInstance.obj
 0001:00011910       ??1LEFontInstance@@UAE@XZ  10012910 f   LEFontInstance.obj
 0001:00011920       ??_ELECharMapper@@UAEPAXI@Z 10012920 f i LEFontInstance.obj
 0001:00011920       ??_GLECharMapper@@UAEPAXI@Z 10012920 f i LEFontInstance.obj
 0001:00011950       ?canDisplay@LEFontInstance@@UBEDK@Z 10012950 f   LEFontInstance.obj
 0001:00011970       ?getDynamicClassID@LEFontInstance@@UBEPBDXZ 10012970 f   LEFontInstance.obj
 0001:00011980       ?getLineHeight@LEFontInstance@@UBEJXZ 10012980 f   LEFontInstance.obj
 0001:000119a0       ?getSubFont@LEFontInstance@@UBEPBV1@QBGPAJJJAAW4LEErrorCode@@@Z 100129a0 f   LEFontInstance.obj
 0001:000119f0       ?mapCharToGlyph@LEFontInstance@@UBEKKPBVLECharMapper@@@Z 100129f0 f   LEFontInstance.obj
 0001:00011a10       ?mapCharToGlyph@LEFontInstance@@UBEKKPBVLECharMapper@@D@Z 10012a10 f   LEFontInstance.obj
 0001:00011a80       ?mapCharsToGlyphs@LEFontInstance@@UBEXQBGJJDPBVLECharMapper@@DAAVLEGlyphStorage@@@Z 10012a80 f   LEFontInstance.obj
 0001:00011b60       ?transformFunits@LEFontInstance@@UBEXMMAAULEPoint@@@Z 10012b60 f   LEFontInstance.obj
 0001:00011bc0       ?xPixelsToUnits@LEFontInstance@@UBEMM@Z 10012bc0 f   LEFontInstance.obj
 0001:00011bf0       ?xUnitsToPoints@LEFontInstance@@UBEMM@Z 10012bf0 f   LEFontInstance.obj
 0001:00011c30       ?yPixelsToUnits@LEFontInstance@@UBEMM@Z 10012c30 f   LEFontInstance.obj
 0001:00011c60       ?yUnitsToPoints@LEFontInstance@@UBEMM@Z 10012c60 f   LEFontInstance.obj
 0001:00011ca0       ??0LEGlyphStorage@@QAE@XZ  10012ca0 f   LEGlyphStorage.obj
 0001:00011cf0       ??1LEGlyphStorage@@UAE@XZ  10012cf0 f   LEGlyphStorage.obj
 0001:00011d90       ??_ELEGlyphStorage@@UAEPAXI@Z 10012d90 f i LEGlyphStorage.obj
 0001:00011d90       ??_GLEGlyphStorage@@UAEPAXI@Z 10012d90 f i LEGlyphStorage.obj
 0001:00011e40       ??_ELEInsertionCallback@@UAEPAXI@Z 10012e40 f i LEGlyphStorage.obj
 0001:00011e40       ??_GLEInsertionCallback@@UAEPAXI@Z 10012e40 f i LEGlyphStorage.obj
 0001:00011e70       ?adjustPosition@LEGlyphStorage@@QAEXJMMAAW4LEErrorCode@@@Z 10012e70 f   LEGlyphStorage.obj
 0001:00011ec0       ?adoptAuxDataArray@LEGlyphStorage@@QAEXAAV1@@Z 10012ec0 f   LEGlyphStorage.obj
 0001:00011ef0       ?adoptCharIndicesArray@LEGlyphStorage@@QAEXAAV1@@Z 10012ef0 f   LEGlyphStorage.obj
 0001:00011f20       ?adoptGlyphArray@LEGlyphStorage@@QAEXAAV1@@Z 10012f20 f   LEGlyphStorage.obj
 0001:00011f80       ?adoptGlyphCount@LEGlyphStorage@@QAEXAAV1@@Z 10012f80 f   LEGlyphStorage.obj
 0001:00011f90       ?adoptGlyphCount@LEGlyphStorage@@QAEXJ@Z 10012f90 f   LEGlyphStorage.obj
 0001:00011fa0       ?allocateAuxData@LEGlyphStorage@@QAEJAAW4LEErrorCode@@@Z 10012fa0 f   LEGlyphStorage.obj
 0001:00012010       ?allocateGlyphArray@LEGlyphStorage@@QAEXJDAAW4LEErrorCode@@@Z 10013010 f   LEGlyphStorage.obj
 0001:00012170       ?allocatePositions@LEGlyphStorage@@QAEJAAW4LEErrorCode@@@Z 10013170 f   LEGlyphStorage.obj
 0001:000121f0       ?applyInsertion@LEGlyphStorage@@MAEDJJQAK@Z 100131f0 f   LEGlyphStorage.obj
 0001:000122e0       ?applyInsertions@LEGlyphStorage@@QAEJXZ 100132e0 f   LEGlyphStorage.obj
 0001:00012370       ?getAuxData@LEGlyphStorage@@QBEKJAAW4LEErrorCode@@@Z 10013370 f   LEGlyphStorage.obj
 0001:000123b0       ?getCharIndex@LEGlyphStorage@@QBEJJAAW4LEErrorCode@@@Z 100133b0 f   LEGlyphStorage.obj
 0001:00012400       ?getCharIndices@LEGlyphStorage@@QBEXQAJJAAW4LEErrorCode@@@Z 10013400 f   LEGlyphStorage.obj
 0001:00012460       ?getDynamicClassID@LEGlyphStorage@@UBEPBDXZ 10013460 f   LEGlyphStorage.obj
 0001:00012470       ?getGlyphID@LEGlyphStorage@@QBEKJAAW4LEErrorCode@@@Z 10013470 f   LEGlyphStorage.obj
 0001:000124c0       ?getGlyphPosition@LEGlyphStorage@@QBEXJAAM0AAW4LEErrorCode@@@Z 100134c0 f   LEGlyphStorage.obj
 0001:00012510       ?getGlyphPositions@LEGlyphStorage@@QBEXQAMAAW4LEErrorCode@@@Z 10013510 f   LEGlyphStorage.obj
 0001:00012560       ?getGlyphs@LEGlyphStorage@@QBEXQAKKAAW4LEErrorCode@@@Z 10013560 f   LEGlyphStorage.obj
 0001:000125c0       ?insertGlyphs@LEGlyphStorage@@QAEPAKJJAAW4LEErrorCode@@@Z 100135c0 f   LEGlyphStorage.obj
 0001:000125d0       ?moveGlyph@LEGlyphStorage@@QAEXJJK@Z 100135d0 f   LEGlyphStorage.obj
 0001:00012820       ?reset@LEGlyphStorage@@QAEXXZ 10013820 f   LEGlyphStorage.obj
 0001:000128b0       ?setAuxData@LEGlyphStorage@@QAEXJKAAW4LEErrorCode@@@Z 100138b0 f   LEGlyphStorage.obj
 0001:000128f0       ?setCharIndex@LEGlyphStorage@@QAEXJJAAW4LEErrorCode@@@Z 100138f0 f   LEGlyphStorage.obj
 0001:00012930       ?setPosition@LEGlyphStorage@@QAEXJMMAAW4LEErrorCode@@@Z 10013930 f   LEGlyphStorage.obj
 0001:00012970       ??0LEInsertionList@@QAE@D@Z 10013970 f   LEInsertionList.obj
 0001:000129a0       ??1LEInsertionList@@QAE@XZ 100139a0 f   LEInsertionList.obj
 0001:000129e0       ?applyInsertions@LEInsertionList@@QAEDPAVLEInsertionCallback@@@Z 100139e0 f   LEInsertionList.obj
 0001:00012a20       ?getDynamicClassID@LEInsertionList@@UBEPBDXZ 10013a20 f   LEInsertionList.obj
 0001:00012a30       ?getGrowAmount@LEInsertionList@@QAEJXZ 10013a30 f   LEInsertionList.obj
 0001:00012a40       ?insert@LEInsertionList@@QAEPAKJJAAW4LEErrorCode@@@Z 10013a40 f   LEInsertionList.obj
 0001:00012ac0       ?reset@LEInsertionList@@QAEXXZ 10013ac0 f   LEInsertionList.obj
 0001:00012b00       ??0CharSubstitutionFilter@@QAE@PBVLEFontInstance@@@Z 10013b00 f   LayoutEngine.obj
 0001:00012b20       ??0LayoutEngine@@IAE@PBVLEFontInstance@@JJJAAW4LEErrorCode@@@Z 10013b20 f   LayoutEngine.obj
 0001:00012ba0       ??1LEGlyphFilter@@UAE@XZ   10013ba0 f   LayoutEngine.obj
 0001:00012bb0       ??1LayoutEngine@@UAE@XZ    10013bb0 f   LayoutEngine.obj
 0001:00012bd0       ??_ECanonMarkFilter@@UAEPAXI@Z 10013bd0 f i LayoutEngine.obj
 0001:00012bd0       ??_GCanonMarkFilter@@UAEPAXI@Z 10013bd0 f i LayoutEngine.obj
 0001:00012c00       ??_ECharSubstitutionFilter@@UAEPAXI@Z 10013c00 f i LayoutEngine.obj
 0001:00012c00       ??_GCharSubstitutionFilter@@UAEPAXI@Z 10013c00 f i LayoutEngine.obj
 0001:00012c30       ??_EDefaultCharMapper@@UAEPAXI@Z 10013c30 f i LayoutEngine.obj
 0001:00012c30       ??_GDefaultCharMapper@@UAEPAXI@Z 10013c30 f i LayoutEngine.obj
 0001:00012c60       ??_ELayoutEngine@@UAEPAXI@Z 10013c60 f i LayoutEngine.obj
 0001:00012c60       ??_GLayoutEngine@@UAEPAXI@Z 10013c60 f i LayoutEngine.obj
 0001:00012c90       ?accept@CanonMarkFilter@@UBEDKAAW4LEErrorCode@@@Z 10013c90 f   LayoutEngine.obj
 0001:00012cc0       ?adjustGlyphPositions@LayoutEngine@@MAEXQBGJJDAAVLEGlyphStorage@@AAW4LEErrorCode@@@Z 10013cc0 f   LayoutEngine.obj
 0001:00012f40       ?adjustMarkGlyphs@LayoutEngine@@KAXAAVLEGlyphStorage@@PAVLEGlyphFilter@@AAW4LEErrorCode@@@Z 10013f40 f   LayoutEngine.obj
 0001:00013050       ?adjustMarkGlyphs@LayoutEngine@@KAXQBGJDAAVLEGlyphStorage@@PAVLEGlyphFilter@@AAW4LEErrorCode@@@Z 10014050 f   LayoutEngine.obj
 0001:000131a0       ?characterProcessing@LayoutEngine@@MAEJQBGJJJDAAPAGAAVLEGlyphStorage@@AAW4LEErrorCode@@@Z 100141a0 f   LayoutEngine.obj
 0001:00013540       ?computeGlyphs@LayoutEngine@@MAEJQBGJJJDAAVLEGlyphStorage@@AAW4LEErrorCode@@@Z 10014540 f   LayoutEngine.obj
 0001:00013630       ?getCharIndices@LayoutEngine@@QBEXQAJJAAW4LEErrorCode@@@Z 10014630 f   LayoutEngine.obj
 0001:00013640       ?getDynamicClassID@LayoutEngine@@UBEPBDXZ 10014640 f   LayoutEngine.obj
 0001:00013650       ?getFontTable@LayoutEngine@@MBEPBXKAAI@Z 10014650 f   LayoutEngine.obj
 0001:00013660       ?getGlyphPosition@LayoutEngine@@QBEXJAAM0AAW4LEErrorCode@@@Z 10014660 f   LayoutEngine.obj
 0001:00013670       ?getGlyphPositions@LayoutEngine@@QBEXQAMAAW4LEErrorCode@@@Z 10014670 f   LayoutEngine.obj
 0001:00013680       ?getGlyphs@LayoutEngine@@UBEXQAKKAAW4LEErrorCode@@@Z 10014680 f   LayoutEngine.obj
 0001:00013690       ?layoutChars@LayoutEngine@@UAEJQBGJJJDMMAAW4LEErrorCode@@@Z 10014690 f   LayoutEngine.obj
 0001:00013770       ?layoutEngineFactory@LayoutEngine@@SAPAV1@PBVLEFontInstance@@JJJAAW4LEErrorCode@@@Z 10014770 f   LayoutEngine.obj
 0001:00013e90       ?mapChar@DefaultCharMapper@@UBEKK@Z 10014e90 f   LayoutEngine.obj
 0001:00013f40       ?mapCharsToGlyphs@LayoutEngine@@MAEXQBGJJDDAAVLEGlyphStorage@@AAW4LEErrorCode@@@Z 10014f40 f   LayoutEngine.obj
 0001:00013fc0       ?positionGlyphs@LayoutEngine@@MAEXAAVLEGlyphStorage@@MMAAW4LEErrorCode@@@Z 10014fc0 f   LayoutEngine.obj
 0001:00014090       ?reset@LayoutEngine@@UAEXXZ 10015090 f   LayoutEngine.obj
 0001:000140a0       ??0LigatureSubstitutionProcessor@@QAE@ABV?$LEReferenceTo@UMorphSubtableHeader@@@@AAW4LEErrorCode@@@Z 100150a0 f   LigatureSubstProc.obj
 0001:000142c0       ??_ELigatureSubstitutionProcessor@@UAEPAXI@Z 100152c0 f i LigatureSubstProc.obj
 0001:000142c0       ??_GLigatureSubstitutionProcessor@@UAEPAXI@Z 100152c0 f i LigatureSubstProc.obj
 0001:00014300       ?beginStateTable@LigatureSubstitutionProcessor@@UAEXXZ 10015300 f   LigatureSubstProc.obj
 0001:00014310       ?getDynamicClassID@LigatureSubstitutionProcessor@@UBEPBDXZ 10015310 f   LigatureSubstProc.obj
 0001:00014320       ?processStateEntry@LigatureSubstitutionProcessor@@UAEFAAVLEGlyphStorage@@AAJEAAW4LEErrorCode@@@Z 10015320 f   LigatureSubstProc.obj
 0001:000147d0       ??0LigatureSubstitutionProcessor2@@QAE@ABV?$LEReferenceTo@UMorphSubtableHeader2@@@@AAW4LEErrorCode@@@Z 100157d0 f   LigatureSubstProc2.obj
 0001:00014a60       ??_ELigatureSubstitutionProcessor2@@UAEPAXI@Z 10015a60 f i LigatureSubstProc2.obj
 0001:00014a60       ??_GLigatureSubstitutionProcessor2@@UAEPAXI@Z 10015a60 f i LigatureSubstProc2.obj
 0001:00014aa0       ?beginStateTable@LigatureSubstitutionProcessor2@@UAEXXZ 10015aa0 f   LigatureSubstProc2.obj
 0001:00014ab0       ?getDynamicClassID@LigatureSubstitutionProcessor2@@UBEPBDXZ 10015ab0 f   LigatureSubstProc2.obj
 0001:00014ac0       ?processStateEntry@LigatureSubstitutionProcessor2@@UAEGAAVLEGlyphStorage@@AAJGAAW4LEErrorCode@@@Z 10015ac0 f   LigatureSubstProc2.obj
 0001:00015260       ?process@LigatureSubstitutionSubtable@@QBEKABVLETableReference@@PAVGlyphIterator@@AAW4LEErrorCode@@PBVLEGlyphFilter@@@Z 10016260 f   LigatureSubstSubtables.obj
 0001:00015b50       ??0LookupProcessor@@IAE@ABVLETableReference@@GGGKKPBUFeatureMap@@JDAAW4LEErrorCode@@@Z 10016b50 f   LookupProcessor.obj
 0001:00016c70       ??1LookupProcessor@@UAE@XZ 10017c70 f   LookupProcessor.obj
 0001:00016cb0       ??_ELookupProcessor@@UAEPAXI@Z 10017cb0 f i LookupProcessor.obj
 0001:00016cb0       ??_GLookupProcessor@@UAEPAXI@Z 10017cb0 f i LookupProcessor.obj
 0001:00016d00       ?applyLookupTable@LookupProcessor@@QBEKABV?$LEReferenceTo@ULookupTable@@@@PAVGlyphIterator@@PBVLEFontInstance@@AAW4LEErrorCode@@@Z 10017d00 f   LookupProcessor.obj
 0001:00016dc0       ?applySingleLookup@LookupProcessor@@QBEKGPAVGlyphIterator@@PBVLEFontInstance@@AAW4LEErrorCode@@@Z 10017dc0 f   LookupProcessor.obj
 0001:00016f10       ?process@LookupProcessor@@QBEJAAVLEGlyphStorage@@PAVGlyphPositionAdjustments@@DABV?$LEReferenceTo@UGlyphDefinitionTableHeader@@@@PBVLEFontInstance@@AAW4LEErrorCode@@@Z 10017f10 f   LookupProcessor.obj
 0001:00017060       ?lookupSegment@BinarySearchLookupTable@@QBEPBULookupSegment@@ABVLETableReference@@PBU2@KAAW4LEErrorCode@@@Z 10018060 f   LookupTables.obj
 0001:00017320       ?lookupSingle@BinarySearchLookupTable@@QBEPBULookupSingle@@ABVLETableReference@@PBU2@KAAW4LEErrorCode@@@Z 10018320 f   LookupTables.obj
 0001:000175e0       ?getGlyphCoverage@LookupSubtable@@QBEJABV?$LEReferenceTo@ULookupSubtable@@@@GKAAW4LEErrorCode@@@Z 100185e0 f   Lookups.obj
 0001:000176b0       ?getLookupSubtable@LookupTable@@QBE?BV?$LEReferenceTo@ULookupSubtable@@@@ABV?$LEReferenceTo@ULookupTable@@@@GAAW4LEErrorCode@@@Z 100186b0 f   Lookups.obj
 0001:00017820       ?getLookupTable@LookupListTable@@QBE?BV?$LEReferenceTo@ULookupTable@@@@ABV?$LEReferenceTo@ULookupListTable@@@@GAAW4LEErrorCode@@@Z 10018820 f   Lookups.obj
 0001:00017990       ??0MPreFixups@@QAE@J@Z     10018990 f   MPreFixups.obj
 0001:000179d0       ??1MPreFixups@@QAE@XZ      100189d0 f   MPreFixups.obj
 0001:000179f0       ?add@MPreFixups@@QAEXJJ@Z  100189f0 f   MPreFixups.obj
 0001:00017a20       ?apply@MPreFixups@@QAEXAAVLEGlyphStorage@@AAW4LEErrorCode@@@Z 10018a20 f   MPreFixups.obj
 0001:00017c90       ??0?$LEReferenceToArrayOf@UMarkRecord@@@@QAE@ABVLETableReference@@AAW4LEErrorCode@@PBUMarkRecord@@K@Z 10018c90 f i MarkArrays.obj
 0001:00017db0       ?getMarkClass@MarkArray@@QBEJABVLETableReference@@KJPBVLEFontInstance@@AAULEPoint@@AAW4LEErrorCode@@@Z 10018db0 f   MarkArrays.obj
 0001:00017ec0       ?process@MarkToBasePositioningSubtable@@QBEJABVLETableReference@@PAVGlyphIterator@@PBVLEFontInstance@@AAW4LEErrorCode@@@Z 10018ec0 f   MarkToBasePosnSubtables.obj
 0001:000189e0       ?process@MarkToLigaturePositioningSubtable@@QBEJABVLETableReference@@PAVGlyphIterator@@PBVLEFontInstance@@AAW4LEErrorCode@@@Z 100199e0 f   MarkToLigaturePosnSubtables.obj
 0001:00019470       ?process@MarkToMarkPositioningSubtable@@QBEJABVLETableReference@@PAVGlyphIterator@@PBVLEFontInstance@@AAW4LEErrorCode@@@Z 1001a470 f   MarkToMarkPosnSubtables.obj
 0001:00019ce0       ?process@MorphTableHeader@@QBEXABVLETableReference@@AAVLEGlyphStorage@@AAW4LEErrorCode@@@Z 1001ace0 f   MorphTables.obj
 0001:0001a2c0       ?process@MorphTableHeader2@@QBEXABV?$LEReferenceTo@UMorphTableHeader2@@@@AAVLEGlyphStorage@@JAAW4LEErrorCode@@@Z 1001b2c0 f   MorphTables2.obj
 0001:0001ac00       ?process@MultipleSubstitutionSubtable@@QBEKABVLETableReference@@PAVGlyphIterator@@AAW4LEErrorCode@@PBVLEGlyphFilter@@@Z 1001bc00 f   MultipleSubstSubtables.obj
 0001:0001b050       ??0NonContextualGlyphSubstitutionProcessor@@IAE@ABV?$LEReferenceTo@UMorphSubtableHeader@@@@AAW4LEErrorCode@@@Z 1001c050 f   NonContextualGlyphSubstProc.obj
 0001:0001b070       ??1NonContextualGlyphSubstitutionProcessor@@MAE@XZ 1001c070 f   NonContextualGlyphSubstProc.obj
 0001:0001b080       ??_ENonContextualGlyphSubstitutionProcessor@@MAEPAXI@Z 1001c080 f i NonContextualGlyphSubstProc.obj
 0001:0001b080       ??_GNonContextualGlyphSubstitutionProcessor@@MAEPAXI@Z 1001c080 f i NonContextualGlyphSubstProc.obj
 0001:0001b0b0       ?createInstance@NonContextualGlyphSubstitutionProcessor@@SAPAVSubtableProcessor@@ABV?$LEReferenceTo@UMorphSubtableHeader@@@@AAW4LEErrorCode@@@Z 1001c0b0 f   NonContextualGlyphSubstProc.obj
 0001:0001b1f0       ??0NonContextualGlyphSubstitutionProcessor2@@IAE@ABV?$LEReferenceTo@UMorphSubtableHeader2@@@@AAW4LEErrorCode@@@Z 1001c1f0 f   NonContextualGlyphSubstProc2.obj
 0001:0001b210       ??1NonContextualGlyphSubstitutionProcessor2@@MAE@XZ 1001c210 f   NonContextualGlyphSubstProc2.obj
 0001:0001b220       ??_ENonContextualGlyphSubstitutionProcessor2@@MAEPAXI@Z 1001c220 f i NonContextualGlyphSubstProc2.obj
 0001:0001b220       ??_GNonContextualGlyphSubstitutionProcessor2@@MAEPAXI@Z 1001c220 f i NonContextualGlyphSubstProc2.obj
 0001:0001b250       ?createInstance@NonContextualGlyphSubstitutionProcessor2@@SAPAVSubtableProcessor2@@ABV?$LEReferenceTo@UMorphSubtableHeader2@@@@AAW4LEErrorCode@@@Z 1001c250 f   NonContextualGlyphSubstProc2.obj
 0001:0001b390       ??0OpenTypeLayoutEngine@@QAE@PBVLEFontInstance@@JJJAAW4LEErrorCode@@@Z 1001c390 f   OpenTypeLayoutEngine.obj
 0001:0001b440       ??0OpenTypeLayoutEngine@@QAE@PBVLEFontInstance@@JJJABV?$LEReferenceTo@UGlyphSubstitutionTableHeader@@@@AAW4LEErrorCode@@@Z 1001c440 f   OpenTypeLayoutEngine.obj
 0001:0001b5e0       ??1OpenTypeLayoutEngine@@UAE@XZ 1001c5e0 f   OpenTypeLayoutEngine.obj
 0001:0001b630       ??_EOpenTypeLayoutEngine@@UAEPAXI@Z 1001c630 f i OpenTypeLayoutEngine.obj
 0001:0001b630       ??_GOpenTypeLayoutEngine@@UAEPAXI@Z 1001c630 f i OpenTypeLayoutEngine.obj
 0001:0001b690       ?adjustGlyphPositions@OpenTypeLayoutEngine@@MAEXQBGJJDAAVLEGlyphStorage@@AAW4LEErrorCode@@@Z 1001c690 f   OpenTypeLayoutEngine.obj
 0001:0001ba70       ?applyTypoFlags@OpenTypeLayoutEngine@@AAEXXZ 1001ca70 f   OpenTypeLayoutEngine.obj
 0001:0001bbf0       ?characterProcessing@OpenTypeLayoutEngine@@MAEJQBGJJJDAAPAGAAVLEGlyphStorage@@AAW4LEErrorCode@@@Z 1001cbf0 f   OpenTypeLayoutEngine.obj
 0001:0001bd10       ?computeGlyphs@OpenTypeLayoutEngine@@MAEJQBGJJJDAAVLEGlyphStorage@@AAW4LEErrorCode@@@Z 1001cd10 f   OpenTypeLayoutEngine.obj
 0001:0001be30       ?getDynamicClassID@OpenTypeLayoutEngine@@UBEPBDXZ 1001ce30 f   OpenTypeLayoutEngine.obj
 0001:0001be40       ?getLangSysTag@OpenTypeLayoutEngine@@SAKJ@Z 1001ce40 f   OpenTypeLayoutEngine.obj
 0001:0001be60       ?getScriptTag@OpenTypeLayoutEngine@@SAKJ@Z 1001ce60 f   OpenTypeLayoutEngine.obj
 0001:0001be80       ?getV2ScriptTag@OpenTypeLayoutEngine@@SAKJ@Z 1001ce80 f   OpenTypeLayoutEngine.obj
 0001:0001bf20       ?glyphPostProcessing@OpenTypeLayoutEngine@@MAEJAAVLEGlyphStorage@@0AAW4LEErrorCode@@@Z 1001cf20 f   OpenTypeLayoutEngine.obj
 0001:0001bf60       ?glyphProcessing@OpenTypeLayoutEngine@@MAEJQBGJJJDAAVLEGlyphStorage@@AAW4LEErrorCode@@@Z 1001cf60 f   OpenTypeLayoutEngine.obj
 0001:0001c060       ?glyphSubstitution@OpenTypeLayoutEngine@@MAEJJJDAAVLEGlyphStorage@@AAW4LEErrorCode@@@Z 1001d060 f   OpenTypeLayoutEngine.obj
 0001:0001c110       ?reset@OpenTypeLayoutEngine@@MAEXXZ 1001d110 f   OpenTypeLayoutEngine.obj
 0001:0001c120       ?setScriptAndLanguageTags@OpenTypeLayoutEngine@@AAEXXZ 1001d120 f   OpenTypeLayoutEngine.obj
 0001:0001c200       ?getGlyphRangeIndex@OpenTypeUtilities@@SAJGABV?$LEReferenceToArrayOf@UGlyphRangeRecord@@@@AAW4LEErrorCode@@@Z 1001d200 f   OpenTypeUtilities.obj
 0001:0001c330       ?getTagOffset@OpenTypeUtilities@@SAGKABV?$LEReferenceToArrayOf@UTagAndOffsetRecord@@@@AAW4LEErrorCode@@@Z 1001d330 f   OpenTypeUtilities.obj
 0001:0001c430       ?highBit@OpenTypeUtilities@@SACJ@Z 1001d430 f   OpenTypeUtilities.obj
 0001:0001c4b0       ?search@OpenTypeUtilities@@SAJKQBKJ@Z 1001d4b0 f   OpenTypeUtilities.obj
 0001:0001c500       ?sort@OpenTypeUtilities@@SAXPAGJ@Z 1001d500 f   OpenTypeUtilities.obj
 0001:0001c560       ?process@PairPositioningFormat2Subtable@@QBEKABV?$LEReferenceTo@UPairPositioningFormat2Subtable@@@@PAVGlyphIterator@@PBVLEFontInstance@@AAW4LEErrorCode@@@Z 1001d560 f   PairPositioningSubtables.obj
 0001:0001ca00       ?process@PairPositioningSubtable@@QBEKABV?$LEReferenceTo@UPairPositioningSubtable@@@@PAVGlyphIterator@@PBVLEFontInstance@@AAW4LEErrorCode@@@Z 1001da00 f   PairPositioningSubtables.obj
 0001:0001d230       ?findLanguage@ScriptListTable@@QBE?AV?$LEReferenceTo@ULangSysTable@@@@ABVLETableReference@@KKAAW4LEErrorCode@@D@Z 1001e230 f   ScriptAndLanguage.obj
 0001:0001d2c0       ?findLanguage@ScriptTable@@QBE?AV?$LEReferenceTo@ULangSysTable@@@@ABVLETableReference@@KAAW4LEErrorCode@@D@Z 1001e2c0 f   ScriptAndLanguage.obj
 0001:0001d4a0       ?findScript@ScriptListTable@@QBE?AV?$LEReferenceTo@UScriptTable@@@@ABVLETableReference@@KAAW4LEErrorCode@@@Z 1001e4a0 f   ScriptAndLanguage.obj
 0001:0001d9a0       ??0SegmentArrayProcessor@@QAE@ABV?$LEReferenceTo@UMorphSubtableHeader@@@@AAW4LEErrorCode@@@Z 1001e9a0 f   SegmentArrayProcessor.obj
 0001:0001db10       ??_ESegmentArrayProcessor@@UAEPAXI@Z 1001eb10 f i SegmentArrayProcessor.obj
 0001:0001db10       ??_GSegmentArrayProcessor@@UAEPAXI@Z 1001eb10 f i SegmentArrayProcessor.obj
 0001:0001db40       ?getDynamicClassID@SegmentArrayProcessor@@UBEPBDXZ 1001eb40 f   SegmentArrayProcessor.obj
 0001:0001db50       ?process@SegmentArrayProcessor@@UAEXAAVLEGlyphStorage@@AAW4LEErrorCode@@@Z 1001eb50 f   SegmentArrayProcessor.obj
 0001:0001dc40       ??0SegmentArrayProcessor2@@QAE@ABV?$LEReferenceTo@UMorphSubtableHeader2@@@@AAW4LEErrorCode@@@Z 1001ec40 f   SegmentArrayProcessor2.obj
 0001:0001ddb0       ??_ESegmentArrayProcessor2@@UAEPAXI@Z 1001edb0 f i SegmentArrayProcessor2.obj
 0001:0001ddb0       ??_GSegmentArrayProcessor2@@UAEPAXI@Z 1001edb0 f i SegmentArrayProcessor2.obj
 0001:0001dde0       ?getDynamicClassID@SegmentArrayProcessor2@@UBEPBDXZ 1001ede0 f   SegmentArrayProcessor2.obj
 0001:0001ddf0       ?process@SegmentArrayProcessor2@@UAEXAAVLEGlyphStorage@@AAW4LEErrorCode@@@Z 1001edf0 f   SegmentArrayProcessor2.obj
 0001:0001df30       ??0SegmentSingleProcessor@@QAE@ABV?$LEReferenceTo@UMorphSubtableHeader@@@@AAW4LEErrorCode@@@Z 1001ef30 f   SegmentSingleProcessor.obj
 0001:0001e0a0       ??_ESegmentSingleProcessor@@UAEPAXI@Z 1001f0a0 f i SegmentSingleProcessor.obj
 0001:0001e0a0       ??_GSegmentSingleProcessor@@UAEPAXI@Z 1001f0a0 f i SegmentSingleProcessor.obj
 0001:0001e0d0       ?getDynamicClassID@SegmentSingleProcessor@@UBEPBDXZ 1001f0d0 f   SegmentSingleProcessor.obj
 0001:0001e0e0       ?process@SegmentSingleProcessor@@UAEXAAVLEGlyphStorage@@AAW4LEErrorCode@@@Z 1001f0e0 f   SegmentSingleProcessor.obj
 0001:0001e170       ??0SegmentSingleProcessor2@@QAE@ABV?$LEReferenceTo@UMorphSubtableHeader2@@@@AAW4LEErrorCode@@@Z 1001f170 f   SegmentSingleProcessor2.obj
 0001:0001e2e0       ??_ESegmentSingleProcessor2@@UAEPAXI@Z 1001f2e0 f i SegmentSingleProcessor2.obj
 0001:0001e2e0       ??_GSegmentSingleProcessor2@@UAEPAXI@Z 1001f2e0 f i SegmentSingleProcessor2.obj
 0001:0001e310       ?getDynamicClassID@SegmentSingleProcessor2@@UBEPBDXZ 1001f310 f   SegmentSingleProcessor2.obj
 0001:0001e320       ?process@SegmentSingleProcessor2@@UAEXAAVLEGlyphStorage@@AAW4LEErrorCode@@@Z 1001f320 f   SegmentSingleProcessor2.obj
 0001:0001e3b0       ??0SimpleArrayProcessor@@QAE@ABV?$LEReferenceTo@UMorphSubtableHeader@@@@AAW4LEErrorCode@@@Z 1001f3b0 f   SimpleArrayProcessor.obj
 0001:0001e520       ??_ESimpleArrayProcessor@@UAEPAXI@Z 1001f520 f i SimpleArrayProcessor.obj
 0001:0001e520       ??_GSimpleArrayProcessor@@UAEPAXI@Z 1001f520 f i SimpleArrayProcessor.obj
 0001:0001e550       ?getDynamicClassID@SimpleArrayProcessor@@UBEPBDXZ 1001f550 f   SimpleArrayProcessor.obj
 0001:0001e560       ?process@SimpleArrayProcessor@@UAEXAAVLEGlyphStorage@@AAW4LEErrorCode@@@Z 1001f560 f   SimpleArrayProcessor.obj
 0001:0001e6a0       ??0SimpleArrayProcessor2@@QAE@ABV?$LEReferenceTo@UMorphSubtableHeader2@@@@AAW4LEErrorCode@@@Z 1001f6a0 f   SimpleArrayProcessor2.obj
 0001:0001e920       ??_ESimpleArrayProcessor2@@UAEPAXI@Z 1001f920 f i SimpleArrayProcessor2.obj
 0001:0001e920       ??_GSimpleArrayProcessor2@@UAEPAXI@Z 1001f920 f i SimpleArrayProcessor2.obj
 0001:0001e960       ?getDynamicClassID@SimpleArrayProcessor2@@UBEPBDXZ 1001f960 f   SimpleArrayProcessor2.obj
 0001:0001e970       ?process@SimpleArrayProcessor2@@UAEXAAVLEGlyphStorage@@AAW4LEErrorCode@@@Z 1001f970 f   SimpleArrayProcessor2.obj
 0001:0001e9f0       ?process@SinglePositioningSubtable@@QBEKABV?$LEReferenceTo@USinglePositioningSubtable@@@@PAVGlyphIterator@@PBVLEFontInstance@@AAW4LEErrorCode@@@Z 1001f9f0 f   SinglePositioningSubtables.obj
 0001:0001ee80       ?process@SingleSubstitutionSubtable@@QBEKABV?$LEReferenceTo@USingleSubstitutionSubtable@@@@PAVGlyphIterator@@AAW4LEErrorCode@@PBVLEGlyphFilter@@@Z 1001fe80 f   SingleSubstitutionSubtables.obj
 0001:0001f3f0       ??0SingleTableProcessor@@QAE@ABV?$LEReferenceTo@UMorphSubtableHeader@@@@AAW4LEErrorCode@@@Z 100203f0 f   SingleTableProcessor.obj
 0001:0001f560       ??_ESingleTableProcessor@@UAEPAXI@Z 10020560 f i SingleTableProcessor.obj
 0001:0001f560       ??_GSingleTableProcessor@@UAEPAXI@Z 10020560 f i SingleTableProcessor.obj
 0001:0001f590       ?getDynamicClassID@SingleTableProcessor@@UBEPBDXZ 10020590 f   SingleTableProcessor.obj
 0001:0001f5a0       ?process@SingleTableProcessor@@UAEXAAVLEGlyphStorage@@AAW4LEErrorCode@@@Z 100205a0 f   SingleTableProcessor.obj
 0001:0001f620       ??0SingleTableProcessor2@@QAE@ABV?$LEReferenceTo@UMorphSubtableHeader2@@@@AAW4LEErrorCode@@@Z 10020620 f   SingleTableProcessor2.obj
 0001:0001f790       ??_ESingleTableProcessor2@@UAEPAXI@Z 10020790 f i SingleTableProcessor2.obj
 0001:0001f790       ??_GSingleTableProcessor2@@UAEPAXI@Z 10020790 f i SingleTableProcessor2.obj
 0001:0001f7c0       ?getDynamicClassID@SingleTableProcessor2@@UBEPBDXZ 100207c0 f   SingleTableProcessor2.obj
 0001:0001f7d0       ?process@SingleTableProcessor2@@UAEXAAVLEGlyphStorage@@AAW4LEErrorCode@@@Z 100207d0 f   SingleTableProcessor2.obj
 0001:0001f850       ??0StateTableProcessor@@IAE@ABV?$LEReferenceTo@UMorphSubtableHeader@@@@AAW4LEErrorCode@@@Z 10020850 f   StateTableProcessor.obj
 0001:0001fb50       ??1StateTableProcessor@@MAE@XZ 10020b50 f   StateTableProcessor.obj
 0001:0001fb70       ??_EStateTableProcessor@@MAEPAXI@Z 10020b70 f i StateTableProcessor.obj
 0001:0001fb70       ??_GStateTableProcessor@@MAEPAXI@Z 10020b70 f i StateTableProcessor.obj
 0001:0001fbb0       ?process@StateTableProcessor@@UAEXAAVLEGlyphStorage@@AAW4LEErrorCode@@@Z 10020bb0 f   StateTableProcessor.obj
 0001:0001fd30       ??0StateTableProcessor2@@IAE@ABV?$LEReferenceTo@UMorphSubtableHeader2@@@@AAW4LEErrorCode@@@Z 10020d30 f   StateTableProcessor2.obj
 0001:000200f0       ??1StateTableProcessor2@@MAE@XZ 100210f0 f   StateTableProcessor2.obj
 0001:00020120       ??_EStateTableProcessor2@@MAEPAXI@Z 10021120 f i StateTableProcessor2.obj
 0001:00020120       ??_GStateTableProcessor2@@MAEPAXI@Z 10021120 f i StateTableProcessor2.obj
 0001:00020170       ?process@StateTableProcessor2@@UAEXAAVLEGlyphStorage@@AAW4LEErrorCode@@@Z 10021170 f   StateTableProcessor2.obj
 0001:00020710       ??0SubtableProcessor@@IAE@ABV?$LEReferenceTo@UMorphSubtableHeader@@@@AAW4LEErrorCode@@@Z 10021710 f   SubtableProcessor.obj
 0001:00020790       ??1SubtableProcessor@@UAE@XZ 10021790 f   SubtableProcessor.obj
 0001:000207a0       ??_ESubtableProcessor@@UAEPAXI@Z 100217a0 f i SubtableProcessor.obj
 0001:000207a0       ??_GSubtableProcessor@@UAEPAXI@Z 100217a0 f i SubtableProcessor.obj
 0001:000207d0       ??0SubtableProcessor2@@IAE@ABV?$LEReferenceTo@UMorphSubtableHeader2@@@@AAW4LEErrorCode@@@Z 100217d0 f   SubtableProcessor2.obj
 0001:00020900       ??1SubtableProcessor2@@UAE@XZ 10021900 f   SubtableProcessor2.obj
 0001:00020910       ??_ESubtableProcessor2@@UAEPAXI@Z 10021910 f i SubtableProcessor2.obj
 0001:00020910       ??_GSubtableProcessor2@@UAEPAXI@Z 10021910 f i SubtableProcessor2.obj
 0001:00020940       ?SetIntField@JNIEnv_@@QAEXPAV_jobject@@PAU_jfieldID@@J@Z 10021940 f i SunLayoutEngine.obj
 0001:00020960       ?putGV@@YAHPAUJNIEnv_@@JJPAV_jobject@@PBVLayoutEngine@@H@Z 10021960 f   SunLayoutEngine.obj
 0001:00020b60       _Java_sun_font_SunLayoutEngine_initGVIDs@8 10021b60 f   SunLayoutEngine.obj
 0001:00020c50       _Java_sun_font_SunLayoutEngine_nativeLayout@84 10021c50 f   SunLayoutEngine.obj
 0001:00020f50       ??0ThaiLayoutEngine@@QAE@PBVLEFontInstance@@JJJAAW4LEErrorCode@@@Z 10021f50 f   ThaiLayoutEngine.obj
 0001:00021010       ??_EThaiLayoutEngine@@UAEPAXI@Z 10022010 f i ThaiLayoutEngine.obj
 0001:00021010       ??_GThaiLayoutEngine@@UAEPAXI@Z 10022010 f i ThaiLayoutEngine.obj
 0001:00021040       ?adjustGlyphPositions@ThaiLayoutEngine@@MAEXQBGJJDAAVLEGlyphStorage@@AAW4LEErrorCode@@@Z 10022040 f   ThaiLayoutEngine.obj
 0001:000210e0       ?computeGlyphs@ThaiLayoutEngine@@MAEJQBGJJJDAAVLEGlyphStorage@@AAW4LEErrorCode@@@Z 100220e0 f   ThaiLayoutEngine.obj
 0001:00021200       ?getDynamicClassID@ThaiLayoutEngine@@UBEPBDXZ 10022200 f   ThaiLayoutEngine.obj
 0001:00021210       ?compose@ThaiShaping@@SAJPBGJJEGPAGAAVLEGlyphStorage@@@Z 10022210 f   ThaiShaping.obj
 0001:00021420       ?doTransition@ThaiShaping@@CAEUStateTransition@1@GJEGPAGAAVLEGlyphStorage@@AAJ@Z 10022420 f   ThaiShaping.obj
 0001:000217b0       ??0TibetanOpenTypeLayoutEngine@@QAE@PBVLEFontInstance@@JJJABV?$LEReferenceTo@UGlyphSubstitutionTableHeader@@@@AAW4LEErrorCode@@@Z 100227b0 f   TibetanLayoutEngine.obj
 0001:000217f0       ??_ETibetanOpenTypeLayoutEngine@@UAEPAXI@Z 100227f0 f i TibetanLayoutEngine.obj
 0001:000217f0       ??_GTibetanOpenTypeLayoutEngine@@UAEPAXI@Z 100227f0 f i TibetanLayoutEngine.obj
 0001:00021820       ?characterProcessing@TibetanOpenTypeLayoutEngine@@MAEJQBGJJJDAAPAGAAVLEGlyphStorage@@AAW4LEErrorCode@@@Z 10022820 f   TibetanLayoutEngine.obj
 0001:00021940       ?getDynamicClassID@TibetanOpenTypeLayoutEngine@@UBEPBDXZ 10022940 f   TibetanLayoutEngine.obj
 0001:00021950       ?getFeatureMap@TibetanReordering@@SAPBUFeatureMap@@AAJ@Z 10022950 f   TibetanReordering.obj
 0001:00021960       ?reorder@TibetanReordering@@SAJPBGJJPAGAAVLEGlyphStorage@@@Z 10022960 f   TibetanReordering.obj
 0001:00021c90       ??0TrimmedArrayProcessor@@QAE@ABV?$LEReferenceTo@UMorphSubtableHeader@@@@AAW4LEErrorCode@@@Z 10022c90 f   TrimmedArrayProcessor.obj
 0001:00021e30       ??_ETrimmedArrayProcessor@@UAEPAXI@Z 10022e30 f i TrimmedArrayProcessor.obj
 0001:00021e30       ??_GTrimmedArrayProcessor@@UAEPAXI@Z 10022e30 f i TrimmedArrayProcessor.obj
 0001:00021e60       ?getDynamicClassID@TrimmedArrayProcessor@@UBEPBDXZ 10022e60 f   TrimmedArrayProcessor.obj
 0001:00021e70       ?process@TrimmedArrayProcessor@@UAEXAAVLEGlyphStorage@@AAW4LEErrorCode@@@Z 10022e70 f   TrimmedArrayProcessor.obj
 0001:00021ee0       ??0TrimmedArrayProcessor2@@QAE@ABV?$LEReferenceTo@UMorphSubtableHeader2@@@@AAW4LEErrorCode@@@Z 10022ee0 f   TrimmedArrayProcessor2.obj
 0001:00022170       ??_ETrimmedArrayProcessor2@@UAEPAXI@Z 10023170 f i TrimmedArrayProcessor2.obj
 0001:00022170       ??_GTrimmedArrayProcessor2@@UAEPAXI@Z 10023170 f i TrimmedArrayProcessor2.obj
 0001:000221b0       ?getDynamicClassID@TrimmedArrayProcessor2@@UBEPBDXZ 100231b0 f   TrimmedArrayProcessor2.obj
 0001:000221c0       ?process@TrimmedArrayProcessor2@@UAEXAAVLEGlyphStorage@@AAW4LEErrorCode@@@Z 100231c0 f   TrimmedArrayProcessor2.obj
 0001:00022240       ?adjustPosition@ValueRecord@@QBEXFGABVLETableReference@@AAVGlyphIterator@@PBVLEFontInstance@@AAW4LEErrorCode@@@Z 10023240 f   ValueRecords.obj
 0001:00022880       ?adjustPosition@ValueRecord@@QBEXGABVLETableReference@@AAVGlyphIterator@@PBVLEFontInstance@@AAW4LEErrorCode@@@Z 10023880 f   ValueRecords.obj
 0001:00022d30       ?getSize@ValueRecord@@SAFG@Z 10023d30 f   ValueRecords.obj
 0001:000232e0       _Java_sun_awt_Win32FontManager_getFontPath@12 100242e0 f   fontpath.obj
 0001:00023460       _Java_sun_awt_Win32FontManager_populateFontFileNameMap0@24 10024460 f   fontpath.obj
 0001:00023c20       _StringCchCatA@12          10024c20 f i fontpath.obj
 0001:000240a0       _Java_sun_font_FreetypeFontScaler_createScalerContextNative@36 100250a0 f   freetypeScaler.obj
 0001:000242a0       _Java_sun_font_FreetypeFontScaler_disposeNativeScaler@20 100252a0 f   freetypeScaler.obj
 0001:00024310       _Java_sun_font_FreetypeFontScaler_getFontMetricsNative@28 10025310 f   freetypeScaler.obj
 0001:00024630       _Java_sun_font_FreetypeFontScaler_getGlyphAdvanceNative@32 10025630 f   freetypeScaler.obj
 0001:00024690       _Java_sun_font_FreetypeFontScaler_getGlyphCodeNative@24 10025690 f   freetypeScaler.obj
 0001:00024740       _Java_sun_font_FreetypeFontScaler_getGlyphImageNative@32 10025740 f   freetypeScaler.obj
 0001:00024770       _Java_sun_font_FreetypeFontScaler_getGlyphMetricsNative@36 10025770 f   freetypeScaler.obj
 0001:00024830       _Java_sun_font_FreetypeFontScaler_getGlyphOutlineBoundsNative@32 10025830 f   freetypeScaler.obj
 0001:000249b0       _Java_sun_font_FreetypeFontScaler_getGlyphOutlineNative@40 100259b0 f   freetypeScaler.obj
 0001:00024a10       _Java_sun_font_FreetypeFontScaler_getGlyphPointNative@36 10025a10 f   freetypeScaler.obj
 0001:00024ae0       _Java_sun_font_FreetypeFontScaler_getGlyphVectorOutlineNative@44 10025ae0 f   freetypeScaler.obj
 0001:00024d30       _Java_sun_font_FreetypeFontScaler_getLayoutTableCacheNative@16 10025d30 f   freetypeScaler.obj
 0001:00024d80       _Java_sun_font_FreetypeFontScaler_getMissingGlyphCodeNative@16 10025d80 f   freetypeScaler.obj
 0001:00024d90       _Java_sun_font_FreetypeFontScaler_getNumGlyphsNative@16 10025d90 f   freetypeScaler.obj
 0001:00024e20       _Java_sun_font_FreetypeFontScaler_getUnitsPerEMNative@16 10025e20 f   freetypeScaler.obj
 0001:00024e40       _Java_sun_font_FreetypeFontScaler_initIDs@12 10025e40 f   freetypeScaler.obj
 0001:00024e70       _Java_sun_font_FreetypeFontScaler_initNativeScaler@28 10025e70 f   freetypeScaler.obj
 0001:00025c40       _Java_sun_font_FileFontStrike__1getGlyphImageFromWindows@32 10026c40 f   lcdglyph.obj
 0001:000265d0       _Java_sun_font_FileFontStrike_initNative@8 100275d0 f   lcdglyph.obj
 0001:00026600       _Java_sun_font_NullFontScaler_getGlyphImage@20 10027600 f   sunFont.obj
 0001:00026620       _Java_sun_font_NullFontScaler_getNullScalerContext@8 10027620 f   sunFont.obj
 0001:00026640       _Java_sun_font_StrikeCache_freeIntMemory@20 10027640 f   sunFont.obj
 0001:000266f0       _Java_sun_font_StrikeCache_freeIntPointer@12 100276f0 f   sunFont.obj
 0001:00026710       _Java_sun_font_StrikeCache_freeLongMemory@20 10027710 f   sunFont.obj
 0001:000267c0       _Java_sun_font_StrikeCache_freeLongPointer@16 100277c0 f   sunFont.obj
 0001:000267e0       _Java_sun_font_StrikeCache_getGlyphCacheDescription@12 100277e0 f   sunFont.obj
 0001:00026900       _Java_sun_font_SunFontManager_initIDs@8 10027900 f   sunFont.obj
 0001:00026910       _freeLayoutTableCache      10027910 f   sunFont.obj
 0001:00026950       _getSunFontIDs             10027950 f   sunFont.obj
 0001:00026f50       _isNullScalerContext       10027f50 f   sunFont.obj
 0001:00026f60       _newLayoutTableCache       10027f60 f   sunFont.obj
 0001:00026f9c       _FT_Init_FreeType          10027f9c f   freetype:freetype.dll
 0001:00026fa2       _FT_Done_FreeType          10027fa2 f   freetype:freetype.dll
 0001:00026fa8       _FT_New_Memory_Face        10027fa8 f   freetype:freetype.dll
 0001:00026fae       _FT_Open_Face              10027fae f   freetype:freetype.dll
 0001:00026fb4       _FT_Done_Face              10027fb4 f   freetype:freetype.dll
 0001:00026fba       _FT_Set_Char_Size          10027fba f   freetype:freetype.dll
 0001:00026fc0       _FT_Load_Glyph             10027fc0 f   freetype:freetype.dll
 0001:00026fc6       _FT_Set_Transform          10027fc6 f   freetype:freetype.dll
 0001:00026fcc       _FT_Render_Glyph           10027fcc f   freetype:freetype.dll
 0001:00026fd2       _FT_Get_Char_Index         10027fd2 f   freetype:freetype.dll
 0001:00026fd8       _FT_MulFix                 10027fd8 f   freetype:freetype.dll
 0001:00026fde       _FT_Matrix_Multiply        10027fde f   freetype:freetype.dll
 0001:00026fe4       _FT_Outline_Get_BBox       10027fe4 f   freetype:freetype.dll
 0001:00026fea       _FT_Activate_Size          10027fea f   freetype:freetype.dll
 0001:00026ff0       _FT_Outline_Decompose      10027ff0 f   freetype:freetype.dll
 0001:00026ff6       _FT_Outline_Get_CBox       10027ff6 f   freetype:freetype.dll
 0001:00026ffe       _FT_Outline_Translate      10027ffe f   freetype:freetype.dll
 0001:00027004       _FT_GlyphSlot_Embolden     10028004 f   freetype:freetype.dll
 0001:0002700a       _FT_Library_SetLcdFilter   1002800a f   freetype:freetype.dll
 0001:00027010       _FT_Property_Set           10028010 f   freetype:freetype.dll
 0001:00027016       _JNU_ThrowArrayIndexOutOfBoundsException@8 10028016 f   java:java.dll
 0001:0002701c       _JNU_ThrowInternalError@8  1002801c f   java:java.dll
 0001:00027022       _JNU_NewStringPlatform@8   10028022 f   java:java.dll
 0001:00027028       _SurfaceData_GetOps@8      10028028 f   awt:awt.dll
 0001:0002702e       _SurfaceData_IntersectBounds@8 1002802e f   awt:awt.dll
 0001:00027034       _GetNativePrim@8           10028034 f   awt:awt.dll
 0001:0002703a       _GrPrim_Sg2dGetCompInfo@16 1002803a f   awt:awt.dll
 0001:00027040       _GrPrim_Sg2dGetClip@12     10028040 f   awt:awt.dll
 0001:00027046       _GrPrim_Sg2dGetPixel@8     10028046 f   awt:awt.dll
 0001:0002704c       _GrPrim_Sg2dGetEaRGB@8     1002804c f   awt:awt.dll
 0001:00027052       _GrPrim_Sg2dGetLCDTextContrast@8 10028052 f   awt:awt.dll
 0001:00027058       _AccelGlyphCache_RemoveAllCellInfos 10028058 f   awt:awt.dll
 0001:0002705e       ??2@YAPAXI@Z               1002805e f   MSVCRT:new_scalar.obj
 0001:00027090       __ftol2_sse                10028090 f   MSVCRT:ftol2.obj
 0001:000270a0       __ftoi2                    100280a0 f   MSVCRT:ftol2.obj
 0001:0002711c       ??3@YAXPAXI@Z              1002811c f   MSVCRT:delete_scalar_size.obj
 0001:0002712a       ??_Etype_info@@UAEPAXI@Z   1002812a f i MSVCRT:std_type_info_static.obj
 0001:0002712a       ??_Gtype_info@@UAEPAXI@Z   1002812a f i MSVCRT:std_type_info_static.obj
 0001:0002714d       @__security_check_cookie@4 1002814d f   MSVCRT:secchk.obj
 0001:0002715b       ??_U@YAPAXI@Z              1002815b f   MSVCRT:new_array.obj
 0001:00027164       ??_V@YAXPAXI@Z             10028164 f   MSVCRT:delete_array_size.obj
 0001:00027180       __ftol3                    10028180 f   MSVCRT:ftol3.obj
 0001:000271f0       __alloca_probe_16          100281f0 f   MSVCRT:alloca16.obj
 0001:00027206       __alloca_probe_8           10028206     MSVCRT:alloca16.obj
 0001:0002755c       __DllMainCRTStartup@12     1002855c f   MSVCRT:dll_dllmain.obj
 0001:0002757f       ??0bad_alloc@std@@QAE@ABV01@@Z 1002857f f i MSVCRT:throw_bad_alloc.obj
 0001:0002759a       ??0bad_alloc@std@@QAE@XZ   1002859a f i MSVCRT:throw_bad_alloc.obj
 0001:000275b2       ??0bad_array_new_length@std@@QAE@ABV01@@Z 100285b2 f i MSVCRT:throw_bad_alloc.obj
 0001:000275cd       ??0bad_array_new_length@std@@QAE@XZ 100285cd f i MSVCRT:throw_bad_alloc.obj
 0001:000275e5       ??0exception@std@@QAE@ABV01@@Z 100285e5 f i MSVCRT:throw_bad_alloc.obj
 0001:00027611       ??1bad_alloc@std@@UAE@XZ   10028611 f i MSVCRT:throw_bad_alloc.obj
 0001:00027611       ??1bad_array_new_length@std@@UAE@XZ 10028611 f i MSVCRT:throw_bad_alloc.obj
 0001:00027622       ??_Ebad_alloc@std@@UAEPAXI@Z 10028622 f i MSVCRT:throw_bad_alloc.obj
 0001:00027622       ??_Ebad_array_new_length@std@@UAEPAXI@Z 10028622 f i MSVCRT:throw_bad_alloc.obj
 0001:00027622       ??_Eexception@std@@UAEPAXI@Z 10028622 f i MSVCRT:throw_bad_alloc.obj
 0001:00027622       ??_Gbad_alloc@std@@UAEPAXI@Z 10028622 f i MSVCRT:throw_bad_alloc.obj
 0001:00027622       ??_Gbad_array_new_length@std@@UAEPAXI@Z 10028622 f i MSVCRT:throw_bad_alloc.obj
 0001:00027622       ??_Gexception@std@@UAEPAXI@Z 10028622 f i MSVCRT:throw_bad_alloc.obj
 0001:0002764f       ?__scrt_throw_std_bad_alloc@@YAXXZ 1002864f f   MSVCRT:throw_bad_alloc.obj
 0001:0002766c       ?__scrt_throw_std_bad_array_new_length@@YAXXZ 1002866c f   MSVCRT:throw_bad_alloc.obj
 0001:00027689       ?what@exception@std@@UBEPBDXZ 10028689 f i MSVCRT:throw_bad_alloc.obj
 0001:00027696       ___isa_available_init      10028696 f   MSVCRT:cpu_disp.obj
 0001:0002786a       ??3@YAXPAX@Z               1002886a f   MSVCRT:delete_scalar.obj
 0001:0002786f       ___raise_securityfailure   1002886f f   MSVCRT:gs_report.obj
 0001:00027897       ___report_gsfailure        10028897 f   MSVCRT:gs_report.obj
 0001:00027991       ??_V@YAXPAX@Z              10028991 f   MSVCRT:delete_array.obj
 0001:000279a0       __alloca_probe             100289a0 f   MSVCRT:chkstk.obj
 0001:000279a0       __chkstk                   100289a0 f   MSVCRT:chkstk.obj
 0001:00027a18       ___security_init_cookie    10028a18 f   MSVCRT:gs_support.obj
 0001:00027a63       _DllMain@12                10028a63 f   MSVCRT:dll_dllmain_stub.obj
 0001:00027a85       ?__scrt_initialize_type_info@@YAXXZ 10028a85 f   MSVCRT:tncleanup.obj
 0001:00027a91       ?__scrt_uninitialize_type_info@@YAXXZ 10028a91 f   MSVCRT:tncleanup.obj
 0001:00027a9d       ___local_stdio_printf_options 10028a9d f i MSVCRT:default_local_stdio_options.obj
 0001:00027aa3       ___local_stdio_scanf_options 10028aa3 f i MSVCRT:default_local_stdio_options.obj
 0001:00027aa9       ___scrt_initialize_default_local_stdio_options 10028aa9 f   MSVCRT:default_local_stdio_options.obj
 0001:00027b0a       ___scrt_acquire_startup_lock 10028b0a f   MSVCRT:utility.obj
 0001:00027b3c       ___scrt_dllmain_after_initialize_c 10028b3c f   MSVCRT:utility.obj
 0001:00027b67       ___scrt_dllmain_before_initialize_c 10028b67 f   MSVCRT:utility.obj
 0001:00027b75       ___scrt_dllmain_crt_thread_attach 10028b75 f   MSVCRT:utility.obj
 0001:00027b94       ___scrt_dllmain_crt_thread_detach 10028b94 f   MSVCRT:utility.obj
 0001:00027ba1       ___scrt_dllmain_exception_filter 10028ba1 f   MSVCRT:utility.obj
 0001:00027bd5       ___scrt_dllmain_uninitialize_c 10028bd5 f   MSVCRT:utility.obj
 0001:00027bf8       ___scrt_dllmain_uninitialize_critical 10028bf8 f   MSVCRT:utility.obj
 0001:00027c05       ___scrt_initialize_crt     10028c05 f   MSVCRT:utility.obj
 0001:00027c3e       ___scrt_initialize_onexit_tables 10028c3e f   MSVCRT:utility.obj
 0001:00027cc5       ___scrt_is_nonwritable_in_current_image 10028cc5 f   MSVCRT:utility.obj
 0001:00027d59       ___scrt_release_startup_lock 10028d59 f   MSVCRT:utility.obj
 0001:00027d76       ___scrt_uninitialize_crt   10028d76 f   MSVCRT:utility.obj
 0001:00027d9e       ___scrt_get_dyn_tls_init_callback 10028d9e f   MSVCRT:dyn_tls_init.obj
 0001:00027da4       ___scrt_fastfail           10028da4 f   MSVCRT:utility_desktop.obj
 0001:00027ebf       __crt_debugger_hook        10028ebf f   MSVCRT:utility_desktop.obj
 0001:00027ec7       __RTC_Initialize           10028ec7 f   MSVCRT:initsect.obj
 0001:00027ef3       __RTC_Terminate            10028ef3 f   MSVCRT:initsect.obj
 0001:00027f20       __SEH_prolog4              10028f20 f   MSVCRT:sehprolg4.obj
 0001:00027f65       __except_handler4          10028f65 f   MSVCRT:chandler4gs.obj
 0001:00027f94       __get_startup_argv_mode    10028f94 f   MSVCRT:argv_mode.obj
 0001:00027f98       ___scrt_is_ucrt_dll_in_use 10028f98 f   MSVCRT:ucrt_detection.obj
 0001:00027fa4       _memset                    10028fa4 f   vcruntime:VCRUNTIME140.dll
 0001:00027faa       __purecall                 10028faa f   vcruntime:VCRUNTIME140.dll
 0001:00027fb0       _memcpy                    10028fb0 f   vcruntime:VCRUNTIME140.dll
 0001:00027fb6       _strrchr                   10028fb6 f   vcruntime:VCRUNTIME140.dll
 0001:00027fbc       _strstr                    10028fbc f   vcruntime:VCRUNTIME140.dll
 0001:00027fc2       _wcsrchr                   10028fc2 f   vcruntime:VCRUNTIME140.dll
 0001:00027fc8       _wcsstr                    10028fc8 f   vcruntime:VCRUNTIME140.dll
 0001:00027fce       ___std_exception_copy      10028fce f   vcruntime:VCRUNTIME140.dll
 0001:00027fd4       ___std_exception_destroy   10028fd4 f   vcruntime:VCRUNTIME140.dll
 0001:00027fda       __CxxThrowException@8      10028fda f   vcruntime:VCRUNTIME140.dll
 0001:00027fe0       ___std_type_info_destroy_list 10028fe0 f   vcruntime:VCRUNTIME140.dll
 0001:00027fe6       __except_handler4_common   10028fe6 f   vcruntime:VCRUNTIME140.dll
 0001:00027fec       _free                      10028fec f   ucrt:api-ms-win-crt-heap-l1-1-0.dll
 0001:00027ff2       _malloc                    10028ff2 f   ucrt:api-ms-win-crt-heap-l1-1-0.dll
 0001:00027ff8       __libm_sse2_pow_precise    10028ff8 f   ucrt:api-ms-win-crt-math-l1-1-0.dll
 0001:00027ffe       _floor                     10028ffe f   ucrt:api-ms-win-crt-math-l1-1-0.dll
 0001:00028004       __libm_sse2_sqrt_precise   10029004 f   ucrt:api-ms-win-crt-math-l1-1-0.dll
 0001:0002800a       __callnewh                 1002900a f   ucrt:api-ms-win-crt-heap-l1-1-0.dll
 0001:00028010       __initterm                 10029010 f   ucrt:api-ms-win-crt-runtime-l1-1-0.dll
 0001:00028016       __initterm_e               10029016 f   ucrt:api-ms-win-crt-runtime-l1-1-0.dll
 0001:0002801c       __seh_filter_dll           1002901c f   ucrt:api-ms-win-crt-runtime-l1-1-0.dll
 0001:00028022       __configure_narrow_argv    10029022 f   ucrt:api-ms-win-crt-runtime-l1-1-0.dll
 0001:00028028       __initialize_narrow_environment 10029028 f   ucrt:api-ms-win-crt-runtime-l1-1-0.dll
 0001:0002802e       __initialize_onexit_table  1002902e f   ucrt:api-ms-win-crt-runtime-l1-1-0.dll
 0001:00028034       __execute_onexit_table     10029034 f   ucrt:api-ms-win-crt-runtime-l1-1-0.dll
 0001:0002803a       __cexit                    1002903a f   ucrt:api-ms-win-crt-runtime-l1-1-0.dll
 0001:00028040       ___acrt_initialize         10029040 f   MSVCRT:ucrt_stubs.obj
 0001:00028040       ___acrt_thread_attach      10029040 f   MSVCRT:ucrt_stubs.obj
 0001:00028040       ___acrt_thread_detach      10029040 f   MSVCRT:ucrt_stubs.obj
 0001:00028040       ___acrt_uninitialize       10029040 f   MSVCRT:ucrt_stubs.obj
 0001:00028040       ___acrt_uninitialize_critical 10029040 f   MSVCRT:ucrt_stubs.obj
 0001:00028040       ___scrt_stub_for_acrt_initialize 10029040 f   MSVCRT:ucrt_stubs.obj
 0001:00028040       ___scrt_stub_for_acrt_thread_attach 10029040 f   MSVCRT:ucrt_stubs.obj
 0001:00028040       ___scrt_stub_for_acrt_thread_detach 10029040 f   MSVCRT:ucrt_stubs.obj
 0001:00028040       ___scrt_stub_for_acrt_uninitialize 10029040 f   MSVCRT:ucrt_stubs.obj
 0001:00028040       ___scrt_stub_for_acrt_uninitialize_critical 10029040 f   MSVCRT:ucrt_stubs.obj
 0001:00028040       ___vcrt_initialize         10029040 f   MSVCRT:ucrt_stubs.obj
 0001:00028040       ___vcrt_thread_attach      10029040 f   MSVCRT:ucrt_stubs.obj
 0001:00028040       ___vcrt_thread_detach      10029040 f   MSVCRT:ucrt_stubs.obj
 0001:00028040       ___vcrt_uninitialize       10029040 f   MSVCRT:ucrt_stubs.obj
 0001:00028040       ___vcrt_uninitialize_critical 10029040 f   MSVCRT:ucrt_stubs.obj
 0001:00028043       __filter_x86_sse2_floating_point_exception 10029043 f   MSVCRT:x86_exception_filter.obj
 0001:00028043       __filter_x86_sse2_floating_point_exception_default 10029043 f   MSVCRT:x86_exception_filter.obj
 0002:00000000       __imp__RegCloseKey@4       1002a000     advapi32:ADVAPI32.dll
 0002:00000004       __imp__RegEnumValueW@32    1002a004     advapi32:ADVAPI32.dll
 0002:00000008       __imp__RegOpenKeyExA@20    1002a008     advapi32:ADVAPI32.dll
 0002:0000000c       __imp__RegQueryInfoKeyA@48 1002a00c     advapi32:ADVAPI32.dll
 0002:00000010       __imp__RegQueryInfoKeyW@48 1002a010     advapi32:ADVAPI32.dll
 0002:00000014       __imp__RegEnumValueA@32    1002a014     advapi32:ADVAPI32.dll
 0002:00000018       \177ADVAPI32_NULL_THUNK_DATA 1002a018     advapi32:ADVAPI32.dll
 0002:0000001c       __imp__GetGlyphOutlineA@28 1002a01c     gdi32:GDI32.dll
 0002:00000020       __imp__GetFontData@20      1002a020     gdi32:GDI32.dll
 0002:00000024       __imp__GetDIBits@28        1002a024     gdi32:GDI32.dll
 0002:00000028       __imp__GetDeviceCaps@8     1002a028     gdi32:GDI32.dll
 0002:0000002c       __imp__SelectObject@8      1002a02c     gdi32:GDI32.dll
 0002:00000030       __imp__CreateFontIndirectW@4 1002a030     gdi32:GDI32.dll
 0002:00000034       __imp__CreateCompatibleDC@4 1002a034     gdi32:GDI32.dll
 0002:00000038       __imp__CreateCompatibleBitmap@12 1002a038     gdi32:GDI32.dll
 0002:0000003c       __imp__EnumFontFamiliesExW@20 1002a03c     gdi32:GDI32.dll
 0002:00000040       __imp__EnumFontFamiliesExA@20 1002a040     gdi32:GDI32.dll
 0002:00000044       __imp__GetStockObject@4    1002a044     gdi32:GDI32.dll
 0002:00000048       __imp__SetBkColor@8        1002a048     gdi32:GDI32.dll
 0002:0000004c       __imp__SetTextColor@8      1002a04c     gdi32:GDI32.dll
 0002:00000050       __imp__GetTextMetricsA@8   1002a050     gdi32:GDI32.dll
 0002:00000054       __imp__ExtTextOutW@32      1002a054     gdi32:GDI32.dll
 0002:00000058       __imp__DeleteObject@4      1002a058     gdi32:GDI32.dll
 0002:0000005c       __imp__SetMapMode@8        1002a05c     gdi32:GDI32.dll
 0002:00000060       \177GDI32_NULL_THUNK_DATA  1002a060     gdi32:GDI32.dll
 0002:00000064       __imp__IsProcessorFeaturePresent@4 1002a064     kernel32:KERNEL32.dll
 0002:00000068       __imp__GetVersion@0        1002a068     kernel32:KERNEL32.dll
 0002:0000006c       __imp__QueryPerformanceCounter@4 1002a06c     kernel32:KERNEL32.dll
 0002:00000070       __imp__GetVersionExA@4     1002a070     kernel32:KERNEL32.dll
 0002:00000074       __imp__TerminateProcess@8  1002a074     kernel32:KERNEL32.dll
 0002:00000078       __imp__GetWindowsDirectoryA@8 1002a078     kernel32:KERNEL32.dll
 0002:0000007c       __imp__GetSystemDirectoryA@8 1002a07c     kernel32:KERNEL32.dll
 0002:00000080       __imp__SetUnhandledExceptionFilter@4 1002a080     kernel32:KERNEL32.dll
 0002:00000084       __imp__GetCurrentThreadId@0 1002a084     kernel32:KERNEL32.dll
 0002:00000088       __imp__GetSystemTimeAsFileTime@4 1002a088     kernel32:KERNEL32.dll
 0002:0000008c       __imp__DisableThreadLibraryCalls@4 1002a08c     kernel32:KERNEL32.dll
 0002:00000090       __imp__InitializeSListHead@4 1002a090     kernel32:KERNEL32.dll
 0002:00000094       __imp__IsDebuggerPresent@0 1002a094     kernel32:KERNEL32.dll
 0002:00000098       __imp__GetCurrentProcessId@0 1002a098     kernel32:KERNEL32.dll
 0002:0000009c       __imp__GetCurrentProcess@0 1002a09c     kernel32:KERNEL32.dll
 0002:000000a0       __imp__UnhandledExceptionFilter@4 1002a0a0     kernel32:KERNEL32.dll
 0002:000000a4       \177KERNEL32_NULL_THUNK_DATA 1002a0a4     kernel32:KERNEL32.dll
 0002:000000a8       __imp__GetDesktopWindow@0  1002a0a8     user32:USER32.dll
 0002:000000ac       __imp__SystemParametersInfoA@16 1002a0ac     user32:USER32.dll
 0002:000000b0       __imp__GetWindowDC@4       1002a0b0     user32:USER32.dll
 0002:000000b4       __imp__ReleaseDC@8         1002a0b4     user32:USER32.dll
 0002:000000b8       __imp__GetDC@4             1002a0b8     user32:USER32.dll
 0002:000000bc       __imp__FillRect@12         1002a0bc     user32:USER32.dll
 0002:000000c0       \177USER32_NULL_THUNK_DATA 1002a0c0     user32:USER32.dll
 0002:000000c4       __imp__memcpy              1002a0c4     vcruntime:VCRUNTIME140.dll
 0002:000000c8       __imp__wcsrchr             1002a0c8     vcruntime:VCRUNTIME140.dll
 0002:000000cc       __imp__wcsstr              1002a0cc     vcruntime:VCRUNTIME140.dll
 0002:000000d0       __imp___purecall           1002a0d0     vcruntime:VCRUNTIME140.dll
 0002:000000d4       __imp__strstr              1002a0d4     vcruntime:VCRUNTIME140.dll
 0002:000000d8       __imp__memset              1002a0d8     vcruntime:VCRUNTIME140.dll
 0002:000000dc       __imp____std_exception_copy 1002a0dc     vcruntime:VCRUNTIME140.dll
 0002:000000e0       __imp__strrchr             1002a0e0     vcruntime:VCRUNTIME140.dll
 0002:000000e4       __imp____std_type_info_destroy_list 1002a0e4     vcruntime:VCRUNTIME140.dll
 0002:000000e8       __imp___CxxThrowException@8 1002a0e8     vcruntime:VCRUNTIME140.dll
 0002:000000ec       __imp____std_exception_destroy 1002a0ec     vcruntime:VCRUNTIME140.dll
 0002:000000f0       __imp___except_handler4_common 1002a0f0     vcruntime:VCRUNTIME140.dll
 0002:000000f4       \177VCRUNTIME140_NULL_THUNK_DATA 1002a0f4     vcruntime:VCRUNTIME140.dll
 0002:000000f8       __imp__getenv              1002a0f8     ucrt:api-ms-win-crt-environment-l1-1-0.dll
 0002:000000fc       \177api-ms-win-crt-environment-l1-1-0_NULL_THUNK_DATA 1002a0fc     ucrt:api-ms-win-crt-environment-l1-1-0.dll
 0002:00000100       __imp___callnewh           1002a100     ucrt:api-ms-win-crt-heap-l1-1-0.dll
 0002:00000104       __imp__realloc             1002a104     ucrt:api-ms-win-crt-heap-l1-1-0.dll
 0002:00000108       __imp__calloc              1002a108     ucrt:api-ms-win-crt-heap-l1-1-0.dll
 0002:0000010c       __imp__malloc              1002a10c     ucrt:api-ms-win-crt-heap-l1-1-0.dll
 0002:00000110       __imp__free                1002a110     ucrt:api-ms-win-crt-heap-l1-1-0.dll
 0002:00000114       \177api-ms-win-crt-heap-l1-1-0_NULL_THUNK_DATA 1002a114     ucrt:api-ms-win-crt-heap-l1-1-0.dll
 0002:00000118       __imp___libm_sse2_sqrt_precise 1002a118     ucrt:api-ms-win-crt-math-l1-1-0.dll
 0002:0000011c       __imp___libm_sse2_pow_precise 1002a11c     ucrt:api-ms-win-crt-math-l1-1-0.dll
 0002:00000120       __imp__floor               1002a120     ucrt:api-ms-win-crt-math-l1-1-0.dll
 0002:00000124       \177api-ms-win-crt-math-l1-1-0_NULL_THUNK_DATA 1002a124     ucrt:api-ms-win-crt-math-l1-1-0.dll
 0002:00000128       __imp___initialize_narrow_environment 1002a128     ucrt:api-ms-win-crt-runtime-l1-1-0.dll
 0002:0000012c       __imp___initialize_onexit_table 1002a12c     ucrt:api-ms-win-crt-runtime-l1-1-0.dll
 0002:00000130       __imp___configure_narrow_argv 1002a130     ucrt:api-ms-win-crt-runtime-l1-1-0.dll
 0002:00000134       __imp___cexit              1002a134     ucrt:api-ms-win-crt-runtime-l1-1-0.dll
 0002:00000138       __imp___initterm           1002a138     ucrt:api-ms-win-crt-runtime-l1-1-0.dll
 0002:0000013c       __imp___initterm_e         1002a13c     ucrt:api-ms-win-crt-runtime-l1-1-0.dll
 0002:00000140       __imp___seh_filter_dll     1002a140     ucrt:api-ms-win-crt-runtime-l1-1-0.dll
 0002:00000144       __imp___execute_onexit_table 1002a144     ucrt:api-ms-win-crt-runtime-l1-1-0.dll
 0002:00000148       \177api-ms-win-crt-runtime-l1-1-0_NULL_THUNK_DATA 1002a148     ucrt:api-ms-win-crt-runtime-l1-1-0.dll
 0002:0000014c       __imp___stricmp            1002a14c     ucrt:api-ms-win-crt-string-l1-1-0.dll
 0002:0000014c       __imp__stricmp             1002a14c     ucrt:api-ms-win-crt-string-l1-1-0.dll
 0002:00000150       __imp___wcsicmp            1002a150     ucrt:api-ms-win-crt-string-l1-1-0.dll
 0002:00000150       __imp__wcsicmp             1002a150     ucrt:api-ms-win-crt-string-l1-1-0.dll
 0002:00000154       \177api-ms-win-crt-string-l1-1-0_NULL_THUNK_DATA 1002a154     ucrt:api-ms-win-crt-string-l1-1-0.dll
 0002:00000158       __imp__SurfaceData_GetOps@8 1002a158     awt:awt.dll
 0002:0000015c       __imp__SurfaceData_IntersectBounds@8 1002a15c     awt:awt.dll
 0002:00000160       __imp__GetNativePrim@8     1002a160     awt:awt.dll
 0002:00000164       __imp__GrPrim_Sg2dGetCompInfo@16 1002a164     awt:awt.dll
 0002:00000168       __imp__GrPrim_Sg2dGetClip@12 1002a168     awt:awt.dll
 0002:0000016c       __imp__GrPrim_Sg2dGetPixel@8 1002a16c     awt:awt.dll
 0002:00000170       __imp__GrPrim_Sg2dGetEaRGB@8 1002a170     awt:awt.dll
 0002:00000174       __imp__GrPrim_Sg2dGetLCDTextContrast@8 1002a174     awt:awt.dll
 0002:00000178       __imp__AccelGlyphCache_RemoveAllCellInfos 1002a178     awt:awt.dll
 0002:0000017c       \177awt_NULL_THUNK_DATA    1002a17c     awt:awt.dll
 0002:00000180       __imp__FT_Done_FreeType    1002a180     freetype:freetype.dll
 0002:00000184       __imp__FT_New_Memory_Face  1002a184     freetype:freetype.dll
 0002:00000188       __imp__FT_Open_Face        1002a188     freetype:freetype.dll
 0002:0000018c       __imp__FT_Done_Face        1002a18c     freetype:freetype.dll
 0002:00000190       __imp__FT_Set_Char_Size    1002a190     freetype:freetype.dll
 0002:00000194       __imp__FT_Property_Set     1002a194     freetype:freetype.dll
 0002:00000198       __imp__FT_Library_SetLcdFilter 1002a198     freetype:freetype.dll
 0002:0000019c       __imp__FT_GlyphSlot_Embolden 1002a19c     freetype:freetype.dll
 0002:000001a0       __imp__FT_Outline_Translate 1002a1a0     freetype:freetype.dll
 0002:000001a4       __imp__FT_Outline_Get_CBox 1002a1a4     freetype:freetype.dll
 0002:000001a8       __imp__FT_Outline_Decompose 1002a1a8     freetype:freetype.dll
 0002:000001ac       __imp__FT_Activate_Size    1002a1ac     freetype:freetype.dll
 0002:000001b0       __imp__FT_Outline_Get_BBox 1002a1b0     freetype:freetype.dll
 0002:000001b4       __imp__FT_Matrix_Multiply  1002a1b4     freetype:freetype.dll
 0002:000001b8       __imp__FT_MulFix           1002a1b8     freetype:freetype.dll
 0002:000001bc       __imp__FT_Get_Char_Index   1002a1bc     freetype:freetype.dll
 0002:000001c0       __imp__FT_Render_Glyph     1002a1c0     freetype:freetype.dll
 0002:000001c4       __imp__FT_Set_Transform    1002a1c4     freetype:freetype.dll
 0002:000001c8       __imp__FT_Load_Glyph       1002a1c8     freetype:freetype.dll
 0002:000001cc       __imp__FT_Init_FreeType    1002a1cc     freetype:freetype.dll
 0002:000001d0       \177freetype_NULL_THUNK_DATA 1002a1d0     freetype:freetype.dll
 0002:000001d4       __imp__JNU_NewStringPlatform@8 1002a1d4     java:java.dll
 0002:000001d8       __imp__JNU_ThrowInternalError@8 1002a1d8     java:java.dll
 0002:000001dc       __imp__JNU_ThrowArrayIndexOutOfBoundsException@8 1002a1dc     java:java.dll
 0002:000001e0       \177java_NULL_THUNK_DATA   1002a1e0     java:java.dll
 0002:000001e4       ___guard_check_icall_fptr  1002a1e4     MSVCRT:guard_support.obj
 0002:000001e8       ___castguard_check_failure_os_handled_fptr 1002a1e8     MSVCRT:guard_support.obj
 0002:000001ec       ___xc_a                    1002a1ec     MSVCRT:initializers.obj
 0002:000001f0       ___xc_z                    1002a1f0     MSVCRT:initializers.obj
 0002:000001f4       ___xi_a                    1002a1f4     MSVCRT:initializers.obj
 0002:000001f8       ___xi_z                    1002a1f8     MSVCRT:initializers.obj
 0002:000001fc       ___xp_a                    1002a1fc     MSVCRT:initializers.obj
 0002:00000200       ___xp_z                    1002a200     MSVCRT:initializers.obj
 0002:00000204       ___xt_a                    1002a204     MSVCRT:initializers.obj
 0002:00000208       ___xt_z                    1002a208     MSVCRT:initializers.obj
 0002:00000214       ??_7ArabicOpenTypeLayoutEngine@@6B@ 1002a214     ArabicLayoutEngine.obj
 0002:00000254       ??_7UnicodeArabicOpenTypeLayoutEngine@@6B@ 1002a254     ArabicLayoutEngine.obj
 0002:00000290       ?shapeTypes@ArabicShaping@@0QBJB 1002a290     ArabicShaping.obj
 0002:00000320       ?glyphSubstitutionTable@CanonShaping@@2QBEB 1002a320     CanonData.obj
 0002:0000de08       ?glyphSubstitutionTableLen@CanonShaping@@2IB 10037e08     CanonData.obj
 0002:0000de0c       ?glyphDefinitionTableLen@CanonShaping@@2IB 10037e0c     CanonData.obj
 0002:0000de10       ?glyphDefinitionTable@CanonShaping@@2QBEB 10037e10     CanonData.obj
 0002:0000e3ec       ??_7ContextualGlyphInsertionProcessor2@@6B@ 100383ec     ContextualGlyphInsertionProc2.obj
 0002:0000e408       ??_7ContextualGlyphSubstitutionProcessor@@6B@ 10038408     ContextualGlyphSubstProc.obj
 0002:0000e424       ??_7ContextualGlyphSubstitutionProcessor2@@6B@ 10038424     ContextualGlyphSubstProc2.obj
 0002:0000e43c       ?fieldMasks@DeviceTable@@0QBGB 1003843c     DeviceTables.obj
 0002:0000e444       ?fieldSignBits@DeviceTable@@0QBGB 10038444     DeviceTables.obj
 0002:0000e44c       ?fieldBits@DeviceTable@@0QBGB 1003844c     DeviceTables.obj
 0002:0000e454       __real@3e2aaaad            10038454     DrawGlyphList.obj
 0002:0000e458       __real@3f000000            10038458     DrawGlyphList.obj
 0002:0000e460       __real@3ff0000000000000    10038460     DrawGlyphList.obj
 0002:0000e468       __real@40400000            10038468     DrawGlyphList.obj
 0002:0000e470       __real@4059000000000000    10038470     DrawGlyphList.obj
 0002:0000e478       __real@406fe00000000000    10038478     DrawGlyphList.obj
 0002:0000e49c       ??_7LEFontInstance@@6B@    1003849c     FontInstanceAdapter.obj
 0002:0000e51c       ??_7FontInstanceAdapter@@6B@ 1003851c     FontInstanceAdapter.obj
 0002:0000e5a4       __real@3f800000            100385a4     FontInstanceAdapter.obj
 0002:0000e5a8       __real@42900000            100385a8     FontInstanceAdapter.obj
 0002:0000e5b0       __xmm@80000000800000008000000080000000 100385b0     FontInstanceAdapter.obj
 0002:0000e5c4       ??_7LEGlyphFilter@@6B@     100385c4     GDEFMarkFilter.obj
 0002:0000e5d0       ??_7GDEFMarkFilter@@6B@    100385d0     GDEFMarkFilter.obj
 0002:0000e5dc       ??_7GXLayoutEngine@@6B@    100385dc     GXLayoutEngine.obj
 0002:0000e610       ??_7GXLayoutEngine2@@6B@   10038610     GXLayoutEngine2.obj
 0002:0000e644       ??_7GlyphIterator@@6B@     10038644     GlyphIterator.obj
 0002:0000e64c       ??_7GlyphPositioningLookupProcessor@@6B@ 1003864c     GlyphPosnLookupProc.obj
 0002:0000e658       ??_7GlyphSubstitutionLookupProcessor@@6B@ 10038658     GlyphSubstLookupProc.obj
 0002:0000e67c       ??_7HanOpenTypeLayoutEngine@@6B@ 1003867c     HanLayoutEngine.obj
 0002:0000e7cc       ??_7HangulOpenTypeLayoutEngine@@6B@ 100387cc     HangulLayoutEngine.obj
 0002:0000fdd0       ??_7IndicOpenTypeLayoutEngine@@6B@ 10039dd0     IndicLayoutEngine.obj
 0002:0000fe10       ??_7IndicRearrangementProcessor@@6B@ 10039e10     IndicRearrangementProcessor.obj
 0002:0000fe2c       ??_7IndicRearrangementProcessor2@@6B@ 10039e2c     IndicRearrangementProcessor2.obj
 0002:0001004c       ??_7KhmerOpenTypeLayoutEngine@@6B@ 1003a04c     KhmerLayoutEngine.obj
 0002:00010378       ??_7LECharMapper@@6B@      1003a378     LEFontInstance.obj
 0002:00010384       ??_7LEInsertionCallback@@6B@ 1003a384     LEGlyphStorage.obj
 0002:00010390       ??_7LEGlyphStorage@@6B@    1003a390     LEGlyphStorage.obj
 0002:000103a0       ??_7LEInsertionList@@6B@   1003a3a0     LEInsertionList.obj
 0002:000103a8       ?controlChars@DefaultCharMapper@@0QBKB 1003a3a8     LayoutEngine.obj
 0002:000103f0       ?controlCharsCount@DefaultCharMapper@@0JB 1003a3f0     LayoutEngine.obj
 0002:000103f4       ?controlCharsZWJCount@DefaultCharMapper@@0JB 1003a3f4     LayoutEngine.obj
 0002:000103f8       ?controlCharsZWJ@DefaultCharMapper@@0QBKB 1003a3f8     LayoutEngine.obj
 0002:00010450       ?kTypoFlagKern@LayoutEngine@@2JB 1003a450     LayoutEngine.obj
 0002:00010454       ?kTypoFlagLiga@LayoutEngine@@2JB 1003a454     LayoutEngine.obj
 0002:0001045c       ??_7LayoutEngine@@6B@      1003a45c     LayoutEngine.obj
 0002:00010490       ??_7CharSubstitutionFilter@@6B@ 1003a490     LayoutEngine.obj
 0002:0001049c       ??_7DefaultCharMapper@@6B@ 1003a49c     LayoutEngine.obj
 0002:000104a8       ??_7CanonMarkFilter@@6B@   1003a4a8     LayoutEngine.obj
 0002:000104b4       ??_7LigatureSubstitutionProcessor@@6B@ 1003a4b4     LigatureSubstProc.obj
 0002:000104d0       ??_7LigatureSubstitutionProcessor2@@6B@ 1003a4d0     LigatureSubstProc2.obj
 0002:000104ec       ??_7LookupProcessor@@6B@   1003a4ec     LookupProcessor.obj
 0002:000104f8       ?mirroredChars@DefaultCharMapper@@0QBKB 1003a4f8     MirroredCharData.obj
 0002:00010a28       ?srahCderorrim@DefaultCharMapper@@0QBKB 1003aa28     MirroredCharData.obj
 0002:00010f58       ?mirroredCharsCount@DefaultCharMapper@@0JB 1003af58     MirroredCharData.obj
 0002:00010f60       ??_7NonContextualGlyphSubstitutionProcessor@@6B@ 1003af60     NonContextualGlyphSubstProc.obj
 0002:00010f6c       ??_7NonContextualGlyphSubstitutionProcessor2@@6B@ 1003af6c     NonContextualGlyphSubstProc2.obj
 0002:0001104c       ??_7OpenTypeLayoutEngine@@6B@ 1003b04c     OpenTypeLayoutEngine.obj
 0002:00011088       ?languageTags@OpenTypeLayoutEngine@@2QBKB 1003b088     ScriptAndLanguageTags.obj
 0002:000111a8       ?scriptTags@OpenTypeLayoutEngine@@0QBKB 1003b1a8     ScriptAndLanguageTags.obj
 0002:00011424       ??_7SegmentArrayProcessor@@6B@ 1003b424     SegmentArrayProcessor.obj
 0002:00011434       ??_7SegmentArrayProcessor2@@6B@ 1003b434     SegmentArrayProcessor2.obj
 0002:00011444       ??_7SegmentSingleProcessor@@6B@ 1003b444     SegmentSingleProcessor.obj
 0002:00011454       ??_7SegmentSingleProcessor2@@6B@ 1003b454     SegmentSingleProcessor2.obj
 0002:00011460       ?shapingTypeTable@ArabicShaping@@0QBEB 1003b460     ShapingTypeData.obj
 0002:00011970       ?shapingTypeTableLen@ArabicShaping@@0IB 1003b970     ShapingTypeData.obj
 0002:00011978       ??_7SimpleArrayProcessor@@6B@ 1003b978     SimpleArrayProcessor.obj
 0002:00011988       ??_7SimpleArrayProcessor2@@6B@ 1003b988     SimpleArrayProcessor2.obj
 0002:00011998       ??_7SingleTableProcessor@@6B@ 1003b998     SingleTableProcessor.obj
 0002:000119a8       ??_7SingleTableProcessor2@@6B@ 1003b9a8     SingleTableProcessor2.obj
 0002:000119b8       ??_7StateTableProcessor@@6B@ 1003b9b8     StateTableProcessor.obj
 0002:000119d0       ??_7StateTableProcessor2@@6B@ 1003b9d0     StateTableProcessor2.obj
 0002:000119e8       ??_7SubtableProcessor@@6B@ 1003b9e8     SubtableProcessor.obj
 0002:000119f4       ??_7SubtableProcessor2@@6B@ 1003b9f4     SubtableProcessor2.obj
 0002:000119fc       ??_C@_0BM@DODCGPJL@sun?1font?1GlyphLayout$GVData@ 1003b9fc     SunLayoutEngine.obj
 0002:00011a18       ??_C@_01JPJNBJEM@I@        1003ba18     SunLayoutEngine.obj
 0002:00011a1c       ??_C@_06HHPHCOMB@_count@   1003ba1c     SunLayoutEngine.obj
 0002:00011a24       ??_C@_06PPHBKICC@_flags@   1003ba24     SunLayoutEngine.obj
 0002:00011a2c       ??_C@_02EBOMBDPA@?$FLI@    1003ba2c     SunLayoutEngine.obj
 0002:00011a30       ??_C@_07PKNHOODJ@_glyphs@  1003ba30     SunLayoutEngine.obj
 0002:00011a38       ??_C@_02MGHEAPDP@?$FLF@    1003ba38     SunLayoutEngine.obj
 0002:00011a3c       ??_C@_0L@BHNDECPI@_positions@ 1003ba3c     SunLayoutEngine.obj
 0002:00011a48       ??_C@_08MEOKMKLN@_indices@ 1003ba48     SunLayoutEngine.obj
 0002:00011a54       ??_C@_0P@EFKBJFIG@count?5negative@ 1003ba54     SunLayoutEngine.obj
 0002:00011a64       ??_C@_0BA@CNGMEPKA@glypharray?5null@ 1003ba64     SunLayoutEngine.obj
 0002:00011a74       ??_C@_00CNPNBAHC@@         1003ba74     SunLayoutEngine.obj
 0002:00011a78       ??_C@_0BD@ODPDFFNE@indices?5array?5null@ 1003ba78     SunLayoutEngine.obj
 0002:00011a90       ??_7ThaiLayoutEngine@@6B@  1003ba90     ThaiLayoutEngine.obj
 0002:00011bd8       ?classTable@ThaiShaping@@0QBEB 1003bbd8     ThaiStateTables.obj
 0002:00011c38       ?thaiStateTable@ThaiShaping@@0QAY0BD@$$CBUStateTransition@1@A 1003bc38     ThaiStateTables.obj
 0002:000123f4       ??_7TibetanOpenTypeLayoutEngine@@6B@ 1003c3f4     TibetanLayoutEngine.obj
 0002:00012a24       ??_7TrimmedArrayProcessor@@6B@ 1003ca24     TrimmedArrayProcessor.obj
 0002:00012a34       ??_7TrimmedArrayProcessor2@@6B@ 1003ca34     TrimmedArrayProcessor2.obj
 0002:00012a60       __real@00000000            1003ca60     ValueRecords.obj
 0002:00012b10       ??_C@_11LOCGONAA@@         1003cb10     fontpath.obj
 0002:00012b14       ??_C@_07GCCENIMJ@?2System@ 1003cb14     fontpath.obj
 0002:00012b1c       ??_C@_09FJGNFLHN@?2System32@ 1003cb1c     fontpath.obj
 0002:00012b28       ??_C@_06MIJGMACG@?2Fonts@  1003cb28     fontpath.obj
 0002:00012b30       ??_C@_01ICJEACDI@?$DL@     1003cb30     fontpath.obj
 0002:00012b34       ??_C@_03NHMNJBCN@?5?$CG?5@ 1003cb34     fontpath.obj
 0002:00012b38       ??_C@_17BCGMALNF@?$AA?5?$AA?$CG?$AA?5@ 1003cb38     fontpath.obj
 0002:00012b40       ??_C@_0BC@LEKPNIDO@java?1util?1HashMap@ 1003cb40     fontpath.obj
 0002:00012b54       ??_C@_0DJ@FLFJBGBN@?$CILjava?1lang?1Object?$DLLjava?1lang?1O@ 1003cb54     fontpath.obj
 0002:00012b90       ??_C@_03KMONJGDG@put@      1003cb90     fontpath.obj
 0002:00012b94       ??_C@_0BG@DHOOFEJE@?$CILjava?1lang?1Object?$DL?$CJZ@ 1003cb94     fontpath.obj
 0002:00012bac       ??_C@_0M@ILMAKOC@containsKey@ 1003cbac     fontpath.obj
 0002:00012bb8       ??_C@_0BE@GPOIDJOH@java?1util?1ArrayList@ 1003cbb8     fontpath.obj
 0002:00012bcc       ??_C@_04PFANPMCN@?$CII?$CJV@ 1003cbcc     fontpath.obj
 0002:00012bd4       ??_C@_06FALKBLGB@?$DMinit?$DO@ 1003cbd4     fontpath.obj
 0002:00012bdc       ??_C@_03BDGOHNNK@add@      1003cbdc     fontpath.obj
 0002:00012be0       ??_C@_0BB@FLFAIHG@java?1lang?1String@ 1003cbe0     fontpath.obj
 0002:00012bf4       ??_C@_0CH@BHMNPKMP@?$CILjava?1util?1Locale?$DL?$CJLjava?1lang?1@ 1003cbf4     fontpath.obj
 0002:00012c1c       ??_C@_0M@IMBDOEKL@toLowerCase@ 1003cc1c     fontpath.obj
 0002:00012c28       ??_C@_19OLAFNMII@?$AA?4?$AAt?$AAt?$AAf@ 1003cc28     fontpath.obj
 0002:00012c34       ??_C@_19MKNEPBPF@?$AA?4?$AAo?$AAt?$AAf@ 1003cc34     fontpath.obj
 0002:00012c58       ??_C@_03GAEACAIP@?$CI?$CJV@ 1003cc58     freetypeScaler.obj
 0002:00012c5c       ??_C@_0BB@NIMAMPFF@invalidateScaler@ 1003cc5c     freetypeScaler.obj
 0002:00012c70       ??_C@_0BE@LLDKDDBI@FREETYPE_PROPERTIES@ 1003cc70     freetypeScaler.obj
 0002:00012c84       ??_C@_08OKLLNAKL@truetype@ 1003cc84     freetypeScaler.obj
 0002:00012c90       ??_C@_0BE@OJJAFABD@interpreter?9version@ 1003cc90     freetypeScaler.obj
 0002:00012ca4       __real@37800000            1003cca4     freetypeScaler.obj
 0002:00012ca8       __real@3c800000            1003cca8     freetypeScaler.obj
 0002:00012cb0       __real@3ef0000000000000    1003ccb0     freetypeScaler.obj
 0002:00012cb8       __real@3f90000000000000    1003ccb8     freetypeScaler.obj
 0002:00012cc0       __real@4050000000000000    1003ccc0     freetypeScaler.obj
 0002:00012cc8       __real@40f0000000000000    1003ccc8     freetypeScaler.obj
 0002:00012cd0       __real@42800000            1003ccd0     freetypeScaler.obj
 0002:00012cd8       __real@c0f0000000000000    1003ccd8     freetypeScaler.obj
 0002:00012ce0       __xmm@00010000000000000000366a00010000 1003cce0     freetypeScaler.obj
 0002:00012cf0       __xmm@80000000000000008000000000000000 1003ccf0     freetypeScaler.obj
 0002:00012d00       ??_C@_0BG@NKHBBPH@sun?1font?1TrueTypeFont@ 1003cd00     sunFont.obj
 0002:00012d18       ??_C@_0BL@GAAGJDLL@?$CILjava?1nio?1ByteBuffer?$DLII?$CJI@ 1003cd18     sunFont.obj
 0002:00012d34       ??_C@_09CKAKNPHP@readBlock@ 1003cd34     sunFont.obj
 0002:00012d40       ??_C@_06JMOJDKIE@?$CIII?$CJ?$FLB@ 1003cd40     sunFont.obj
 0002:00012d48       ??_C@_09IDIEPDPI@readBytes@ 1003cd48     sunFont.obj
 0002:00012d54       ??_C@_0BD@OPLCIPMH@sun?1font?1Type1Font@ 1003cd54     sunFont.obj
 0002:00012d68       ??_C@_0BJ@LMHMPPKE@?$CILjava?1nio?1ByteBuffer?$DL?$CJV@ 1003cd68     sunFont.obj
 0002:00012d84       ??_C@_08CJNGBMAG@readFile@ 1003cd84     sunFont.obj
 0002:00012d90       ??_C@_0BM@DGICEJAA@java?1awt?1geom?1Point2D$Float@ 1003cd90     sunFont.obj
 0002:00012dac       ??_C@_05BHHDPELC@?$CIFF?$CJV@ 1003cdac     sunFont.obj
 0002:00012db4       ??_C@_01BIAFAFID@F@        1003cdb4     sunFont.obj
 0002:00012db8       ??_C@_01FJMABOPO@x@        1003cdb8     sunFont.obj
 0002:00012dbc       ??_C@_01EANLCPLP@y@        1003cdbc     sunFont.obj
 0002:00012dc0       ??_C@_0BH@ENELCGL@sun?1font?1StrikeMetrics@ 1003cdc0     sunFont.obj
 0002:00012dd8       ??_C@_0O@LBAHCNJL@?$CIFFFFFFFFFF?$CJV@ 1003cdd8     sunFont.obj
 0002:00012de8       ??_C@_0CA@PDMBNICK@java?1awt?1geom?1Rectangle2D$Float@ 1003cde8     sunFont.obj
 0002:00012e08       ??_C@_07PMCFNNPC@?$CIFFFF?$CJV@ 1003ce08     sunFont.obj
 0002:00012e10       ??_C@_05IGKADHGO@width@    1003ce10     sunFont.obj
 0002:00012e18       ??_C@_06LNLHEAAG@height@   1003ce18     sunFont.obj
 0002:00012e20       ??_C@_0BK@COJNCHEM@java?1awt?1geom?1GeneralPath@ 1003ce20     sunFont.obj
 0002:00012e3c       ??_C@_0L@MDPODKN@?$CII?$FLBI?$FLFI?$CJV@ 1003ce3c     sunFont.obj
 0002:00012e48       ??_C@_0BA@OKNBFGCN@sun?1font?1Font2D@ 1003ce48     sunFont.obj
 0002:00012e58       ??_C@_04DIFHPCLD@?$CII?$CJI@ 1003ce58     sunFont.obj
 0002:00012e60       ??_C@_0M@NMGOHDEJ@charToGlyph@ 1003ce60     sunFont.obj
 0002:00012e6c       ??_C@_0BP@CBNLOFNN@?$CI?$CJLsun?1font?1CharToGlyphMapper?$DL@ 1003ce6c     sunFont.obj
 0002:00012e8c       ??_C@_09DGCMEJKL@getMapper@ 1003ce8c     sunFont.obj
 0002:00012e98       ??_C@_05IPLNOPFN@?$CII?$CJ?$FLB@ 1003ce98     sunFont.obj
 0002:00012ea0       ??_C@_0O@DBNIPDIH@getTableBytes@ 1003cea0     sunFont.obj
 0002:00012eb0       ??_C@_04DGAFFDEF@?$CIC?$CJZ@ 1003ceb0     sunFont.obj
 0002:00012eb8       ??_C@_0L@PGEPPKMA@canDisplay@ 1003ceb8     sunFont.obj
 0002:00012ec4       ??_C@_0BL@GAPGNAAC@sun?1font?1CharToGlyphMapper@ 1003cec4     sunFont.obj
 0002:00012ee0       ??_C@_0BI@GDBHNKM@sun?1font?1PhysicalStrike@ 1003cee0     sunFont.obj
 0002:00012ef8       ??_C@_0CB@IBGFEOCM@?$CII?$CJLjava?1awt?1geom?1Point2D$Float@ 1003cef8     sunFont.obj
 0002:00012f1c       ??_C@_0BA@FMKHNFIF@getGlyphMetrics@ 1003cf1c     sunFont.obj
 0002:00012f2c       ??_C@_0CC@IBLMDHKA@?$CIII?$CJLjava?1awt?1geom?1Point2D$Floa@ 1003cf2c     sunFont.obj
 0002:00012f50       ??_C@_0O@NHLNHECD@getGlyphPoint@ 1003cf50     sunFont.obj
 0002:00012f60       ??_C@_0CB@CONGGNHA@?$CILjava?1awt?1geom?1Point2D$Float?$DL?$CJ@ 1003cf60     sunFont.obj
 0002:00012f84       ??_C@_0M@MJABIGBP@adjustPoint@ 1003cf84     sunFont.obj
 0002:00012f90       ??_C@_01LELAEKIP@J@        1003cf90     sunFont.obj
 0002:00012f94       ??_C@_0P@DPIICNJB@pScalerContext@ 1003cf94     sunFont.obj
 0002:00012fa4       ??_C@_0BD@LPHBDEDB@sun?1font?1GlyphList@ 1003cfa4     sunFont.obj
 0002:00012fb8       ??_C@_03BKCJCHLK@len@      1003cfb8     sunFont.obj
 0002:00012fbc       ??_C@_02GKMBEADD@?$FLJ@    1003cfbc     sunFont.obj
 0002:00012fc0       ??_C@_06IAHKIHIK@images@   1003cfc0     sunFont.obj
 0002:00012fc8       ??_C@_01POHCFINO@Z@        1003cfc8     sunFont.obj
 0002:00012fcc       ??_C@_0N@CLHDJEN@usePositions@ 1003cfcc     sunFont.obj
 0002:00012fdc       ??_C@_09HEJILCIA@positions@ 1003cfdc     sunFont.obj
 0002:00012fe8       ??_C@_0M@IOGNPDID@lcdRGBOrder@ 1003cfe8     sunFont.obj
 0002:00012ff4       ??_C@_0N@OIMCCICM@lcdSubPixPos@ 1003cff4     sunFont.obj
 0002:00013024       ??_7type_info@@6B@         1003d024     MSVCRT:std_type_info_static.obj
 0002:00013048       __pDefaultRawDllMain       1003d048     MSVCRT:dll_dllmain.obj
 0002:00013048       __pRawDllMain              1003d048     MSVCRT:dll_dllmain.obj
 0002:00013050       ??_7exception@std@@6B@     1003d050     MSVCRT:throw_bad_alloc.obj
 0002:00013058       ??_C@_0BC@EOODALEL@Unknown?5exception@ 1003d058     MSVCRT:throw_bad_alloc.obj
 0002:00013070       ??_7bad_alloc@std@@6B@     1003d070     MSVCRT:throw_bad_alloc.obj
 0002:00013078       ??_C@_0P@GHFPNOJB@bad?5allocation@ 1003d078     MSVCRT:throw_bad_alloc.obj
 0002:0001308c       ??_7bad_array_new_length@std@@6B@ 1003d08c     MSVCRT:throw_bad_alloc.obj
 0002:00013094       ??_C@_0BF@KINCDENJ@bad?5array?5new?5length@ 1003d094     MSVCRT:throw_bad_alloc.obj
 0002:000130b8       __load_config_used         1003d0b8     MSVCRT:loadcfg.obj
 0002:00013200       ??_R4ArabicOpenTypeLayoutEngine@@6B@ 1003d200     ArabicLayoutEngine.obj
 0002:00013214       ??_R3ArabicOpenTypeLayoutEngine@@8 1003d214     ArabicLayoutEngine.obj
 0002:00013224       ??_R2ArabicOpenTypeLayoutEngine@@8 1003d224     ArabicLayoutEngine.obj
 0002:00013238       ??_R1A@?0A@EA@ArabicOpenTypeLayoutEngine@@8 1003d238     ArabicLayoutEngine.obj
 0002:00013254       ??_R1A@?0A@EA@OpenTypeLayoutEngine@@8 1003d254     ArabicLayoutEngine.obj
 0002:00013270       ??_R3OpenTypeLayoutEngine@@8 1003d270     ArabicLayoutEngine.obj
 0002:00013280       ??_R2OpenTypeLayoutEngine@@8 1003d280     ArabicLayoutEngine.obj
 0002:00013290       ??_R1A@?0A@EA@LayoutEngine@@8 1003d290     ArabicLayoutEngine.obj
 0002:000132ac       ??_R3LayoutEngine@@8       1003d2ac     ArabicLayoutEngine.obj
 0002:000132bc       ??_R2LayoutEngine@@8       1003d2bc     ArabicLayoutEngine.obj
 0002:000132c8       ??_R13?0A@EA@UObject@@8    1003d2c8     ArabicLayoutEngine.obj
 0002:000132e4       ??_R3UObject@@8            1003d2e4     ArabicLayoutEngine.obj
 0002:000132f4       ??_R2UObject@@8            1003d2f4     ArabicLayoutEngine.obj
 0002:000132fc       ??_R1A@?0A@EA@UObject@@8   1003d2fc     ArabicLayoutEngine.obj
 0002:00013318       ??_R4UnicodeArabicOpenTypeLayoutEngine@@6B@ 1003d318     ArabicLayoutEngine.obj
 0002:0001332c       ??_R3UnicodeArabicOpenTypeLayoutEngine@@8 1003d32c     ArabicLayoutEngine.obj
 0002:0001333c       ??_R2UnicodeArabicOpenTypeLayoutEngine@@8 1003d33c     ArabicLayoutEngine.obj
 0002:00013354       ??_R1A@?0A@EA@UnicodeArabicOpenTypeLayoutEngine@@8 1003d354     ArabicLayoutEngine.obj
 0002:00013370       ??_R4ContextualGlyphInsertionProcessor2@@6B@ 1003d370     ContextualGlyphInsertionProc2.obj
 0002:00013384       ??_R3ContextualGlyphInsertionProcessor2@@8 1003d384     ContextualGlyphInsertionProc2.obj
 0002:00013394       ??_R2ContextualGlyphInsertionProcessor2@@8 1003d394     ContextualGlyphInsertionProc2.obj
 0002:000133a8       ??_R1A@?0A@EA@ContextualGlyphInsertionProcessor2@@8 1003d3a8     ContextualGlyphInsertionProc2.obj
 0002:000133c4       ??_R1A@?0A@EA@StateTableProcessor2@@8 1003d3c4     ContextualGlyphInsertionProc2.obj
 0002:000133e0       ??_R3StateTableProcessor2@@8 1003d3e0     ContextualGlyphInsertionProc2.obj
 0002:000133f0       ??_R2StateTableProcessor2@@8 1003d3f0     ContextualGlyphInsertionProc2.obj
 0002:00013400       ??_R1A@?0A@EA@SubtableProcessor2@@8 1003d400     ContextualGlyphInsertionProc2.obj
 0002:0001341c       ??_R3SubtableProcessor2@@8 1003d41c     ContextualGlyphInsertionProc2.obj
 0002:0001342c       ??_R2SubtableProcessor2@@8 1003d42c     ContextualGlyphInsertionProc2.obj
 0002:00013438       ??_R13?0A@EA@UMemory@@8    1003d438     ContextualGlyphInsertionProc2.obj
 0002:00013454       ??_R3UMemory@@8            1003d454     ContextualGlyphInsertionProc2.obj
 0002:00013464       ??_R2UMemory@@8            1003d464     ContextualGlyphInsertionProc2.obj
 0002:0001346c       ??_R1A@?0A@EA@UMemory@@8   1003d46c     ContextualGlyphInsertionProc2.obj
 0002:00013488       ??_R4ContextualGlyphSubstitutionProcessor@@6B@ 1003d488     ContextualGlyphSubstProc.obj
 0002:0001349c       ??_R3ContextualGlyphSubstitutionProcessor@@8 1003d49c     ContextualGlyphSubstProc.obj
 0002:000134ac       ??_R2ContextualGlyphSubstitutionProcessor@@8 1003d4ac     ContextualGlyphSubstProc.obj
 0002:000134c0       ??_R1A@?0A@EA@ContextualGlyphSubstitutionProcessor@@8 1003d4c0     ContextualGlyphSubstProc.obj
 0002:000134dc       ??_R1A@?0A@EA@StateTableProcessor@@8 1003d4dc     ContextualGlyphSubstProc.obj
 0002:000134f8       ??_R3StateTableProcessor@@8 1003d4f8     ContextualGlyphSubstProc.obj
 0002:00013508       ??_R2StateTableProcessor@@8 1003d508     ContextualGlyphSubstProc.obj
 0002:00013518       ??_R1A@?0A@EA@SubtableProcessor@@8 1003d518     ContextualGlyphSubstProc.obj
 0002:00013534       ??_R3SubtableProcessor@@8  1003d534     ContextualGlyphSubstProc.obj
 0002:00013544       ??_R2SubtableProcessor@@8  1003d544     ContextualGlyphSubstProc.obj
 0002:00013550       ??_R4ContextualGlyphSubstitutionProcessor2@@6B@ 1003d550     ContextualGlyphSubstProc2.obj
 0002:00013564       ??_R3ContextualGlyphSubstitutionProcessor2@@8 1003d564     ContextualGlyphSubstProc2.obj
 0002:00013574       ??_R2ContextualGlyphSubstitutionProcessor2@@8 1003d574     ContextualGlyphSubstProc2.obj
 0002:00013588       ??_R1A@?0A@EA@ContextualGlyphSubstitutionProcessor2@@8 1003d588     ContextualGlyphSubstProc2.obj
 0002:000135a4       ??_R4LEFontInstance@@6B@   1003d5a4     FontInstanceAdapter.obj
 0002:000135b8       ??_R3LEFontInstance@@8     1003d5b8     FontInstanceAdapter.obj
 0002:000135c8       ??_R2LEFontInstance@@8     1003d5c8     FontInstanceAdapter.obj
 0002:000135d4       ??_R1A@?0A@EA@LEFontInstance@@8 1003d5d4     FontInstanceAdapter.obj
 0002:000135f0       ??_R4FontInstanceAdapter@@6B@ 1003d5f0     FontInstanceAdapter.obj
 0002:00013604       ??_R3FontInstanceAdapter@@8 1003d604     FontInstanceAdapter.obj
 0002:00013614       ??_R2FontInstanceAdapter@@8 1003d614     FontInstanceAdapter.obj
 0002:00013624       ??_R1A@?0A@EA@FontInstanceAdapter@@8 1003d624     FontInstanceAdapter.obj
 0002:00013640       ??_R4LEGlyphFilter@@6B@    1003d640     GDEFMarkFilter.obj
 0002:00013654       ??_R3LEGlyphFilter@@8      1003d654     GDEFMarkFilter.obj
 0002:00013664       ??_R2LEGlyphFilter@@8      1003d664     GDEFMarkFilter.obj
 0002:0001366c       ??_R1A@?0A@EA@LEGlyphFilter@@8 1003d66c     GDEFMarkFilter.obj
 0002:00013688       ??_R4GDEFMarkFilter@@6B@   1003d688     GDEFMarkFilter.obj
 0002:0001369c       ??_R3GDEFMarkFilter@@8     1003d69c     GDEFMarkFilter.obj
 0002:000136ac       ??_R2GDEFMarkFilter@@8     1003d6ac     GDEFMarkFilter.obj
 0002:000136bc       ??_R1A@?0A@EA@GDEFMarkFilter@@8 1003d6bc     GDEFMarkFilter.obj
 0002:000136d8       ??_R4GXLayoutEngine@@6B@   1003d6d8     GXLayoutEngine.obj
 0002:000136ec       ??_R3GXLayoutEngine@@8     1003d6ec     GXLayoutEngine.obj
 0002:000136fc       ??_R2GXLayoutEngine@@8     1003d6fc     GXLayoutEngine.obj
 0002:0001370c       ??_R1A@?0A@EA@GXLayoutEngine@@8 1003d70c     GXLayoutEngine.obj
 0002:00013728       ??_R4GXLayoutEngine2@@6B@  1003d728     GXLayoutEngine2.obj
 0002:0001373c       ??_R3GXLayoutEngine2@@8    1003d73c     GXLayoutEngine2.obj
 0002:0001374c       ??_R2GXLayoutEngine2@@8    1003d74c     GXLayoutEngine2.obj
 0002:0001375c       ??_R1A@?0A@EA@GXLayoutEngine2@@8 1003d75c     GXLayoutEngine2.obj
 0002:00013778       ??_R4GlyphIterator@@6B@    1003d778     GlyphIterator.obj
 0002:0001378c       ??_R3GlyphIterator@@8      1003d78c     GlyphIterator.obj
 0002:0001379c       ??_R2GlyphIterator@@8      1003d79c     GlyphIterator.obj
 0002:000137a8       ??_R1A@?0A@EA@GlyphIterator@@8 1003d7a8     GlyphIterator.obj
 0002:000137c4       ??_R4GlyphPositioningLookupProcessor@@6B@ 1003d7c4     GlyphPosnLookupProc.obj
 0002:000137d8       ??_R3GlyphPositioningLookupProcessor@@8 1003d7d8     GlyphPosnLookupProc.obj
 0002:000137e8       ??_R2GlyphPositioningLookupProcessor@@8 1003d7e8     GlyphPosnLookupProc.obj
 0002:000137f8       ??_R1A@?0A@EA@GlyphPositioningLookupProcessor@@8 1003d7f8     GlyphPosnLookupProc.obj
 0002:00013814       ??_R1A@?0A@EA@LookupProcessor@@8 1003d814     GlyphPosnLookupProc.obj
 0002:00013830       ??_R3LookupProcessor@@8    1003d830     GlyphPosnLookupProc.obj
 0002:00013840       ??_R2LookupProcessor@@8    1003d840     GlyphPosnLookupProc.obj
 0002:0001384c       ??_R4GlyphSubstitutionLookupProcessor@@6B@ 1003d84c     GlyphSubstLookupProc.obj
 0002:00013860       ??_R3GlyphSubstitutionLookupProcessor@@8 1003d860     GlyphSubstLookupProc.obj
 0002:00013870       ??_R2GlyphSubstitutionLookupProcessor@@8 1003d870     GlyphSubstLookupProc.obj
 0002:00013880       ??_R1A@?0A@EA@GlyphSubstitutionLookupProcessor@@8 1003d880     GlyphSubstLookupProc.obj
 0002:0001389c       ??_R4HanOpenTypeLayoutEngine@@6B@ 1003d89c     HanLayoutEngine.obj
 0002:000138b0       ??_R3HanOpenTypeLayoutEngine@@8 1003d8b0     HanLayoutEngine.obj
 0002:000138c0       ??_R2HanOpenTypeLayoutEngine@@8 1003d8c0     HanLayoutEngine.obj
 0002:000138d4       ??_R1A@?0A@EA@HanOpenTypeLayoutEngine@@8 1003d8d4     HanLayoutEngine.obj
 0002:000138f0       ??_R4HangulOpenTypeLayoutEngine@@6B@ 1003d8f0     HangulLayoutEngine.obj
 0002:00013904       ??_R3HangulOpenTypeLayoutEngine@@8 1003d904     HangulLayoutEngine.obj
 0002:00013914       ??_R2HangulOpenTypeLayoutEngine@@8 1003d914     HangulLayoutEngine.obj
 0002:00013928       ??_R1A@?0A@EA@HangulOpenTypeLayoutEngine@@8 1003d928     HangulLayoutEngine.obj
 0002:00013944       ??_R4IndicOpenTypeLayoutEngine@@6B@ 1003d944     IndicLayoutEngine.obj
 0002:00013958       ??_R3IndicOpenTypeLayoutEngine@@8 1003d958     IndicLayoutEngine.obj
 0002:00013968       ??_R2IndicOpenTypeLayoutEngine@@8 1003d968     IndicLayoutEngine.obj
 0002:0001397c       ??_R1A@?0A@EA@IndicOpenTypeLayoutEngine@@8 1003d97c     IndicLayoutEngine.obj
 0002:00013998       ??_R4IndicRearrangementProcessor@@6B@ 1003d998     IndicRearrangementProcessor.obj
 0002:000139ac       ??_R3IndicRearrangementProcessor@@8 1003d9ac     IndicRearrangementProcessor.obj
 0002:000139bc       ??_R2IndicRearrangementProcessor@@8 1003d9bc     IndicRearrangementProcessor.obj
 0002:000139d0       ??_R1A@?0A@EA@IndicRearrangementProcessor@@8 1003d9d0     IndicRearrangementProcessor.obj
 0002:000139ec       ??_R4IndicRearrangementProcessor2@@6B@ 1003d9ec     IndicRearrangementProcessor2.obj
 0002:00013a00       ??_R3IndicRearrangementProcessor2@@8 1003da00     IndicRearrangementProcessor2.obj
 0002:00013a10       ??_R2IndicRearrangementProcessor2@@8 1003da10     IndicRearrangementProcessor2.obj
 0002:00013a24       ??_R1A@?0A@EA@IndicRearrangementProcessor2@@8 1003da24     IndicRearrangementProcessor2.obj
 0002:00013a40       ??_R4KhmerOpenTypeLayoutEngine@@6B@ 1003da40     KhmerLayoutEngine.obj
 0002:00013a54       ??_R3KhmerOpenTypeLayoutEngine@@8 1003da54     KhmerLayoutEngine.obj
 0002:00013a64       ??_R2KhmerOpenTypeLayoutEngine@@8 1003da64     KhmerLayoutEngine.obj
 0002:00013a78       ??_R1A@?0A@EA@KhmerOpenTypeLayoutEngine@@8 1003da78     KhmerLayoutEngine.obj
 0002:00013a94       ??_R4LECharMapper@@6B@     1003da94     LEFontInstance.obj
 0002:00013aa8       ??_R3LECharMapper@@8       1003daa8     LEFontInstance.obj
 0002:00013ab8       ??_R2LECharMapper@@8       1003dab8     LEFontInstance.obj
 0002:00013ac0       ??_R1A@?0A@EA@LECharMapper@@8 1003dac0     LEFontInstance.obj
 0002:00013adc       ??_R4LEInsertionCallback@@6B@ 1003dadc     LEGlyphStorage.obj
 0002:00013af0       ??_R3LEInsertionCallback@@8 1003daf0     LEGlyphStorage.obj
 0002:00013b00       ??_R2LEInsertionCallback@@8 1003db00     LEGlyphStorage.obj
 0002:00013b08       ??_R1A@?0A@EA@LEInsertionCallback@@8 1003db08     LEGlyphStorage.obj
 0002:00013b24       ??_R4LEGlyphStorage@@6B@   1003db24     LEGlyphStorage.obj
 0002:00013b38       ??_R3LEGlyphStorage@@8     1003db38     LEGlyphStorage.obj
 0002:00013b48       ??_R2LEGlyphStorage@@8     1003db48     LEGlyphStorage.obj
 0002:00013b58       ??_R1A@?0A@EA@LEGlyphStorage@@8 1003db58     LEGlyphStorage.obj
 0002:00013b74       ??_R1A@?0A@EN@LEInsertionCallback@@8 1003db74     LEGlyphStorage.obj
 0002:00013b90       ??_R4LEInsertionList@@6B@  1003db90     LEInsertionList.obj
 0002:00013ba4       ??_R3LEInsertionList@@8    1003dba4     LEInsertionList.obj
 0002:00013bb4       ??_R2LEInsertionList@@8    1003dbb4     LEInsertionList.obj
 0002:00013bc0       ??_R1A@?0A@EA@LEInsertionList@@8 1003dbc0     LEInsertionList.obj
 0002:00013bdc       ??_R4LayoutEngine@@6B@     1003dbdc     LayoutEngine.obj
 0002:00013bf0       ??_R4CharSubstitutionFilter@@6B@ 1003dbf0     LayoutEngine.obj
 0002:00013c04       ??_R3CharSubstitutionFilter@@8 1003dc04     LayoutEngine.obj
 0002:00013c14       ??_R2CharSubstitutionFilter@@8 1003dc14     LayoutEngine.obj
 0002:00013c24       ??_R1A@?0A@EA@CharSubstitutionFilter@@8 1003dc24     LayoutEngine.obj
 0002:00013c40       ??_R4DefaultCharMapper@@6B@ 1003dc40     LayoutEngine.obj
 0002:00013c54       ??_R3DefaultCharMapper@@8  1003dc54     LayoutEngine.obj
 0002:00013c64       ??_R2DefaultCharMapper@@8  1003dc64     LayoutEngine.obj
 0002:00013c74       ??_R1A@?0A@EA@DefaultCharMapper@@8 1003dc74     LayoutEngine.obj
 0002:00013c90       ??_R4CanonMarkFilter@@6B@  1003dc90     LayoutEngine.obj
 0002:00013ca4       ??_R3CanonMarkFilter@@8    1003dca4     LayoutEngine.obj
 0002:00013cb4       ??_R2CanonMarkFilter@@8    1003dcb4     LayoutEngine.obj
 0002:00013cc4       ??_R1A@?0A@EA@CanonMarkFilter@@8 1003dcc4     LayoutEngine.obj
 0002:00013ce0       ??_R4LigatureSubstitutionProcessor@@6B@ 1003dce0     LigatureSubstProc.obj
 0002:00013cf4       ??_R3LigatureSubstitutionProcessor@@8 1003dcf4     LigatureSubstProc.obj
 0002:00013d04       ??_R2LigatureSubstitutionProcessor@@8 1003dd04     LigatureSubstProc.obj
 0002:00013d18       ??_R1A@?0A@EA@LigatureSubstitutionProcessor@@8 1003dd18     LigatureSubstProc.obj
 0002:00013d34       ??_R4LigatureSubstitutionProcessor2@@6B@ 1003dd34     LigatureSubstProc2.obj
 0002:00013d48       ??_R3LigatureSubstitutionProcessor2@@8 1003dd48     LigatureSubstProc2.obj
 0002:00013d58       ??_R2LigatureSubstitutionProcessor2@@8 1003dd58     LigatureSubstProc2.obj
 0002:00013d6c       ??_R1A@?0A@EA@LigatureSubstitutionProcessor2@@8 1003dd6c     LigatureSubstProc2.obj
 0002:00013d88       ??_R4LookupProcessor@@6B@  1003dd88     LookupProcessor.obj
 0002:00013d9c       ??_R4NonContextualGlyphSubstitutionProcessor@@6B@ 1003dd9c     NonContextualGlyphSubstProc.obj
 0002:00013db0       ??_R3NonContextualGlyphSubstitutionProcessor@@8 1003ddb0     NonContextualGlyphSubstProc.obj
 0002:00013dc0       ??_R2NonContextualGlyphSubstitutionProcessor@@8 1003ddc0     NonContextualGlyphSubstProc.obj
 0002:00013dd0       ??_R1A@?0A@EA@NonContextualGlyphSubstitutionProcessor@@8 1003ddd0     NonContextualGlyphSubstProc.obj
 0002:00013dec       ??_R4NonContextualGlyphSubstitutionProcessor2@@6B@ 1003ddec     NonContextualGlyphSubstProc2.obj
 0002:00013e00       ??_R3NonContextualGlyphSubstitutionProcessor2@@8 1003de00     NonContextualGlyphSubstProc2.obj
 0002:00013e10       ??_R2NonContextualGlyphSubstitutionProcessor2@@8 1003de10     NonContextualGlyphSubstProc2.obj
 0002:00013e20       ??_R1A@?0A@EA@NonContextualGlyphSubstitutionProcessor2@@8 1003de20     NonContextualGlyphSubstProc2.obj
 0002:00013e3c       ??_R4OpenTypeLayoutEngine@@6B@ 1003de3c     OpenTypeLayoutEngine.obj
 0002:00013e50       ??_R4SegmentArrayProcessor@@6B@ 1003de50     SegmentArrayProcessor.obj
 0002:00013e64       ??_R3SegmentArrayProcessor@@8 1003de64     SegmentArrayProcessor.obj
 0002:00013e74       ??_R2SegmentArrayProcessor@@8 1003de74     SegmentArrayProcessor.obj
 0002:00013e88       ??_R1A@?0A@EA@SegmentArrayProcessor@@8 1003de88     SegmentArrayProcessor.obj
 0002:00013ea4       ??_R4SegmentArrayProcessor2@@6B@ 1003dea4     SegmentArrayProcessor2.obj
 0002:00013eb8       ??_R3SegmentArrayProcessor2@@8 1003deb8     SegmentArrayProcessor2.obj
 0002:00013ec8       ??_R2SegmentArrayProcessor2@@8 1003dec8     SegmentArrayProcessor2.obj
 0002:00013edc       ??_R1A@?0A@EA@SegmentArrayProcessor2@@8 1003dedc     SegmentArrayProcessor2.obj
 0002:00013ef8       ??_R4SegmentSingleProcessor@@6B@ 1003def8     SegmentSingleProcessor.obj
 0002:00013f0c       ??_R3SegmentSingleProcessor@@8 1003df0c     SegmentSingleProcessor.obj
 0002:00013f1c       ??_R2SegmentSingleProcessor@@8 1003df1c     SegmentSingleProcessor.obj
 0002:00013f30       ??_R1A@?0A@EA@SegmentSingleProcessor@@8 1003df30     SegmentSingleProcessor.obj
 0002:00013f4c       ??_R4SegmentSingleProcessor2@@6B@ 1003df4c     SegmentSingleProcessor2.obj
 0002:00013f60       ??_R3SegmentSingleProcessor2@@8 1003df60     SegmentSingleProcessor2.obj
 0002:00013f70       ??_R2SegmentSingleProcessor2@@8 1003df70     SegmentSingleProcessor2.obj
 0002:00013f84       ??_R1A@?0A@EA@SegmentSingleProcessor2@@8 1003df84     SegmentSingleProcessor2.obj
 0002:00013fa0       ??_R4SimpleArrayProcessor@@6B@ 1003dfa0     SimpleArrayProcessor.obj
 0002:00013fb4       ??_R3SimpleArrayProcessor@@8 1003dfb4     SimpleArrayProcessor.obj
 0002:00013fc4       ??_R2SimpleArrayProcessor@@8 1003dfc4     SimpleArrayProcessor.obj
 0002:00013fd8       ??_R1A@?0A@EA@SimpleArrayProcessor@@8 1003dfd8     SimpleArrayProcessor.obj
 0002:00013ff4       ??_R4SimpleArrayProcessor2@@6B@ 1003dff4     SimpleArrayProcessor2.obj
 0002:00014008       ??_R3SimpleArrayProcessor2@@8 1003e008     SimpleArrayProcessor2.obj
 0002:00014018       ??_R2SimpleArrayProcessor2@@8 1003e018     SimpleArrayProcessor2.obj
 0002:0001402c       ??_R1A@?0A@EA@SimpleArrayProcessor2@@8 1003e02c     SimpleArrayProcessor2.obj
 0002:00014048       ??_R4SingleTableProcessor@@6B@ 1003e048     SingleTableProcessor.obj
 0002:0001405c       ??_R3SingleTableProcessor@@8 1003e05c     SingleTableProcessor.obj
 0002:0001406c       ??_R2SingleTableProcessor@@8 1003e06c     SingleTableProcessor.obj
 0002:00014080       ??_R1A@?0A@EA@SingleTableProcessor@@8 1003e080     SingleTableProcessor.obj
 0002:0001409c       ??_R4SingleTableProcessor2@@6B@ 1003e09c     SingleTableProcessor2.obj
 0002:000140b0       ??_R3SingleTableProcessor2@@8 1003e0b0     SingleTableProcessor2.obj
 0002:000140c0       ??_R2SingleTableProcessor2@@8 1003e0c0     SingleTableProcessor2.obj
 0002:000140d4       ??_R1A@?0A@EA@SingleTableProcessor2@@8 1003e0d4     SingleTableProcessor2.obj
 0002:000140f0       ??_R4StateTableProcessor@@6B@ 1003e0f0     StateTableProcessor.obj
 0002:00014104       ??_R4StateTableProcessor2@@6B@ 1003e104     StateTableProcessor2.obj
 0002:00014118       ??_R4SubtableProcessor@@6B@ 1003e118     SubtableProcessor.obj
 0002:0001412c       ??_R4SubtableProcessor2@@6B@ 1003e12c     SubtableProcessor2.obj
 0002:00014140       ??_R4ThaiLayoutEngine@@6B@ 1003e140     ThaiLayoutEngine.obj
 0002:00014154       ??_R3ThaiLayoutEngine@@8   1003e154     ThaiLayoutEngine.obj
 0002:00014164       ??_R2ThaiLayoutEngine@@8   1003e164     ThaiLayoutEngine.obj
 0002:00014174       ??_R1A@?0A@EA@ThaiLayoutEngine@@8 1003e174     ThaiLayoutEngine.obj
 0002:00014190       ??_R4TibetanOpenTypeLayoutEngine@@6B@ 1003e190     TibetanLayoutEngine.obj
 0002:000141a4       ??_R3TibetanOpenTypeLayoutEngine@@8 1003e1a4     TibetanLayoutEngine.obj
 0002:000141b4       ??_R2TibetanOpenTypeLayoutEngine@@8 1003e1b4     TibetanLayoutEngine.obj
 0002:000141c8       ??_R1A@?0A@EA@TibetanOpenTypeLayoutEngine@@8 1003e1c8     TibetanLayoutEngine.obj
 0002:000141e4       ??_R4TrimmedArrayProcessor@@6B@ 1003e1e4     TrimmedArrayProcessor.obj
 0002:000141f8       ??_R3TrimmedArrayProcessor@@8 1003e1f8     TrimmedArrayProcessor.obj
 0002:00014208       ??_R2TrimmedArrayProcessor@@8 1003e208     TrimmedArrayProcessor.obj
 0002:0001421c       ??_R1A@?0A@EA@TrimmedArrayProcessor@@8 1003e21c     TrimmedArrayProcessor.obj
 0002:00014238       ??_R4TrimmedArrayProcessor2@@6B@ 1003e238     TrimmedArrayProcessor2.obj
 0002:0001424c       ??_R3TrimmedArrayProcessor2@@8 1003e24c     TrimmedArrayProcessor2.obj
 0002:0001425c       ??_R2TrimmedArrayProcessor2@@8 1003e25c     TrimmedArrayProcessor2.obj
 0002:00014270       ??_R1A@?0A@EA@TrimmedArrayProcessor2@@8 1003e270     TrimmedArrayProcessor2.obj
 0002:0001428c       ??_R4type_info@@6B@        1003e28c     MSVCRT:std_type_info_static.obj
 0002:000142a0       ??_R3type_info@@8          1003e2a0     MSVCRT:std_type_info_static.obj
 0002:000142b0       ??_R2type_info@@8          1003e2b0     MSVCRT:std_type_info_static.obj
 0002:000142b8       ??_R1A@?0A@EA@type_info@@8 1003e2b8     MSVCRT:std_type_info_static.obj
 0002:000142d4       ??_R4exception@std@@6B@    1003e2d4     MSVCRT:throw_bad_alloc.obj
 0002:000142e8       ??_R3exception@std@@8      1003e2e8     MSVCRT:throw_bad_alloc.obj
 0002:000142f8       ??_R2exception@std@@8      1003e2f8     MSVCRT:throw_bad_alloc.obj
 0002:00014300       ??_R1A@?0A@EA@exception@std@@8 1003e300     MSVCRT:throw_bad_alloc.obj
 0002:0001431c       ??_R4bad_alloc@std@@6B@    1003e31c     MSVCRT:throw_bad_alloc.obj
 0002:00014330       ??_R3bad_alloc@std@@8      1003e330     MSVCRT:throw_bad_alloc.obj
 0002:00014340       ??_R2bad_alloc@std@@8      1003e340     MSVCRT:throw_bad_alloc.obj
 0002:0001434c       ??_R1A@?0A@EA@bad_alloc@std@@8 1003e34c     MSVCRT:throw_bad_alloc.obj
 0002:00014368       ??_R4bad_array_new_length@std@@6B@ 1003e368     MSVCRT:throw_bad_alloc.obj
 0002:0001437c       ??_R3bad_array_new_length@std@@8 1003e37c     MSVCRT:throw_bad_alloc.obj
 0002:0001438c       ??_R2bad_array_new_length@std@@8 1003e38c     MSVCRT:throw_bad_alloc.obj
 0002:0001439c       ??_R1A@?0A@EA@bad_array_new_length@std@@8 1003e39c     MSVCRT:throw_bad_alloc.obj
 0002:000143b8       ___safe_se_handler_table   1003e3b8     <linker-defined>
 0002:000143bc       ___volatile_metadata       1003e3bc     <linker-defined>
 0002:0001476c       ___rtc_iaa                 1003e76c     MSVCRT:initsect.obj
 0002:00014770       ___rtc_izz                 1003e770     MSVCRT:initsect.obj
 0002:00014774       ___rtc_taa                 1003e774     MSVCRT:initsect.obj
 0002:00014778       ___rtc_tzz                 1003e778     MSVCRT:initsect.obj
 0002:000147e4       __TI2?AVbad_alloc@std@@    1003e7e4     MSVCRT:throw_bad_alloc.obj
 0002:000147f4       __CTA2?AVbad_alloc@std@@   1003e7f4     MSVCRT:throw_bad_alloc.obj
 0002:00014800       __CT??_R0?AVbad_alloc@std@@@8??0bad_alloc@std@@QAE@ABV01@@Z12 1003e800     MSVCRT:throw_bad_alloc.obj
 0002:0001481c       __CT??_R0?AVexception@std@@@8??0exception@std@@QAE@ABV01@@Z12 1003e81c     MSVCRT:throw_bad_alloc.obj
 0002:00014838       __TI3?AVbad_array_new_length@std@@ 1003e838     MSVCRT:throw_bad_alloc.obj
 0002:00014848       __CTA3?AVbad_array_new_length@std@@ 1003e848     MSVCRT:throw_bad_alloc.obj
 0002:00014858       __CT??_R0?AVbad_array_new_length@std@@@8??0bad_array_new_length@std@@QAE@ABV01@@Z12 1003e858     MSVCRT:throw_bad_alloc.obj
 0002:000151d0       __IMPORT_DESCRIPTOR_freetype 1003f1d0     freetype:freetype.dll
 0002:000151e4       __IMPORT_DESCRIPTOR_java   1003f1e4     java:java.dll
 0002:000151f8       __IMPORT_DESCRIPTOR_ADVAPI32 1003f1f8     advapi32:ADVAPI32.dll
 0002:0001520c       __IMPORT_DESCRIPTOR_USER32 1003f20c     user32:USER32.dll
 0002:00015220       __IMPORT_DESCRIPTOR_GDI32  1003f220     gdi32:GDI32.dll
 0002:00015234       __IMPORT_DESCRIPTOR_awt    1003f234     awt:awt.dll
 0002:00015248       __IMPORT_DESCRIPTOR_KERNEL32 1003f248     kernel32:KERNEL32.dll
 0002:0001525c       __IMPORT_DESCRIPTOR_VCRUNTIME140 1003f25c     vcruntime:VCRUNTIME140.dll
 0002:00015270       __IMPORT_DESCRIPTOR_api-ms-win-crt-heap-l1-1-0 1003f270     ucrt:api-ms-win-crt-heap-l1-1-0.dll
 0002:00015284       __IMPORT_DESCRIPTOR_api-ms-win-crt-math-l1-1-0 1003f284     ucrt:api-ms-win-crt-math-l1-1-0.dll
 0002:00015298       __IMPORT_DESCRIPTOR_api-ms-win-crt-environment-l1-1-0 1003f298     ucrt:api-ms-win-crt-environment-l1-1-0.dll
 0002:000152ac       __IMPORT_DESCRIPTOR_api-ms-win-crt-runtime-l1-1-0 1003f2ac     ucrt:api-ms-win-crt-runtime-l1-1-0.dll
 0002:000152c0       __IMPORT_DESCRIPTOR_api-ms-win-crt-string-l1-1-0 1003f2c0     ucrt:api-ms-win-crt-string-l1-1-0.dll
 0002:000152d4       __NULL_IMPORT_DESCRIPTOR   1003f2d4     freetype:freetype.dll
 0003:00000000       _defaultGammaLUT           10040000     DrawGlyphList.obj
 0003:00000100       _defaultInvGammaLUT        10040100     DrawGlyphList.obj
 0003:00000210       __fltused                  10040210     MSVCRT:fltused.obj
 0003:00000214       ___security_cookie_complement 10040214     MSVCRT:gs_cookie.obj
 0003:00000218       ___security_cookie         10040218     MSVCRT:gs_cookie.obj
 0003:00000220       ___isa_enabled             10040220     MSVCRT:cpu_disp.obj
 0003:00000230       ___scrt_native_dllmain_reason 10040230     MSVCRT:utility.obj
 0003:00000240       ___scrt_ucrt_dll_is_in_use 10040240     MSVCRT:ucrt_stubs.obj
 0003:00000244       ??_R0?AVbad_alloc@std@@@8  10040244     MSVCRT:throw_bad_alloc.obj
 0003:00000260       ??_R0?AVexception@std@@@8  10040260     MSVCRT:throw_bad_alloc.obj
 0003:0000027c       ??_R0?AVbad_array_new_length@std@@@8 1004027c     MSVCRT:throw_bad_alloc.obj
 0003:000002a4       ??_R0?AVArabicOpenTypeLayoutEngine@@@8 100402a4     ArabicLayoutEngine.obj
 0003:000002d0       ??_R0?AVOpenTypeLayoutEngine@@@8 100402d0     ArabicLayoutEngine.obj
 0003:000002f4       ??_R0?AVLayoutEngine@@@8   100402f4     ArabicLayoutEngine.obj
 0003:00000310       ??_R0?AUUObject@@@8        10040310     ArabicLayoutEngine.obj
 0003:00000328       ??_R0?AVUnicodeArabicOpenTypeLayoutEngine@@@8 10040328     ArabicLayoutEngine.obj
 0003:00000358       ??_R0?AVContextualGlyphInsertionProcessor2@@@8 10040358     ContextualGlyphInsertionProc2.obj
 0003:0000038c       ??_R0?AVStateTableProcessor2@@@8 1004038c     ContextualGlyphInsertionProc2.obj
 0003:000003b0       ??_R0?AVSubtableProcessor2@@@8 100403b0     ContextualGlyphInsertionProc2.obj
 0003:000003d4       ??_R0?AUUMemory@@@8        100403d4     ContextualGlyphInsertionProc2.obj
 0003:000003ec       ??_R0?AVContextualGlyphSubstitutionProcessor@@@8 100403ec     ContextualGlyphSubstProc.obj
 0003:00000420       ??_R0?AVStateTableProcessor@@@8 10040420     ContextualGlyphSubstProc.obj
 0003:00000444       ??_R0?AVSubtableProcessor@@@8 10040444     ContextualGlyphSubstProc.obj
 0003:00000464       ??_R0?AVContextualGlyphSubstitutionProcessor2@@@8 10040464     ContextualGlyphSubstProc2.obj
 0003:00000498       ??_R0?AVLEFontInstance@@@8 10040498     FontInstanceAdapter.obj
 0003:000004b8       ??_R0?AVFontInstanceAdapter@@@8 100404b8     FontInstanceAdapter.obj
 0003:000004dc       ??_R0?AVLEGlyphFilter@@@8  100404dc     GDEFMarkFilter.obj
 0003:000004f8       ??_R0?AVGDEFMarkFilter@@@8 100404f8     GDEFMarkFilter.obj
 0003:00000518       ??_R0?AVGXLayoutEngine@@@8 10040518     GXLayoutEngine.obj
 0003:00000538       ??_R0?AVGXLayoutEngine2@@@8 10040538     GXLayoutEngine2.obj
 0003:00000558       ??_R0?AVGlyphIterator@@@8  10040558     GlyphIterator.obj
 0003:00000574       ??_R0?AVGlyphPositioningLookupProcessor@@@8 10040574     GlyphPosnLookupProc.obj
 0003:000005a4       ??_R0?AVLookupProcessor@@@8 100405a4     GlyphPosnLookupProc.obj
 0003:000005c4       ??_R0?AVGlyphSubstitutionLookupProcessor@@@8 100405c4     GlyphSubstLookupProc.obj
 0003:000005f4       ??_R0?AVHanOpenTypeLayoutEngine@@@8 100405f4     HanLayoutEngine.obj
 0003:0000061c       ??_R0?AVHangulOpenTypeLayoutEngine@@@8 1004061c     HangulLayoutEngine.obj
 0003:00000648       ??_R0?AVIndicOpenTypeLayoutEngine@@@8 10040648     IndicLayoutEngine.obj
 0003:00000670       ??_R0?AVIndicRearrangementProcessor@@@8 10040670     IndicRearrangementProcessor.obj
 0003:0000069c       ??_R0?AVIndicRearrangementProcessor2@@@8 1004069c     IndicRearrangementProcessor2.obj
 0003:000006c8       ??_R0?AVKhmerOpenTypeLayoutEngine@@@8 100406c8     KhmerLayoutEngine.obj
 0003:000006f0       ??_R0?AVLECharMapper@@@8   100406f0     LEFontInstance.obj
 0003:0000070c       ??_R0?AVLEInsertionCallback@@@8 1004070c     LEGlyphStorage.obj
 0003:00000730       ??_R0?AVLEGlyphStorage@@@8 10040730     LEGlyphStorage.obj
 0003:00000750       ??_R0?AVLEInsertionList@@@8 10040750     LEInsertionList.obj
 0003:00000770       ??_R0?AVCharSubstitutionFilter@@@8 10040770     LayoutEngine.obj
 0003:00000798       ??_R0?AVDefaultCharMapper@@@8 10040798     LayoutEngine.obj
 0003:000007b8       ??_R0?AVCanonMarkFilter@@@8 100407b8     LayoutEngine.obj
 0003:000007d8       ??_R0?AVLigatureSubstitutionProcessor@@@8 100407d8     LigatureSubstProc.obj
 0003:00000804       ??_R0?AVLigatureSubstitutionProcessor2@@@8 10040804     LigatureSubstProc2.obj
 0003:00000834       ??_R0?AVNonContextualGlyphSubstitutionProcessor@@@8 10040834     NonContextualGlyphSubstProc.obj
 0003:0000086c       ??_R0?AVNonContextualGlyphSubstitutionProcessor2@@@8 1004086c     NonContextualGlyphSubstProc2.obj
 0003:000008a4       ??_R0?AVSegmentArrayProcessor@@@8 100408a4     SegmentArrayProcessor.obj
 0003:000008c8       ??_R0?AVSegmentArrayProcessor2@@@8 100408c8     SegmentArrayProcessor2.obj
 0003:000008f0       ??_R0?AVSegmentSingleProcessor@@@8 100408f0     SegmentSingleProcessor.obj
 0003:00000918       ??_R0?AVSegmentSingleProcessor2@@@8 10040918     SegmentSingleProcessor2.obj
 0003:00000940       ??_R0?AVSimpleArrayProcessor@@@8 10040940     SimpleArrayProcessor.obj
 0003:00000964       ??_R0?AVSimpleArrayProcessor2@@@8 10040964     SimpleArrayProcessor2.obj
 0003:00000988       ??_R0?AVSingleTableProcessor@@@8 10040988     SingleTableProcessor.obj
 0003:000009ac       ??_R0?AVSingleTableProcessor2@@@8 100409ac     SingleTableProcessor2.obj
 0003:000009d0       ??_R0?AVThaiLayoutEngine@@@8 100409d0     ThaiLayoutEngine.obj
 0003:000009f0       ??_R0?AVTibetanOpenTypeLayoutEngine@@@8 100409f0     TibetanLayoutEngine.obj
 0003:00000a1c       ??_R0?AVTrimmedArrayProcessor@@@8 10040a1c     TrimmedArrayProcessor.obj
 0003:00000a40       ??_R0?AVTrimmedArrayProcessor2@@@8 10040a40     TrimmedArrayProcessor2.obj
 0003:00000a68       ??_R0?AVtype_info@@@8      10040a68     MSVCRT:std_type_info_static.obj
 0003:00000cb8       ___isa_available           10040cb8     MSVCRT:cpu_disp.obj
 0003:00000cbc       ___favor                   10040cbc     MSVCRT:cpu_disp.obj
 0003:00000fe0       ?__type_info_root_node@@3U__type_info_node@@A 10040fe0     MSVCRT:tncleanup.obj
 0003:00000fe8       ?_OptionsStorage@?1??__local_stdio_printf_options@@9@4_KA 10040fe8     MSVCRT:default_local_stdio_options.obj
 0003:00000ff0       ?_OptionsStorage@?1??__local_stdio_scanf_options@@9@4_KA 10040ff0     MSVCRT:default_local_stdio_options.obj
 0003:00000ff8       ___scrt_current_native_startup_state 10040ff8     MSVCRT:utility.obj
 0003:00000ffc       ___scrt_native_startup_lock 10040ffc     MSVCRT:utility.obj
 0003:0000101c       ___scrt_debugger_hook_flag 1004101c     MSVCRT:utility_desktop.obj
 0003:00001020       _sunFontIDs                10041020     <common>
 0003:000010c0       _lcdInvGammaLUT            100410c0     <common>
 0003:00001320       _lcdGammaLUT               10041320     <common>
 0003:0000157c       ___dyn_tls_init_callback   1004157c     <common>

 entry point at        0001:0002755c

 Static symbols

 0000:fffbb000       .debug$S                   10000000     fontmanager.exp
 0000:fffbb000       .debug$S                   10000000     vcruntime:VCRUNTIME140.dll
 0000:fffbb000       .debug$S                   10000000     vcruntime:VCRUNTIME140.dll
 0000:fffbb000       .debug$S                   10000000     vcruntime:VCRUNTIME140.dll
 0000:fffbb000       .debug$S                   10000000     vcruntime:VCRUNTIME140.dll
 0000:fffbb000       .debug$S                   10000000     vcruntime:VCRUNTIME140.dll
 0000:fffbb000       .debug$S                   10000000     vcruntime:VCRUNTIME140.dll
 0000:fffbb000       .debug$S                   10000000     vcruntime:VCRUNTIME140.dll
 0000:fffbb000       .debug$S                   10000000     vcruntime:VCRUNTIME140.dll
 0000:fffbb000       .debug$S                   10000000     vcruntime:VCRUNTIME140.dll
 0000:fffbb000       .debug$S                   10000000     vcruntime:VCRUNTIME140.dll
 0000:fffbb000       .debug$S                   10000000     vcruntime:VCRUNTIME140.dll
 0000:fffbb000       .debug$S                   10000000     vcruntime:VCRUNTIME140.dll
 0000:fffbb000       .debug$S                   10000000     vcruntime:VCRUNTIME140.dll
 0000:fffbb000       .debug$S                   10000000     vcruntime:VCRUNTIME140.dll
 0000:fffbb000       .debug$S                   10000000     ucrt:api-ms-win-crt-environment-l1-1-0.dll
 0000:fffbb000       .debug$S                   10000000     ucrt:api-ms-win-crt-heap-l1-1-0.dll
 0000:fffbb000       .debug$S                   10000000     ucrt:api-ms-win-crt-heap-l1-1-0.dll
 0000:fffbb000       .debug$S                   10000000     ucrt:api-ms-win-crt-heap-l1-1-0.dll
 0000:fffbb000       .debug$S                   10000000     ucrt:api-ms-win-crt-heap-l1-1-0.dll
 0000:fffbb000       .debug$S                   10000000     ucrt:api-ms-win-crt-heap-l1-1-0.dll
 0000:fffbb000       .debug$S                   10000000     ucrt:api-ms-win-crt-math-l1-1-0.dll
 0000:fffbb000       .debug$S                   10000000     ucrt:api-ms-win-crt-math-l1-1-0.dll
 0000:fffbb000       .debug$S                   10000000     ucrt:api-ms-win-crt-math-l1-1-0.dll
 0000:fffbb000       .debug$S                   10000000     ucrt:api-ms-win-crt-math-l1-1-0.dll
 0000:fffbb000       .debug$S                   10000000     ucrt:api-ms-win-crt-runtime-l1-1-0.dll
 0000:fffbb000       .debug$S                   10000000     ucrt:api-ms-win-crt-runtime-l1-1-0.dll
 0000:fffbb000       .debug$S                   10000000     ucrt:api-ms-win-crt-runtime-l1-1-0.dll
 0000:fffbb000       .debug$S                   10000000     ucrt:api-ms-win-crt-runtime-l1-1-0.dll
 0000:fffbb000       .debug$S                   10000000     ucrt:api-ms-win-crt-runtime-l1-1-0.dll
 0000:fffbb000       .debug$S                   10000000     ucrt:api-ms-win-crt-runtime-l1-1-0.dll
 0000:fffbb000       .debug$S                   10000000     ucrt:api-ms-win-crt-runtime-l1-1-0.dll
 0000:fffbb000       .debug$S                   10000000     ucrt:api-ms-win-crt-runtime-l1-1-0.dll
 0000:fffbb000       .debug$S                   10000000     ucrt:api-ms-win-crt-runtime-l1-1-0.dll
 0000:fffbb000       .debug$S                   10000000     ucrt:api-ms-win-crt-runtime-l1-1-0.dll
 0000:fffbb000       .debug$S                   10000000     ucrt:api-ms-win-crt-runtime-l1-1-0.dll
 0000:fffbb000       .debug$S                   10000000     ucrt:api-ms-win-crt-runtime-l1-1-0.dll
 0000:fffbb000       .debug$S                   10000000     ucrt:api-ms-win-crt-string-l1-1-0.dll
 0000:fffbb000       .debug$S                   10000000     ucrt:api-ms-win-crt-string-l1-1-0.dll
 0000:fffbb000       .debug$S                   10000000     advapi32:ADVAPI32.dll
 0000:fffbb000       .debug$S                   10000000     advapi32:ADVAPI32.dll
 0000:fffbb000       .debug$S                   10000000     advapi32:ADVAPI32.dll
 0000:fffbb000       .debug$S                   10000000     advapi32:ADVAPI32.dll
 0000:fffbb000       .debug$S                   10000000     advapi32:ADVAPI32.dll
 0000:fffbb000       .debug$S                   10000000     advapi32:ADVAPI32.dll
 0000:fffbb000       .debug$S                   10000000     gdi32:GDI32.dll
 0000:fffbb000       .debug$S                   10000000     gdi32:GDI32.dll
 0000:fffbb000       .debug$S                   10000000     gdi32:GDI32.dll
 0000:fffbb000       .debug$S                   10000000     gdi32:GDI32.dll
 0000:fffbb000       .debug$S                   10000000     gdi32:GDI32.dll
 0000:fffbb000       .debug$S                   10000000     gdi32:GDI32.dll
 0000:fffbb000       .debug$S                   10000000     gdi32:GDI32.dll
 0000:fffbb000       .debug$S                   10000000     gdi32:GDI32.dll
 0000:fffbb000       .debug$S                   10000000     gdi32:GDI32.dll
 0000:fffbb000       .debug$S                   10000000     gdi32:GDI32.dll
 0000:fffbb000       .debug$S                   10000000     gdi32:GDI32.dll
 0000:fffbb000       .debug$S                   10000000     gdi32:GDI32.dll
 0000:fffbb000       .debug$S                   10000000     gdi32:GDI32.dll
 0000:fffbb000       .debug$S                   10000000     gdi32:GDI32.dll
 0000:fffbb000       .debug$S                   10000000     gdi32:GDI32.dll
 0000:fffbb000       .debug$S                   10000000     gdi32:GDI32.dll
 0000:fffbb000       .debug$S                   10000000     gdi32:GDI32.dll
 0000:fffbb000       .debug$S                   10000000     kernel32:KERNEL32.dll
 0000:fffbb000       .debug$S                   10000000     kernel32:KERNEL32.dll
 0000:fffbb000       .debug$S                   10000000     kernel32:KERNEL32.dll
 0000:fffbb000       .debug$S                   10000000     kernel32:KERNEL32.dll
 0000:fffbb000       .debug$S                   10000000     kernel32:KERNEL32.dll
 0000:fffbb000       .debug$S                   10000000     kernel32:KERNEL32.dll
 0000:fffbb000       .debug$S                   10000000     kernel32:KERNEL32.dll
 0000:fffbb000       .debug$S                   10000000     kernel32:KERNEL32.dll
 0000:fffbb000       .debug$S                   10000000     kernel32:KERNEL32.dll
 0000:fffbb000       .debug$S                   10000000     kernel32:KERNEL32.dll
 0000:fffbb000       .debug$S                   10000000     kernel32:KERNEL32.dll
 0000:fffbb000       .debug$S                   10000000     kernel32:KERNEL32.dll
 0000:fffbb000       .debug$S                   10000000     kernel32:KERNEL32.dll
 0000:fffbb000       .debug$S                   10000000     kernel32:KERNEL32.dll
 0000:fffbb000       .debug$S                   10000000     kernel32:KERNEL32.dll
 0000:fffbb000       .debug$S                   10000000     kernel32:KERNEL32.dll
 0000:fffbb000       .debug$S                   10000000     kernel32:KERNEL32.dll
 0000:fffbb000       .debug$S                   10000000     kernel32:KERNEL32.dll
 0000:fffbb000       .debug$S                   10000000     user32:USER32.dll
 0000:fffbb000       .debug$S                   10000000     user32:USER32.dll
 0000:fffbb000       .debug$S                   10000000     user32:USER32.dll
 0000:fffbb000       .debug$S                   10000000     user32:USER32.dll
 0000:fffbb000       .debug$S                   10000000     user32:USER32.dll
 0000:fffbb000       .debug$S                   10000000     user32:USER32.dll
 0000:fffbb000       .debug$S                   10000000     awt:awt.dll
 0000:fffbb000       .debug$S                   10000000     awt:awt.dll
 0000:fffbb000       .debug$S                   10000000     awt:awt.dll
 0000:fffbb000       .debug$S                   10000000     awt:awt.dll
 0000:fffbb000       .debug$S                   10000000     awt:awt.dll
 0000:fffbb000       .debug$S                   10000000     awt:awt.dll
 0000:fffbb000       .debug$S                   10000000     awt:awt.dll
 0000:fffbb000       .debug$S                   10000000     awt:awt.dll
 0000:fffbb000       .debug$S                   10000000     awt:awt.dll
 0000:fffbb000       .debug$S                   10000000     freetype:freetype.dll
 0000:fffbb000       .debug$S                   10000000     freetype:freetype.dll
 0000:fffbb000       .debug$S                   10000000     freetype:freetype.dll
 0000:fffbb000       .debug$S                   10000000     freetype:freetype.dll
 0000:fffbb000       .debug$S                   10000000     freetype:freetype.dll
 0000:fffbb000       .debug$S                   10000000     freetype:freetype.dll
 0000:fffbb000       .debug$S                   10000000     freetype:freetype.dll
 0000:fffbb000       .debug$S                   10000000     freetype:freetype.dll
 0000:fffbb000       .debug$S                   10000000     freetype:freetype.dll
 0000:fffbb000       .debug$S                   10000000     freetype:freetype.dll
 0000:fffbb000       .debug$S                   10000000     freetype:freetype.dll
 0000:fffbb000       .debug$S                   10000000     freetype:freetype.dll
 0000:fffbb000       .debug$S                   10000000     freetype:freetype.dll
 0000:fffbb000       .debug$S                   10000000     freetype:freetype.dll
 0000:fffbb000       .debug$S                   10000000     freetype:freetype.dll
 0000:fffbb000       .debug$S                   10000000     freetype:freetype.dll
 0000:fffbb000       .debug$S                   10000000     freetype:freetype.dll
 0000:fffbb000       .debug$S                   10000000     freetype:freetype.dll
 0000:fffbb000       .debug$S                   10000000     freetype:freetype.dll
 0000:fffbb000       .debug$S                   10000000     freetype:freetype.dll
 0000:fffbb000       .debug$S                   10000000     java:java.dll
 0000:fffbb000       .debug$S                   10000000     java:java.dll
 0000:fffbb000       .debug$S                   10000000     java:java.dll
 0001:00005c50       $LN179                     10006c50     ContextualSubstSubtables.obj
 0001:00007138       $LN325                     10008138     ContextualSubstSubtables.obj
 0001:00007cb0       _drawGlyphList             10008cb0 f   DrawGlyphList.obj
 0001:00007e20       _drawGlyphListLCD          10008e20 f   DrawGlyphList.obj
 0001:0000a270       $LN42                      1000b270     GlyphIterator.obj
 0001:0000a4e8       $LN46                      1000b4e8     GlyphIterator.obj
 0001:0000a688       $LN46                      1000b688     GlyphIterator.obj
 0001:0000b70c       $LN413                     1000c70c     GlyphPosnLookupProc.obj
 0001:0000bc48       $LN323                     1000cc48     GlyphSubstLookupProc.obj
 0001:0000d614       $LN315                     1000e614     IndicRearrangementProcessor.obj
 0001:0000e508       $LN315                     1000f508     IndicRearrangementProcessor2.obj
 0001:000103a0       $LN449                     100113a0     IndicReordering.obj
 0001:000103b8       $LN448                     100113b8     IndicReordering.obj
 0001:00013de8       $LN209                     10014de8     LayoutEngine.obj
 0001:00013e08       $LN208                     10014e08     LayoutEngine.obj
 0001:00013e30       $LN211                     10014e30     LayoutEngine.obj
 0001:00013e38       $LN210                     10014e38     LayoutEngine.obj
 0001:00013e50       $LN213                     10014e50     LayoutEngine.obj
 0001:00013e64       $LN212                     10014e64     LayoutEngine.obj
 0001:0001a2ac       $LN269                     1001b2ac     MorphTables.obj
 0001:0001aba4       $LN384                     1001bba4     MorphTables2.obj
 0001:0001abc8       $LN383                     1001bbc8     MorphTables2.obj
 0001:0001abe4       $LN385                     1001bbe4     MorphTables2.obj
 0001:0001b1c8       $LN74                      1001c1c8     NonContextualGlyphSubstProc.obj
 0001:0001b368       $LN74                      1001c368     NonContextualGlyphSubstProc2.obj
 0001:0001bed4       $LN16                      1001ced4     OpenTypeLayoutEngine.obj
 0001:0001befc       $LN15                      1001cefc     OpenTypeLayoutEngine.obj
 0001:0001c1b0       $LN26                      1001d1b0     OpenTypeLayoutEngine.obj
 0001:0001c1d8       $LN25                      1001d1d8     OpenTypeLayoutEngine.obj
 0001:00021404       $LN63                      10022404     ThaiShaping.obj
 0001:0002140c       $LN62                      1002240c     ThaiShaping.obj
 0001:00021784       $LN38                      10022784     ThaiShaping.obj
 0001:00022d60       _CheckFontFamilyProcW@16   10023d60 f   fontpath.obj
 0001:00022db0       _EnumFamilyNamesA@16       10023db0 f   fontpath.obj
 0001:00022ee0       _EnumFamilyNamesW@16       10023ee0 f   fontpath.obj
 0001:00023050       _EnumFontFacesInFamilyProcA@16 10024050 f   fontpath.obj
 0001:000230e0       _EnumFontFacesInFamilyProcW@16 100240e0 f   fontpath.obj
 0001:00023260       _GetOSVersion              10024260 f   fontpath.obj
 0001:00023cd0       _registerFontW             10024cd0 f   fontpath.obj
 0001:00023e50       _moveTo                    10024e50 f   freetypeScaler.obj
 0001:00023ec0       _lineTo                    10024ec0 f   freetypeScaler.obj
 0001:00023f20       _conicTo                   10024f20 f   freetypeScaler.obj
 0001:00023fc0       _cubicTo                   10024fc0 f   freetypeScaler.obj
 0001:000250c0       _ReadTTFontFileFunc        100260c0 f   freetypeScaler.obj
 0001:00025220       _getFTOutline              10026220 f   freetypeScaler.obj
 0001:000252e0       _getGlyphGeneralPath       100262e0 f   freetypeScaler.obj
 0001:000254a0       _getGlyphImageNativeInternal 100264a0 f   freetypeScaler.obj
 0001:00025ae0       _invalidateJavaScaler      10026ae0 f   freetypeScaler.obj
 0001:00025b60       _setupFTContext            10026b60 f   freetypeScaler.obj
 0001:00026980       _initFontIDs               10027980 f   sunFont.obj
 0001:00027090       $$000000                   10028090     MSVCRT:ftol2.obj
 0001:000270a0       $$000000                   100280a0     MSVCRT:ftol2.obj
 0001:000270b1       L3B                        100280b1     MSVCRT:ftol2.obj
 0001:000270f4       L3F                        100280f4     MSVCRT:ftol2.obj
 0001:000270fc       L40                        100280fc     MSVCRT:ftol2.obj
 0001:0002710f       L41                        1002810f     MSVCRT:ftol2.obj
 0001:00027180       $$000000                   10028180     MSVCRT:ftol3.obj
 0001:0002719f       _ftol3_default             1002819f     MSVCRT:ftol3.obj
 0001:000271b3       _ftol3_notsafe             100281b3     MSVCRT:ftol3.obj
 0001:000271d3       _ftol3_mincheck            100281d3     MSVCRT:ftol3.obj
 0001:000271d9       _ftol3_NaN                 100281d9     MSVCRT:ftol3.obj
 0001:000271e1       _ftol3_retmin              100281e1     MSVCRT:ftol3.obj
 0001:000271f0       $$000000                   100281f0     MSVCRT:alloca16.obj
 0001:00027206       alloca_8                   10028206     MSVCRT:alloca16.obj
 0001:0002721c       ?dllmain_crt_dispatch@@YGHQAUHINSTANCE__@@KQAX@Z 1002821c f   MSVCRT:dll_dllmain.obj
 0001:0002726f       ?dllmain_crt_process_attach@@YAHQAUHINSTANCE__@@QAX@Z 1002826f f   MSVCRT:dll_dllmain.obj
 0001:00027376       ?dllmain_crt_process_detach@@YAH_N@Z 10028376 f   MSVCRT:dll_dllmain.obj
 0001:00027426       ?dllmain_dispatch@@YAHQAUHINSTANCE__@@KQAX@Z 10028426 f   MSVCRT:dll_dllmain.obj
 0001:00027531       ?dllmain_raw@@YGHQAUHINSTANCE__@@KQAX@Z 10028531 f   MSVCRT:dll_dllmain.obj
 0001:000279a0       $$000000                   100289a0     MSVCRT:chkstk.obj
 0001:000279b4       cs10                       100289b4     MSVCRT:chkstk.obj
 0001:000279c2       cs20                       100289c2     MSVCRT:chkstk.obj
 0001:000279cb       ___get_entropy             100289cb f   MSVCRT:gs_support.obj
 0001:00027ac6       ?find_pe_section@@YAPAU_IMAGE_SECTION_HEADER@@QAEI@Z 10028ac6 f   MSVCRT:utility.obj
 0001:00027f20       $$000000                   10028f20     MSVCRT:sehprolg4.obj
 0002:000002a8       ?featureMap@@3QBUFeatureMap@@B 1002a2a8     ArabicShaping.obj
 0002:0000e480       ?cacheMap@@3QBKB           10038480     FontInstanceAdapter.obj
 0002:0000e660       ?featureMap@@3QBUFeatureMap@@B 10038660     HanLayoutEngine.obj
 0002:0000e6b8       ?stateTable@@3QAY05$$CBUStateTransition@@A 100386b8     HangulLayoutEngine.obj
 0002:0000e7a8       ?featureMap@@3QBUFeatureMap@@B 100387a8     HangulLayoutEngine.obj
 0002:0000e808       ?devaCharClasses@@3QBKB    10038808     IndicClassTables.obj
 0002:0000e9cc       ?bengSplitTable@@3QAY02$$CBGA 100389cc     IndicClassTables.obj
 0002:0000e9d8       ?bengCharClasses@@3QBKB    100389d8     IndicClassTables.obj
 0002:0000ebc4       ?oryaSplitTable@@3QAY02$$CBGA 10038bc4     IndicClassTables.obj
 0002:0000ebd8       ?punjCharClasses@@3QBKB    10038bd8     IndicClassTables.obj
 0002:0000edb0       ?gujrCharClasses@@3QBKB    10038db0     IndicClassTables.obj
 0002:0000ef70       ?oryaCharClasses@@3QBKB    10038f70     IndicClassTables.obj
 0002:0000f138       ?tamlCharClasses@@3QBKB    10039138     IndicClassTables.obj
 0002:0000f308       ?teluCharClasses@@3QBKB    10039308     IndicClassTables.obj
 0002:0000f4c8       ?kndaCharClasses@@3QBKB    100394c8     IndicClassTables.obj
 0002:0000f688       ?mlymCharClasses@@3QBKB    10039688     IndicClassTables.obj
 0002:0000f848       ?sinhCharClasses@@3QBKB    10039848     IndicClassTables.obj
 0002:0000fa1c       ?tamlSplitTable@@3QAY02$$CBGA 10039a1c     IndicClassTables.obj
 0002:0000fa30       ?teluSplitTable@@3QAY02$$CBGA 10039a30     IndicClassTables.obj
 0002:0000fa38       ?kndaSplitTable@@3QAY02$$CBGA 10039a38     IndicClassTables.obj
 0002:0000fa58       ?mlymSplitTable@@3QAY02$$CBGA 10039a58     IndicClassTables.obj
 0002:0000fa6c       ?sinhSplitTable@@3QAY02$$CBGA 10039a6c     IndicClassTables.obj
 0002:0000fa84       ?devaClassTable@@3UIndicClassTable@@B 10039a84     IndicClassTables.obj
 0002:0000fa98       ?bengClassTable@@3UIndicClassTable@@B 10039a98     IndicClassTables.obj
 0002:0000faac       ?punjClassTable@@3UIndicClassTable@@B 10039aac     IndicClassTables.obj
 0002:0000fac0       ?gujrClassTable@@3UIndicClassTable@@B 10039ac0     IndicClassTables.obj
 0002:0000fad4       ?oryaClassTable@@3UIndicClassTable@@B 10039ad4     IndicClassTables.obj
 0002:0000fae8       ?tamlClassTable@@3UIndicClassTable@@B 10039ae8     IndicClassTables.obj
 0002:0000fafc       ?teluClassTable@@3UIndicClassTable@@B 10039afc     IndicClassTables.obj
 0002:0000fb10       ?kndaClassTable@@3UIndicClassTable@@B 10039b10     IndicClassTables.obj
 0002:0000fb24       ?mlymClassTable@@3UIndicClassTable@@B 10039b24     IndicClassTables.obj
 0002:0000fb38       ?sinhClassTable@@3UIndicClassTable@@B 10039b38     IndicClassTables.obj
 0002:0000fb50       ?indicClassTables@@3QBQBUIndicClassTable@@B 10039b50     IndicClassTables.obj
 0002:0000fe48       ?featureMap@@3QBUFeatureMap@@B 10039e48     IndicReordering.obj
 0002:0000fed0       ?v2FeatureMap@@3QBUFeatureMap@@B 10039ed0     IndicReordering.obj
 0002:0000ff68       ?stateTable@@3QAY0BA@$$CBCA 10039f68     IndicReordering.obj
 0002:00010088       ?khmerCharClasses@@3QBKB   1003a088     KhmerReordering.obj
 0002:00010208       ?khmerClassTable@@3UKhmerClassTable@@B 1003a208     KhmerReordering.obj
 0002:00010210       ?featureMap@@3QBUFeatureMap@@B 1003a210     KhmerReordering.obj
 0002:00010278       ?khmerStateTable@@3QAY0M@$$CBCA 1003a278     KhmerReordering.obj
 0002:00010448       ?canonFeatureMap@@3QBUFeatureMap@@B 1003a448     LayoutEngine.obj
 0002:00010f78       ?featureMap@@3QBUFeatureMap@@B 1003af78     OpenTypeLayoutEngine.obj
 0002:00011ac0       ?leftAboveVowels@?1??leftAboveVowel@ThaiShaping@@CAGGE@Z@4QAY06$$CBGA 1003bac0     ThaiShaping.obj
 0002:00011af8       ?lowerRightTones@?1??lowerRightTone@ThaiShaping@@CAGGE@Z@4QAY06$$CBGA 1003baf8     ThaiShaping.obj
 0002:00011b30       ?lowerLeftTones@?1??lowerLeftTone@ThaiShaping@@CAGGE@Z@4QAY06$$CBGA 1003bb30     ThaiShaping.obj
 0002:00011b68       ?upperLeftTones@?1??upperLeftTone@ThaiShaping@@CAGGE@Z@4QAY06$$CBGA 1003bb68     ThaiShaping.obj
 0002:00011ba0       ?lowerBelowVowels@?1??lowerBelowVowel@ThaiShaping@@CAGGE@Z@4QAY02$$CBGA 1003bba0     ThaiShaping.obj
 0002:00011bb8       ?noDescenderCODs@?1??noDescenderCOD@ThaiShaping@@CAGGE@Z@4QAY03$$CBGA 1003bbb8     ThaiShaping.obj
 0002:00012430       ?tibetanCharClasses@@3QBKB 1003c430     TibetanReordering.obj
 0002:00012830       ?tibetanClassTable@@3UTibetanClassTable@@B 1003c830     TibetanReordering.obj
 0002:00012838       ?featureMap@@3QBUFeatureMap@@B 1003c838     TibetanReordering.obj
 0002:000128a8       ?tibetanStateTable@@3QAY0BB@$$CBCA 1003c8a8     TibetanReordering.obj
 0002:00012a40       ?bitsInNibble@?1??getFieldCount@ValueRecord@@CAFG@Z@4QBFB 1003ca40     ValueRecords.obj
 0002:00012a64       _FONTKEY_NT                1003ca64     fontpath.obj
 0002:00012a98       _FONTKEY_WIN               1003ca98     fontpath.obj
 0002:00012ac8       ?TTSUFFIX@?1??RegistryToBaseTTNameA@@9@9 1003cac8     fontpath.obj
 0002:00012ad4       ?OTSUFFIX@?1??RegistryToBaseTTNameA@@9@9 1003cad4     fontpath.obj
 0002:00012ae0       ?TTSUFFIX@?1??RegistryToBaseTTNameW@@9@9 1003cae0     fontpath.obj
 0002:00012af8       ?OTSUFFIX@?1??RegistryToBaseTTNameW@@9@9 1003caf8     fontpath.obj
 0002:00012c40       ?outline_funcs@?1??addToGP@@9@9 1003cc40     freetypeScaler.obj
 0002:00013010       two32                      1003d010     MSVCRT:ftol2.obj
 0002:00013014       two63                      1003d014     MSVCRT:ftol2.obj
 0002:00013018       two64                      1003d018     MSVCRT:ftol2.obj
 0002:0001301c       _NaN                       1003d01c     MSVCRT:ftol2.obj
 0002:00013030       _NaN                       1003d030     MSVCRT:ftol3.obj
 0002:00013034       _onept5                    1003d034     MSVCRT:ftol3.obj
 0002:00013038       _DP2to32                   1003d038     MSVCRT:ftol3.obj
 0002:00013038       _Int32ToUInt32             1003d038     MSVCRT:ftol3.obj
 0002:000130ac       _GS_ExceptionPointers      1003d0ac     MSVCRT:gs_report.obj
 0002:00014780       __sehtable$?dllmain_crt_process_attach@@YAHQAUHINSTANCE__@@QAX@Z 1003e780     MSVCRT:dll_dllmain.obj
 0002:000147a0       __sehtable$?dllmain_crt_process_detach@@YAH_N@Z 1003e7a0     MSVCRT:dll_dllmain.obj
 0002:000147c8       __sehtable$?dllmain_dispatch@@YAHQAUHINSTANCE__@@KQAX@Z 1003e7c8     MSVCRT:dll_dllmain.obj
 0002:00014878       __sehtable$___scrt_is_nonwritable_in_current_image 1003e878     MSVCRT:utility.obj
 0002:000148a0       .edata                     1003e8a0     fontmanager.exp
 0002:000148c8       rgpv                       1003e8c8     fontmanager.exp
 0002:00014960       rgszName                   1003e960     fontmanager.exp
 0002:000149f8       rgwOrd                     1003e9f8     fontmanager.exp
 0002:00014a44       szName                     1003ea44     fontmanager.exp
 0002:00014a54       $N00001                    1003ea54     fontmanager.exp
 0002:00014a82       $N00002                    1003ea82     fontmanager.exp
 0002:00014abd       $N00003                    1003eabd     fontmanager.exp
 0002:00014af9       $N00004                    1003eaf9     fontmanager.exp
 0002:00014b24       $N00005                    1003eb24     fontmanager.exp
 0002:00014b63       $N00006                    1003eb63     fontmanager.exp
 0002:00014b9c       $N00007                    1003eb9c     fontmanager.exp
 0002:00014bd6       $N00008                    1003ebd6     fontmanager.exp
 0002:00014c11       $N00009                    1003ec11     fontmanager.exp
 0002:00014c49       $N00010                    1003ec49     fontmanager.exp
 0002:00014c82       $N00011                    1003ec82     fontmanager.exp
 0002:00014cbd       $N00012                    1003ecbd     fontmanager.exp
 0002:00014cfe       $N00013                    1003ecfe     fontmanager.exp
 0002:00014d39       $N00014                    1003ed39     fontmanager.exp
 0002:00014d72       $N00015                    1003ed72     fontmanager.exp
 0002:00014db3       $N00016                    1003edb3     fontmanager.exp
 0002:00014df2       $N00017                    1003edf2     fontmanager.exp
 0002:00014e31       $N00018                    1003ee31     fontmanager.exp
 0002:00014e69       $N00019                    1003ee69     fontmanager.exp
 0002:00014ea2       $N00020                    1003eea2     fontmanager.exp
 0002:00014ecf       $N00021                    1003eecf     fontmanager.exp
 0002:00014f05       $N00022                    1003ef05     fontmanager.exp
 0002:00014f34       $N00023                    1003ef34     fontmanager.exp
 0002:00014f69       $N00024                    1003ef69     fontmanager.exp
 0002:00014f95       $N00025                    1003ef95     fontmanager.exp
 0002:00014fc2       $N00026                    1003efc2     fontmanager.exp
 0002:00014fef       $N00027                    1003efef     fontmanager.exp
 0002:0001501d       $N00028                    1003f01d     fontmanager.exp
 0002:00015054       $N00029                    1003f054     fontmanager.exp
 0002:0001507c       $N00030                    1003f07c     fontmanager.exp
 0002:000150a7       $N00031                    1003f0a7     fontmanager.exp
 0002:000150d6       $N00032                    1003f0d6     fontmanager.exp
 0002:00015110       $N00033                    1003f110     fontmanager.exp
 0002:0001514c       $N00034                    1003f14c     fontmanager.exp
 0002:00015182       $N00035                    1003f182     fontmanager.exp
 0002:00015197       $N00036                    1003f197     fontmanager.exp
 0002:000151a5       $N00037                    1003f1a5     fontmanager.exp
 0002:000151b9       $N00038                    1003f1b9     fontmanager.exp
 0002:0001565e       .idata$6                   1003f65e     freetype:freetype.dll
 0002:000156d2       .idata$6                   1003f6d2     java:java.dll
 0002:00015742       .idata$6                   1003f742     advapi32:ADVAPI32.dll
 0002:000157aa       .idata$6                   1003f7aa     user32:USER32.dll
 0002:000158e4       .idata$6                   1003f8e4     gdi32:GDI32.dll
 0002:000159f2       .idata$6                   1003f9f2     awt:awt.dll
 0002:00015b6a       .idata$6                   1003fb6a     kernel32:KERNEL32.dll
 0002:00015c42       .idata$6                   1003fc42     vcruntime:VCRUNTIME140.dll
 0002:00015d8a       .idata$6                   1003fd8a     ucrt:api-ms-win-crt-heap-l1-1-0.dll
 0002:00015daa       .idata$6                   1003fdaa     ucrt:api-ms-win-crt-math-l1-1-0.dll
 0002:00015dca       .idata$6                   1003fdca     ucrt:api-ms-win-crt-environment-l1-1-0.dll
 0002:00015df0       .idata$6                   1003fdf0     ucrt:api-ms-win-crt-runtime-l1-1-0.dll
 0002:00015e12       .idata$6                   1003fe12     ucrt:api-ms-win-crt-string-l1-1-0.dll
 0003:00000200       ?gvdClassName@@3PBDB       10040200     SunLayoutEngine.obj
 0003:00000a80       ?z@?1??getStaticClassID@ArabicOpenTypeLayoutEngine@@SAPBDXZ@4DA 10040a80     ArabicLayoutEngine.obj
 0003:00000a81       ?z@?1??getStaticClassID@ContextualGlyphInsertionProcessor2@@SAPBDXZ@4DA 10040a81     ContextualGlyphInsertionProc2.obj
 0003:00000a82       ?z@?1??getStaticClassID@ContextualGlyphSubstitutionProcessor@@SAPBDXZ@4DA 10040a82     ContextualGlyphSubstProc.obj
 0003:00000a83       ?z@?1??getStaticClassID@ContextualGlyphSubstitutionProcessor2@@SAPBDXZ@4DA 10040a83     ContextualGlyphSubstProc2.obj
 0003:00000a84       ?z@?1??getStaticClassID@GXLayoutEngine@@SAPBDXZ@4DA 10040a84     GXLayoutEngine.obj
 0003:00000a85       ?z@?1??getStaticClassID@GXLayoutEngine2@@SAPBDXZ@4DA 10040a85     GXLayoutEngine2.obj
 0003:00000a86       ?z@?1??getStaticClassID@HanOpenTypeLayoutEngine@@SAPBDXZ@4DA 10040a86     HanLayoutEngine.obj
 0003:00000a87       ?z@?1??getStaticClassID@HangulOpenTypeLayoutEngine@@SAPBDXZ@4DA 10040a87     HangulLayoutEngine.obj
 0003:00000a88       ?z@?1??getStaticClassID@IndicOpenTypeLayoutEngine@@SAPBDXZ@4DA 10040a88     IndicLayoutEngine.obj
 0003:00000a89       ?z@?1??getStaticClassID@IndicRearrangementProcessor@@SAPBDXZ@4DA 10040a89     IndicRearrangementProcessor.obj
 0003:00000a8a       ?z@?1??getStaticClassID@IndicRearrangementProcessor2@@SAPBDXZ@4DA 10040a8a     IndicRearrangementProcessor2.obj
 0003:00000a8b       ?z@?1??getStaticClassID@KhmerOpenTypeLayoutEngine@@SAPBDXZ@4DA 10040a8b     KhmerLayoutEngine.obj
 0003:00000a8c       ?z@?1??getStaticClassID@LEFontInstance@@SAPBDXZ@4DA 10040a8c     LEFontInstance.obj
 0003:00000a8d       ?z@?1??getStaticClassID@LEGlyphStorage@@SAPBDXZ@4DA 10040a8d     LEGlyphStorage.obj
 0003:00000a8e       ?z@?1??getStaticClassID@LEInsertionList@@SAPBDXZ@4DA 10040a8e     LEInsertionList.obj
 0003:00000a8f       ?z@?1??getStaticClassID@LayoutEngine@@SAPBDXZ@4DA 10040a8f     LayoutEngine.obj
 0003:00000a90       ?z@?1??getStaticClassID@LigatureSubstitutionProcessor@@SAPBDXZ@4DA 10040a90     LigatureSubstProc.obj
 0003:00000a91       ?z@?1??getStaticClassID@LigatureSubstitutionProcessor2@@SAPBDXZ@4DA 10040a91     LigatureSubstProc2.obj
 0003:00000a92       ?z@?1??getStaticClassID@OpenTypeLayoutEngine@@SAPBDXZ@4DA 10040a92     OpenTypeLayoutEngine.obj
 0003:00000a93       ?z@?1??getStaticClassID@SegmentArrayProcessor@@SAPBDXZ@4DA 10040a93     SegmentArrayProcessor.obj
 0003:00000a94       ?z@?1??getStaticClassID@SegmentArrayProcessor2@@SAPBDXZ@4DA 10040a94     SegmentArrayProcessor2.obj
 0003:00000a95       ?z@?1??getStaticClassID@SegmentSingleProcessor@@SAPBDXZ@4DA 10040a95     SegmentSingleProcessor.obj
 0003:00000a96       ?z@?1??getStaticClassID@SegmentSingleProcessor2@@SAPBDXZ@4DA 10040a96     SegmentSingleProcessor2.obj
 0003:00000a97       ?z@?1??getStaticClassID@SimpleArrayProcessor@@SAPBDXZ@4DA 10040a97     SimpleArrayProcessor.obj
 0003:00000a98       ?z@?1??getStaticClassID@SimpleArrayProcessor2@@SAPBDXZ@4DA 10040a98     SimpleArrayProcessor2.obj
 0003:00000a99       ?z@?1??getStaticClassID@SingleTableProcessor@@SAPBDXZ@4DA 10040a99     SingleTableProcessor.obj
 0003:00000a9a       ?z@?1??getStaticClassID@SingleTableProcessor2@@SAPBDXZ@4DA 10040a9a     SingleTableProcessor2.obj
 0003:00000a9c       ?gvdClass@@3PAV_jclass@@A  10040a9c     SunLayoutEngine.obj
 0003:00000aa0       ?gvdCountFID@@3PAU_jfieldID@@A 10040aa0     SunLayoutEngine.obj
 0003:00000aa4       ?gvdFlagsFID@@3PAU_jfieldID@@A 10040aa4     SunLayoutEngine.obj
 0003:00000aa8       ?gvdGlyphsFID@@3PAU_jfieldID@@A 10040aa8     SunLayoutEngine.obj
 0003:00000aac       ?gvdPositionsFID@@3PAU_jfieldID@@A 10040aac     SunLayoutEngine.obj
 0003:00000ab0       ?gvdIndicesFID@@3PAU_jfieldID@@A 10040ab0     SunLayoutEngine.obj
 0003:00000ab4       ?z@?1??getStaticClassID@ThaiLayoutEngine@@SAPBDXZ@4DA 10040ab4     ThaiLayoutEngine.obj
 0003:00000ab5       ?z@?1??getStaticClassID@TibetanOpenTypeLayoutEngine@@SAPBDXZ@4DA 10040ab5     TibetanLayoutEngine.obj
 0003:00000ab6       ?z@?1??getStaticClassID@TrimmedArrayProcessor@@SAPBDXZ@4DA 10040ab6     TrimmedArrayProcessor.obj
 0003:00000ab7       ?z@?1??getStaticClassID@TrimmedArrayProcessor2@@SAPBDXZ@4DA 10040ab7     TrimmedArrayProcessor2.obj
 0003:00000ab8       _UNICODE_OS                10040ab8     fontpath.obj
 0003:00000abc       _screenDC                  10040abc     fontpath.obj
 0003:00000ac0       _invalidateScalerMID       10040ac0     freetypeScaler.obj
 0003:00000ac8       _igLUTable                 10040ac8     lcdglyph.obj
 0003:00000cac       _theNullScalerContext      10040cac     sunFont.obj
 0003:00000cb0       _initialisedFontIDs        10040cb0     sunFont.obj
 0003:00000cb4       ?__proc_attached@@3HA      10040cb4     MSVCRT:dll_dllmain.obj
 0003:00000cc0       _GS_ExceptionRecord        10040cc0     MSVCRT:gs_report.obj
 0003:00000d10       _GS_ContextRecord          10040d10     MSVCRT:gs_report.obj
 0003:00001000       ?is_initialized_as_dll@@3_NA 10041000     MSVCRT:utility.obj
 0003:00001001       ?module_local_atexit_table_initialized@@3_NA 10041001     MSVCRT:utility.obj
 0003:00001004       ?module_local_atexit_table@@3U_onexit_table_t@@A 10041004     MSVCRT:utility.obj
 0003:00001010       ?module_local_at_quick_exit_table@@3U_onexit_table_t@@A 10041010     MSVCRT:utility.obj
 0004:00000060       $R000000                   10042060     fontmanager.dll.res
